
ASL_test.elf:     file format elf32-littlearm

Sections:
Idx Name          Size      VMA       LMA       File off  Algn
  0 .isr_vector   000001ac  08000000  08000000  00010000  2**0
                  CONTENTS, ALLOC, LOAD, READONLY, DATA
  1 .text         0000d33c  080001b0  080001b0  000101b0  2**3
                  CONTENTS, ALLOC, LOAD, READONLY, CODE
  2 .rodata       00020f38  0800d4ec  0800d4ec  0001d4ec  2**2
                  CONTENTS, ALLOC, LOAD, READONLY, DATA
  3 .ARM.extab    00000000  0802e424  0802e424  00040934  2**0
                  CONTENTS
  4 .ARM          00000008  0802e424  0802e424  0003e424  2**2
                  CONTENTS, ALLOC, LOAD, READONLY, DATA
  5 .preinit_array 00000000  0802e42c  0802e42c  00040934  2**0
                  CONTENTS, ALLOC, LOAD, DATA
  6 .init_array   00000004  0802e42c  0802e42c  0003e42c  2**2
                  CONTENTS, ALLOC, LOAD, DATA
  7 .fini_array   00000004  0802e430  0802e430  0003e430  2**2
                  CONTENTS, ALLOC, LOAD, DATA
  8 .data         00000934  20000000  0802e434  00040000  2**2
                  CONTENTS, ALLOC, LOAD, DATA
  9 .bss          00003d48  20000934  0802ed68  00040934  2**2
                  ALLOC
 10 ._user_heap_stack 00000604  2000467c  0802ed68  0004467c  2**0
                  ALLOC
 11 .ARM.attributes 00000034  00000000  00000000  00040934  2**0
                  CONTENTS, READONLY
 12 .debug_info   0000e30f  00000000  00000000  00040968  2**0
                  CONTENTS, READONLY, DEBUGGING
 13 .debug_abbrev 0000254c  00000000  00000000  0004ec77  2**0
                  CONTENTS, READONLY, DEBUGGING
 14 .debug_aranges 00000ae8  00000000  00000000  000511c8  2**3
                  CONTENTS, READONLY, DEBUGGING
 15 .debug_ranges 000009a0  00000000  00000000  00051cb0  2**3
                  CONTENTS, READONLY, DEBUGGING
 16 .debug_macro  00024bb5  00000000  00000000  00052650  2**0
                  CONTENTS, READONLY, DEBUGGING
 17 .debug_line   0000b4d4  00000000  00000000  00077205  2**0
                  CONTENTS, READONLY, DEBUGGING
 18 .debug_str    000dd4dc  00000000  00000000  000826d9  2**0
                  CONTENTS, READONLY, DEBUGGING
 19 .comment      000061a1  00000000  00000000  0015fbb5  2**0
                  CONTENTS, READONLY
 20 .iar.rtmodel  000001e7  00000000  00000000  00165d56  2**0
                  CONTENTS, READONLY
 21 .iar_vfe_header 00000024  00000000  00000000  00165f40  2**2
                  CONTENTS, READONLY
 22 .debug_frame  00007ad0  00000000  00000000  00165f64  2**2
                  CONTENTS, READONLY, DEBUGGING

Disassembly of section .text:

080001b0 <__do_global_dtors_aux>:
 80001b0:	b510      	push	{r4, lr}
 80001b2:	4c05      	ldr	r4, [pc, #20]	; (80001c8 <__do_global_dtors_aux+0x18>)
 80001b4:	7823      	ldrb	r3, [r4, #0]
 80001b6:	b933      	cbnz	r3, 80001c6 <__do_global_dtors_aux+0x16>
 80001b8:	4b04      	ldr	r3, [pc, #16]	; (80001cc <__do_global_dtors_aux+0x1c>)
 80001ba:	b113      	cbz	r3, 80001c2 <__do_global_dtors_aux+0x12>
 80001bc:	4804      	ldr	r0, [pc, #16]	; (80001d0 <__do_global_dtors_aux+0x20>)
 80001be:	f3af 8000 	nop.w
 80001c2:	2301      	movs	r3, #1
 80001c4:	7023      	strb	r3, [r4, #0]
 80001c6:	bd10      	pop	{r4, pc}
 80001c8:	20000934 	.word	0x20000934
 80001cc:	00000000 	.word	0x00000000
 80001d0:	0800d4d4 	.word	0x0800d4d4

080001d4 <frame_dummy>:
 80001d4:	b508      	push	{r3, lr}
 80001d6:	4b03      	ldr	r3, [pc, #12]	; (80001e4 <frame_dummy+0x10>)
 80001d8:	b11b      	cbz	r3, 80001e2 <frame_dummy+0xe>
 80001da:	4903      	ldr	r1, [pc, #12]	; (80001e8 <frame_dummy+0x14>)
 80001dc:	4803      	ldr	r0, [pc, #12]	; (80001ec <frame_dummy+0x18>)
 80001de:	f3af 8000 	nop.w
 80001e2:	bd08      	pop	{r3, pc}
 80001e4:	00000000 	.word	0x00000000
 80001e8:	20000938 	.word	0x20000938
 80001ec:	0800d4d4 	.word	0x0800d4d4

080001f0 <_ai_platform_get_io_buffers_info>:
 80001f0:	e92d 4ff2 	stmdb	sp!, {r1, r4, r5, r6, r7, r8, r9, sl, fp, lr}
 80001f4:	2500      	movs	r5, #0
 80001f6:	46aa      	mov	sl, r5
 80001f8:	b082      	sub	sp, #8
 80001fa:	4607      	mov	r7, r0
 80001fc:	46ab      	mov	fp, r5
 80001fe:	46d0      	mov	r8, sl
 8000200:	46d1      	mov	r9, sl
 8000202:	e028      	b.n	8000256 <_ai_platform_get_io_buffers_info+0x66>
 8000204:	2000      	movs	r0, #0
 8000206:	e01c      	b.n	8000242 <_ai_platform_get_io_buffers_info+0x52>
 8000208:	f850 400a 	ldr.w	r4, [r0, sl]
 800020c:	b364      	cbz	r4, 8000268 <_ai_platform_get_io_buffers_info+0x78>
 800020e:	68b8      	ldr	r0, [r7, #8]
 8000210:	6841      	ldr	r1, [r0, #4]
 8000212:	6880      	ldr	r0, [r0, #8]
 8000214:	4440      	add	r0, r8
 8000216:	eb01 0609 	add.w	r6, r1, r9
 800021a:	9000      	str	r0, [sp, #0]
 800021c:	69a1      	ldr	r1, [r4, #24]
 800021e:	6808      	ldr	r0, [r1, #0]
 8000220:	f005 fd58 	bl	8005cd4 <ai_array_to_buffer_fmt>
 8000224:	6030      	str	r0, [r6, #0]
 8000226:	2101      	movs	r1, #1
 8000228:	80b1      	strh	r1, [r6, #4]
 800022a:	68e0      	ldr	r0, [r4, #12]
 800022c:	68c1      	ldr	r1, [r0, #12]
 800022e:	80f1      	strh	r1, [r6, #6]
 8000230:	6882      	ldr	r2, [r0, #8]
 8000232:	8132      	strh	r2, [r6, #8]
 8000234:	6840      	ldr	r0, [r0, #4]
 8000236:	60f0      	str	r0, [r6, #12]
 8000238:	69a1      	ldr	r1, [r4, #24]
 800023a:	688a      	ldr	r2, [r1, #8]
 800023c:	6132      	str	r2, [r6, #16]
 800023e:	9800      	ldr	r0, [sp, #0]
 8000240:	b9e0      	cbnz	r0, 800027c <_ai_platform_get_io_buffers_info+0x8c>
 8000242:	6170      	str	r0, [r6, #20]
 8000244:	1c6d      	adds	r5, r5, #1
 8000246:	f10b 0b01 	add.w	fp, fp, #1
 800024a:	f109 0918 	add.w	r9, r9, #24
 800024e:	f108 0808 	add.w	r8, r8, #8
 8000252:	f10a 0a04 	add.w	sl, sl, #4
 8000256:	2f00      	cmp	r7, #0
 8000258:	bf14      	ite	ne
 800025a:	8838      	ldrhne	r0, [r7, #0]
 800025c:	2000      	moveq	r0, #0
 800025e:	4583      	cmp	fp, r0
 8000260:	d202      	bcs.n	8000268 <_ai_platform_get_io_buffers_info+0x78>
 8000262:	6878      	ldr	r0, [r7, #4]
 8000264:	2800      	cmp	r0, #0
 8000266:	d1cf      	bne.n	8000208 <_ai_platform_get_io_buffers_info+0x18>
 8000268:	b2a8      	uxth	r0, r5
 800026a:	b118      	cbz	r0, 8000274 <_ai_platform_get_io_buffers_info+0x84>
 800026c:	68b9      	ldr	r1, [r7, #8]
 800026e:	9802      	ldr	r0, [sp, #8]
 8000270:	684a      	ldr	r2, [r1, #4]
 8000272:	6002      	str	r2, [r0, #0]
 8000274:	b2a8      	uxth	r0, r5
 8000276:	b003      	add	sp, #12
 8000278:	e8bd 8ff0 	ldmia.w	sp!, {r4, r5, r6, r7, r8, r9, sl, fp, pc}
 800027c:	9900      	ldr	r1, [sp, #0]
 800027e:	2000      	movs	r0, #0
 8000280:	6008      	str	r0, [r1, #0]
 8000282:	9a00      	ldr	r2, [sp, #0]
 8000284:	6820      	ldr	r0, [r4, #0]
 8000286:	6050      	str	r0, [r2, #4]
 8000288:	2800      	cmp	r0, #0
 800028a:	bf1c      	itt	ne
 800028c:	8840      	ldrhne	r0, [r0, #2]
 800028e:	2800      	cmpne	r0, #0
 8000290:	d0b8      	beq.n	8000204 <_ai_platform_get_io_buffers_info+0x14>
 8000292:	9800      	ldr	r0, [sp, #0]
 8000294:	2101      	movs	r1, #1
 8000296:	6001      	str	r1, [r0, #0]
 8000298:	9800      	ldr	r0, [sp, #0]
 800029a:	e7d2      	b.n	8000242 <_ai_platform_get_io_buffers_info+0x52>

0800029c <_platform_network_state_setup>:
 800029c:	b430      	push	{r4, r5}
 800029e:	68d3      	ldr	r3, [r2, #12]
 80002a0:	6955      	ldr	r5, [r2, #20]
 80002a2:	68dc      	ldr	r4, [r3, #12]
 80002a4:	68eb      	ldr	r3, [r5, #12]
 80002a6:	435c      	muls	r4, r3
 80002a8:	6084      	str	r4, [r0, #8]
 80002aa:	888d      	ldrh	r5, [r1, #4]
 80002ac:	436c      	muls	r4, r5
 80002ae:	60c4      	str	r4, [r0, #12]
 80002b0:	6909      	ldr	r1, [r1, #16]
 80002b2:	68c3      	ldr	r3, [r0, #12]
 80002b4:	6041      	str	r1, [r0, #4]
 80002b6:	4419      	add	r1, r3
 80002b8:	6001      	str	r1, [r0, #0]
 80002ba:	6992      	ldr	r2, [r2, #24]
 80002bc:	6814      	ldr	r4, [r2, #0]
 80002be:	00a1      	lsls	r1, r4, #2
 80002c0:	d407      	bmi.n	80002d2 <_platform_network_state_setup+0x36>
 80002c2:	6894      	ldr	r4, [r2, #8]
 80002c4:	68d1      	ldr	r1, [r2, #12]
 80002c6:	6843      	ldr	r3, [r0, #4]
 80002c8:	1a64      	subs	r4, r4, r1
 80002ca:	1919      	adds	r1, r3, r4
 80002cc:	6091      	str	r1, [r2, #8]
 80002ce:	6840      	ldr	r0, [r0, #4]
 80002d0:	60d0      	str	r0, [r2, #12]
 80002d2:	bc30      	pop	{r4, r5}
 80002d4:	4770      	bx	lr

080002d6 <ai_platform_runtime_get_revision>:
 80002d6:	f8df 0814 	ldr.w	r0, [pc, #2068]	; 8000aec <.text_18>
 80002da:	6801      	ldr	r1, [r0, #0]
 80002dc:	0849      	lsrs	r1, r1, #1
 80002de:	0049      	lsls	r1, r1, #1
 80002e0:	6001      	str	r1, [r0, #0]
 80002e2:	2001      	movs	r0, #1
 80002e4:	f8df 1808 	ldr.w	r1, [pc, #2056]	; 8000af0 <.text_19>
 80002e8:	6088      	str	r0, [r1, #8]
 80002ea:	6888      	ldr	r0, [r1, #8]
 80002ec:	2800      	cmp	r0, #0
 80002ee:	d1fc      	bne.n	80002ea <ai_platform_runtime_get_revision+0x14>
 80002f0:	f8df 2800 	ldr.w	r2, [pc, #2048]	; 8000af4 <.text_20>
 80002f4:	600a      	str	r2, [r1, #0]
 80002f6:	6808      	ldr	r0, [r1, #0]
 80002f8:	f8df 17fc 	ldr.w	r1, [pc, #2044]	; 8000af8 <.text_21>
 80002fc:	4288      	cmp	r0, r1
 80002fe:	d000      	beq.n	8000302 <ai_platform_runtime_get_revision+0x2c>
 8000300:	e7fe      	b.n	8000300 <ai_platform_runtime_get_revision+0x2a>
 8000302:	a0ad      	add	r0, pc, #692	; (adr r0, 80005b8 <.text_13>)
 8000304:	4770      	bx	lr

08000306 <ai_platform_runtime_get_version>:
 8000306:	f8df 07e4 	ldr.w	r0, [pc, #2020]	; 8000aec <.text_18>
 800030a:	6801      	ldr	r1, [r0, #0]
 800030c:	0849      	lsrs	r1, r1, #1
 800030e:	0049      	lsls	r1, r1, #1
 8000310:	6001      	str	r1, [r0, #0]
 8000312:	2001      	movs	r0, #1
 8000314:	f8df 17d8 	ldr.w	r1, [pc, #2008]	; 8000af0 <.text_19>
 8000318:	6088      	str	r0, [r1, #8]
 800031a:	6888      	ldr	r0, [r1, #8]
 800031c:	2800      	cmp	r0, #0
 800031e:	d1fc      	bne.n	800031a <ai_platform_runtime_get_version+0x14>
 8000320:	f8df 27d0 	ldr.w	r2, [pc, #2000]	; 8000af4 <.text_20>
 8000324:	600a      	str	r2, [r1, #0]
 8000326:	6808      	ldr	r0, [r1, #0]
 8000328:	f8df 17cc 	ldr.w	r1, [pc, #1996]	; 8000af8 <.text_21>
 800032c:	4288      	cmp	r0, r1
 800032e:	d000      	beq.n	8000332 <ai_platform_runtime_get_version+0x2c>
 8000330:	e7fe      	b.n	8000330 <ai_platform_runtime_get_version+0x2a>
 8000332:	f20f 72d0 	addw	r2, pc, #2000	; 0x7d0
 8000336:	6810      	ldr	r0, [r2, #0]
 8000338:	4770      	bx	lr

0800033a <ai_platform_api_get_version>:
 800033a:	f8df 07b0 	ldr.w	r0, [pc, #1968]	; 8000aec <.text_18>
 800033e:	6801      	ldr	r1, [r0, #0]
 8000340:	0849      	lsrs	r1, r1, #1
 8000342:	0049      	lsls	r1, r1, #1
 8000344:	6001      	str	r1, [r0, #0]
 8000346:	2001      	movs	r0, #1
 8000348:	f8df 17a4 	ldr.w	r1, [pc, #1956]	; 8000af0 <.text_19>
 800034c:	6088      	str	r0, [r1, #8]
 800034e:	6888      	ldr	r0, [r1, #8]
 8000350:	2800      	cmp	r0, #0
 8000352:	d1fc      	bne.n	800034e <ai_platform_api_get_version+0x14>
 8000354:	f8df 279c 	ldr.w	r2, [pc, #1948]	; 8000af4 <.text_20>
 8000358:	600a      	str	r2, [r1, #0]
 800035a:	6808      	ldr	r0, [r1, #0]
 800035c:	f8df 1798 	ldr.w	r1, [pc, #1944]	; 8000af8 <.text_21>
 8000360:	4288      	cmp	r0, r1
 8000362:	d000      	beq.n	8000366 <ai_platform_api_get_version+0x2c>
 8000364:	e7fe      	b.n	8000364 <ai_platform_api_get_version+0x2a>
 8000366:	f20f 72a0 	addw	r2, pc, #1952	; 0x7a0
 800036a:	6810      	ldr	r0, [r2, #0]
 800036c:	4770      	bx	lr

0800036e <ai_platform_interface_api_get_version>:
 800036e:	f8df 077c 	ldr.w	r0, [pc, #1916]	; 8000aec <.text_18>
 8000372:	6801      	ldr	r1, [r0, #0]
 8000374:	0849      	lsrs	r1, r1, #1
 8000376:	0049      	lsls	r1, r1, #1
 8000378:	6001      	str	r1, [r0, #0]
 800037a:	2001      	movs	r0, #1
 800037c:	f8df 1770 	ldr.w	r1, [pc, #1904]	; 8000af0 <.text_19>
 8000380:	6088      	str	r0, [r1, #8]
 8000382:	6888      	ldr	r0, [r1, #8]
 8000384:	2800      	cmp	r0, #0
 8000386:	d1fc      	bne.n	8000382 <ai_platform_interface_api_get_version+0x14>
 8000388:	f8df 2768 	ldr.w	r2, [pc, #1896]	; 8000af4 <.text_20>
 800038c:	600a      	str	r2, [r1, #0]
 800038e:	6808      	ldr	r0, [r1, #0]
 8000390:	f8df 1764 	ldr.w	r1, [pc, #1892]	; 8000af8 <.text_21>
 8000394:	4288      	cmp	r0, r1
 8000396:	d000      	beq.n	800039a <ai_platform_interface_api_get_version+0x2c>
 8000398:	e7fe      	b.n	8000398 <ai_platform_interface_api_get_version+0x2a>
 800039a:	f20f 7270 	addw	r2, pc, #1904	; 0x770
 800039e:	6810      	ldr	r0, [r2, #0]
 80003a0:	4770      	bx	lr

080003a2 <ai_platform_context_acquire>:
 80003a2:	b120      	cbz	r0, 80003ae <ai_platform_context_acquire+0xc>
 80003a4:	6801      	ldr	r1, [r0, #0]
 80003a6:	f8df 2754 	ldr.w	r2, [pc, #1876]	; 8000afc <.text_22>
 80003aa:	4291      	cmp	r1, r2
 80003ac:	d000      	beq.n	80003b0 <ai_platform_context_acquire+0xe>
 80003ae:	2000      	movs	r0, #0
 80003b0:	f8df 1738 	ldr.w	r1, [pc, #1848]	; 8000aec <.text_18>
 80003b4:	680a      	ldr	r2, [r1, #0]
 80003b6:	0852      	lsrs	r2, r2, #1
 80003b8:	0052      	lsls	r2, r2, #1
 80003ba:	600a      	str	r2, [r1, #0]
 80003bc:	2101      	movs	r1, #1
 80003be:	f8df 2730 	ldr.w	r2, [pc, #1840]	; 8000af0 <.text_19>
 80003c2:	6091      	str	r1, [r2, #8]
 80003c4:	6891      	ldr	r1, [r2, #8]
 80003c6:	2900      	cmp	r1, #0
 80003c8:	d1fc      	bne.n	80003c4 <ai_platform_context_acquire+0x22>
 80003ca:	f8df 3728 	ldr.w	r3, [pc, #1832]	; 8000af4 <.text_20>
 80003ce:	6013      	str	r3, [r2, #0]
 80003d0:	6811      	ldr	r1, [r2, #0]
 80003d2:	f8df 2724 	ldr.w	r2, [pc, #1828]	; 8000af8 <.text_21>
 80003d6:	4291      	cmp	r1, r2
 80003d8:	d000      	beq.n	80003dc <ai_platform_context_acquire+0x3a>
 80003da:	e7fe      	b.n	80003da <ai_platform_context_acquire+0x38>
 80003dc:	4770      	bx	lr

080003de <ai_platform_context_release>:
 80003de:	f8df 171c 	ldr.w	r1, [pc, #1820]	; 8000afc <.text_22>
 80003e2:	6001      	str	r1, [r0, #0]
 80003e4:	4770      	bx	lr

080003e6 <ai_platform_network_get_error>:
 80003e6:	b120      	cbz	r0, 80003f2 <ai_platform_network_get_error+0xc>
 80003e8:	6801      	ldr	r1, [r0, #0]
 80003ea:	f8df 2710 	ldr.w	r2, [pc, #1808]	; 8000afc <.text_22>
 80003ee:	4291      	cmp	r1, r2
 80003f0:	d000      	beq.n	80003f4 <ai_platform_network_get_error+0xe>
 80003f2:	2000      	movs	r0, #0
 80003f4:	f8df 16f4 	ldr.w	r1, [pc, #1780]	; 8000aec <.text_18>
 80003f8:	680a      	ldr	r2, [r1, #0]
 80003fa:	0852      	lsrs	r2, r2, #1
 80003fc:	0052      	lsls	r2, r2, #1
 80003fe:	600a      	str	r2, [r1, #0]
 8000400:	2101      	movs	r1, #1
 8000402:	f8df 26ec 	ldr.w	r2, [pc, #1772]	; 8000af0 <.text_19>
 8000406:	6091      	str	r1, [r2, #8]
 8000408:	6891      	ldr	r1, [r2, #8]
 800040a:	2900      	cmp	r1, #0
 800040c:	d1fc      	bne.n	8000408 <ai_platform_network_get_error+0x22>
 800040e:	f8df 36e4 	ldr.w	r3, [pc, #1764]	; 8000af4 <.text_20>
 8000412:	6013      	str	r3, [r2, #0]
 8000414:	6811      	ldr	r1, [r2, #0]
 8000416:	f8df 26e0 	ldr.w	r2, [pc, #1760]	; 8000af8 <.text_21>
 800041a:	4291      	cmp	r1, r2
 800041c:	d000      	beq.n	8000420 <ai_platform_network_get_error+0x3a>
 800041e:	e7fe      	b.n	800041e <ai_platform_network_get_error+0x38>
 8000420:	2800      	cmp	r0, #0
 8000422:	bf1c      	itt	ne
 8000424:	3010      	addne	r0, #16
 8000426:	f000 bb83 	bne.w	8000b30 <core_get_error>
 800042a:	f20f 60f4 	addw	r0, pc, #1780	; 0x6f4
 800042e:	6800      	ldr	r0, [r0, #0]
 8000430:	4770      	bx	lr

08000432 <ai_platform_network_set_error>:
 8000432:	2800      	cmp	r0, #0
 8000434:	bf1c      	itt	ne
 8000436:	3010      	addne	r0, #16
 8000438:	f000 bb7f 	bne.w	8000b3a <core_set_error>
 800043c:	4770      	bx	lr

0800043e <ai_platform_api_get_network_report>:
 800043e:	e92d 4ff0 	stmdb	sp!, {r4, r5, r6, r7, r8, r9, sl, fp, lr}
 8000442:	ea5f 0900 	movs.w	r9, r0
 8000446:	b081      	sub	sp, #4
 8000448:	460c      	mov	r4, r1
 800044a:	d005      	beq.n	8000458 <ai_platform_api_get_network_report+0x1a>
 800044c:	f8d9 0000 	ldr.w	r0, [r9]
 8000450:	f8df 16a8 	ldr.w	r1, [pc, #1704]	; 8000afc <.text_22>
 8000454:	4288      	cmp	r0, r1
 8000456:	d001      	beq.n	800045c <ai_platform_api_get_network_report+0x1e>
 8000458:	f04f 0900 	mov.w	r9, #0
 800045c:	f8df 568c 	ldr.w	r5, [pc, #1676]	; 8000aec <.text_18>
 8000460:	f8df 668c 	ldr.w	r6, [pc, #1676]	; 8000af0 <.text_19>
 8000464:	6828      	ldr	r0, [r5, #0]
 8000466:	0840      	lsrs	r0, r0, #1
 8000468:	0040      	lsls	r0, r0, #1
 800046a:	6028      	str	r0, [r5, #0]
 800046c:	2101      	movs	r1, #1
 800046e:	60b1      	str	r1, [r6, #8]
 8000470:	68b0      	ldr	r0, [r6, #8]
 8000472:	2800      	cmp	r0, #0
 8000474:	d1fc      	bne.n	8000470 <ai_platform_api_get_network_report+0x32>
 8000476:	f8df 767c 	ldr.w	r7, [pc, #1660]	; 8000af4 <.text_20>
 800047a:	f8df 867c 	ldr.w	r8, [pc, #1660]	; 8000af8 <.text_21>
 800047e:	6037      	str	r7, [r6, #0]
 8000480:	6830      	ldr	r0, [r6, #0]
 8000482:	4540      	cmp	r0, r8
 8000484:	d000      	beq.n	8000488 <ai_platform_api_get_network_report+0x4a>
 8000486:	e7fe      	b.n	8000486 <ai_platform_api_get_network_report+0x48>
 8000488:	f1b9 0f00 	cmp.w	r9, #0
 800048c:	bf18      	it	ne
 800048e:	2c00      	cmpne	r4, #0
 8000490:	d034      	beq.n	80004fc <ai_platform_api_get_network_report+0xbe>
 8000492:	2000      	movs	r0, #0
 8000494:	66e0      	str	r0, [r4, #108]	; 0x6c
 8000496:	f8d9 2050 	ldr.w	r2, [r9, #80]	; 0x50
 800049a:	b152      	cbz	r2, 80004b2 <ai_platform_api_get_network_report+0x74>
 800049c:	e000      	b.n	80004a0 <ai_platform_api_get_network_report+0x62>
 800049e:	4602      	mov	r2, r0
 80004a0:	6ee1      	ldr	r1, [r4, #108]	; 0x6c
 80004a2:	1c49      	adds	r1, r1, #1
 80004a4:	66e1      	str	r1, [r4, #108]	; 0x6c
 80004a6:	68d0      	ldr	r0, [r2, #12]
 80004a8:	4282      	cmp	r2, r0
 80004aa:	bf18      	it	ne
 80004ac:	2800      	cmpne	r0, #0
 80004ae:	d1f6      	bne.n	800049e <ai_platform_api_get_network_report+0x60>
 80004b0:	b911      	cbnz	r1, 80004b8 <ai_platform_api_get_network_report+0x7a>
 80004b2:	2218      	movs	r2, #24
 80004b4:	2111      	movs	r1, #17
 80004b6:	e01d      	b.n	80004f4 <ai_platform_api_get_network_report+0xb6>
 80004b8:	f8b9 0048 	ldrh.w	r0, [r9, #72]	; 0x48
 80004bc:	b108      	cbz	r0, 80004c2 <ai_platform_api_get_network_report+0x84>
 80004be:	f8d9 004c 	ldr.w	r0, [r9, #76]	; 0x4c
 80004c2:	f104 0134 	add.w	r1, r4, #52	; 0x34
 80004c6:	f7ff fe93 	bl	80001f0 <_ai_platform_get_io_buffers_info>
 80004ca:	8620      	strh	r0, [r4, #48]	; 0x30
 80004cc:	b910      	cbnz	r0, 80004d4 <ai_platform_api_get_network_report+0x96>
 80004ce:	2218      	movs	r2, #24
 80004d0:	2112      	movs	r1, #18
 80004d2:	e00f      	b.n	80004f4 <ai_platform_api_get_network_report+0xb6>
 80004d4:	f8b9 0048 	ldrh.w	r0, [r9, #72]	; 0x48
 80004d8:	2802      	cmp	r0, #2
 80004da:	bfa6      	itte	ge
 80004dc:	f8d9 004c 	ldrge.w	r0, [r9, #76]	; 0x4c
 80004e0:	300c      	addge	r0, #12
 80004e2:	2000      	movlt	r0, #0
 80004e4:	f104 0138 	add.w	r1, r4, #56	; 0x38
 80004e8:	f7ff fe82 	bl	80001f0 <_ai_platform_get_io_buffers_info>
 80004ec:	8660      	strh	r0, [r4, #50]	; 0x32
 80004ee:	b948      	cbnz	r0, 8000504 <ai_platform_api_get_network_report+0xc6>
 80004f0:	2218      	movs	r2, #24
 80004f2:	2113      	movs	r1, #19
 80004f4:	f109 0010 	add.w	r0, r9, #16
 80004f8:	f000 fb1f 	bl	8000b3a <core_set_error>
 80004fc:	2000      	movs	r0, #0
 80004fe:	b001      	add	sp, #4
 8000500:	e8bd 8ff0 	ldmia.w	sp!, {r4, r5, r6, r7, r8, r9, sl, fp, pc}
 8000504:	f8d9 0004 	ldr.w	r0, [r9, #4]
 8000508:	6720      	str	r0, [r4, #112]	; 0x70
 800050a:	f109 0230 	add.w	r2, r9, #48	; 0x30
 800050e:	e892 5c09 	ldmia.w	r2, {r0, r3, sl, fp, ip, lr}
 8000512:	f104 013c 	add.w	r1, r4, #60	; 0x3c
 8000516:	f109 0918 	add.w	r9, r9, #24
 800051a:	e881 5c09 	stmia.w	r1, {r0, r3, sl, fp, ip, lr}
 800051e:	e899 540e 	ldmia.w	r9, {r1, r2, r3, sl, ip, lr}
 8000522:	f104 0054 	add.w	r0, r4, #84	; 0x54
 8000526:	e880 540e 	stmia.w	r0, {r1, r2, r3, sl, ip, lr}
 800052a:	6828      	ldr	r0, [r5, #0]
 800052c:	0840      	lsrs	r0, r0, #1
 800052e:	0040      	lsls	r0, r0, #1
 8000530:	6028      	str	r0, [r5, #0]
 8000532:	2301      	movs	r3, #1
 8000534:	60b3      	str	r3, [r6, #8]
 8000536:	68b0      	ldr	r0, [r6, #8]
 8000538:	2800      	cmp	r0, #0
 800053a:	d1fc      	bne.n	8000536 <ai_platform_api_get_network_report+0xf8>
 800053c:	6037      	str	r7, [r6, #0]
 800053e:	6831      	ldr	r1, [r6, #0]
 8000540:	4541      	cmp	r1, r8
 8000542:	d000      	beq.n	8000546 <ai_platform_api_get_network_report+0x108>
 8000544:	e7fe      	b.n	8000544 <ai_platform_api_get_network_report+0x106>
 8000546:	a01c      	add	r0, pc, #112	; (adr r0, 80005b8 <.text_13>)
 8000548:	6120      	str	r0, [r4, #16]
 800054a:	6829      	ldr	r1, [r5, #0]
 800054c:	0849      	lsrs	r1, r1, #1
 800054e:	0049      	lsls	r1, r1, #1
 8000550:	6029      	str	r1, [r5, #0]
 8000552:	60b3      	str	r3, [r6, #8]
 8000554:	68b0      	ldr	r0, [r6, #8]
 8000556:	2800      	cmp	r0, #0
 8000558:	d1fc      	bne.n	8000554 <ai_platform_api_get_network_report+0x116>
 800055a:	6037      	str	r7, [r6, #0]
 800055c:	6831      	ldr	r1, [r6, #0]
 800055e:	4541      	cmp	r1, r8
 8000560:	d000      	beq.n	8000564 <ai_platform_api_get_network_report+0x126>
 8000562:	e7fe      	b.n	8000562 <ai_platform_api_get_network_report+0x124>
 8000564:	f20f 509c 	addw	r0, pc, #1436	; 0x59c
 8000568:	6802      	ldr	r2, [r0, #0]
 800056a:	6162      	str	r2, [r4, #20]
 800056c:	6829      	ldr	r1, [r5, #0]
 800056e:	0849      	lsrs	r1, r1, #1
 8000570:	0049      	lsls	r1, r1, #1
 8000572:	6029      	str	r1, [r5, #0]
 8000574:	60b3      	str	r3, [r6, #8]
 8000576:	68b0      	ldr	r0, [r6, #8]
 8000578:	2800      	cmp	r0, #0
 800057a:	d1fc      	bne.n	8000576 <ai_platform_api_get_network_report+0x138>
 800057c:	6037      	str	r7, [r6, #0]
 800057e:	6831      	ldr	r1, [r6, #0]
 8000580:	4541      	cmp	r1, r8
 8000582:	d000      	beq.n	8000586 <ai_platform_api_get_network_report+0x148>
 8000584:	e7fe      	b.n	8000584 <ai_platform_api_get_network_report+0x146>
 8000586:	f20f 5080 	addw	r0, pc, #1408	; 0x580
 800058a:	6802      	ldr	r2, [r0, #0]
 800058c:	6262      	str	r2, [r4, #36]	; 0x24
 800058e:	6829      	ldr	r1, [r5, #0]
 8000590:	0849      	lsrs	r1, r1, #1
 8000592:	0049      	lsls	r1, r1, #1
 8000594:	6029      	str	r1, [r5, #0]
 8000596:	60b3      	str	r3, [r6, #8]
 8000598:	68b0      	ldr	r0, [r6, #8]
 800059a:	2800      	cmp	r0, #0
 800059c:	d1fc      	bne.n	8000598 <ai_platform_api_get_network_report+0x15a>
 800059e:	6037      	str	r7, [r6, #0]
 80005a0:	6831      	ldr	r1, [r6, #0]
 80005a2:	4541      	cmp	r1, r8
 80005a4:	d000      	beq.n	80005a8 <ai_platform_api_get_network_report+0x16a>
 80005a6:	e7fe      	b.n	80005a6 <ai_platform_api_get_network_report+0x168>
 80005a8:	f20f 5060 	addw	r0, pc, #1376	; 0x560
 80005ac:	6802      	ldr	r2, [r0, #0]
 80005ae:	62a2      	str	r2, [r4, #40]	; 0x28
 80005b0:	2001      	movs	r0, #1
 80005b2:	b001      	add	sp, #4
 80005b4:	e8bd 8ff0 	ldmia.w	sp!, {r4, r5, r6, r7, r8, r9, sl, fp, pc}

080005b8 <.text_13>:
 80005b8:	00000000 	.word	0x00000000

080005bc <ai_platform_network_create>:
 80005bc:	b570      	push	{r4, r5, r6, lr}
 80005be:	9d04      	ldr	r5, [sp, #16]
 80005c0:	4604      	mov	r4, r0
 80005c2:	9805      	ldr	r0, [sp, #20]
 80005c4:	b2db      	uxtb	r3, r3
 80005c6:	042d      	lsls	r5, r5, #16
 80005c8:	ea45 6503 	orr.w	r5, r5, r3, lsl #24
 80005cc:	ea45 2500 	orr.w	r5, r5, r0, lsl #8
 80005d0:	f20f 5050 	addw	r0, pc, #1360	; 0x550
 80005d4:	6806      	ldr	r6, [r0, #0]
 80005d6:	f8df 0514 	ldr.w	r0, [pc, #1300]	; 8000aec <.text_18>
 80005da:	6801      	ldr	r1, [r0, #0]
 80005dc:	0849      	lsrs	r1, r1, #1
 80005de:	0049      	lsls	r1, r1, #1
 80005e0:	6001      	str	r1, [r0, #0]
 80005e2:	2001      	movs	r0, #1
 80005e4:	f8df 1508 	ldr.w	r1, [pc, #1288]	; 8000af0 <.text_19>
 80005e8:	6088      	str	r0, [r1, #8]
 80005ea:	6888      	ldr	r0, [r1, #8]
 80005ec:	2800      	cmp	r0, #0
 80005ee:	d1fc      	bne.n	80005ea <ai_platform_network_create+0x2e>
 80005f0:	f8df 3500 	ldr.w	r3, [pc, #1280]	; 8000af4 <.text_20>
 80005f4:	600b      	str	r3, [r1, #0]
 80005f6:	6808      	ldr	r0, [r1, #0]
 80005f8:	f8df 14fc 	ldr.w	r1, [pc, #1276]	; 8000af8 <.text_21>
 80005fc:	4288      	cmp	r0, r1
 80005fe:	d000      	beq.n	8000602 <ai_platform_network_create+0x46>
 8000600:	e7fe      	b.n	8000600 <ai_platform_network_create+0x44>
 8000602:	b91c      	cbnz	r4, 800060c <ai_platform_network_create+0x50>
 8000604:	f20f 5020 	addw	r0, pc, #1312	; 0x520
 8000608:	6800      	ldr	r0, [r0, #0]
 800060a:	bd70      	pop	{r4, r5, r6, pc}
 800060c:	f8df 14ec 	ldr.w	r1, [pc, #1260]	; 8000afc <.text_22>
 8000610:	6011      	str	r1, [r2, #0]
 8000612:	6022      	str	r2, [r4, #0]
 8000614:	f000 fa8a 	bl	8000b2c <core_init>
 8000618:	b910      	cbnz	r0, 8000620 <ai_platform_network_create+0x64>
 800061a:	f20f 40f4 	addw	r0, pc, #1268	; 0x4f4
 800061e:	e00d      	b.n	800063c <ai_platform_network_create+0x80>
 8000620:	f8df 14dc 	ldr.w	r1, [pc, #1244]	; 8000b00 <.text_23>
 8000624:	428d      	cmp	r5, r1
 8000626:	bf28      	it	cs
 8000628:	f20f 40e8 	addwcs	r0, pc, #1256	; 0x4e8
 800062c:	d206      	bcs.n	800063c <ai_platform_network_create+0x80>
 800062e:	f20f 40e8 	addw	r0, pc, #1256	; 0x4e8
 8000632:	f000 fa97 	bl	8000b64 <ai_check_custom_types>
 8000636:	b920      	cbnz	r0, 8000642 <ai_platform_network_create+0x86>
 8000638:	f20f 40e0 	addw	r0, pc, #1248	; 0x4e0
 800063c:	6806      	ldr	r6, [r0, #0]
 800063e:	2100      	movs	r1, #0
 8000640:	6021      	str	r1, [r4, #0]
 8000642:	4630      	mov	r0, r6
 8000644:	bd70      	pop	{r4, r5, r6, pc}

08000646 <ai_platform_network_destroy>:
 8000646:	b130      	cbz	r0, 8000656 <ai_platform_network_destroy+0x10>
 8000648:	6801      	ldr	r1, [r0, #0]
 800064a:	f8df 24b0 	ldr.w	r2, [pc, #1200]	; 8000afc <.text_22>
 800064e:	4291      	cmp	r1, r2
 8000650:	bf08      	it	eq
 8000652:	4602      	moveq	r2, r0
 8000654:	d000      	beq.n	8000658 <ai_platform_network_destroy+0x12>
 8000656:	2200      	movs	r2, #0
 8000658:	f8df 1490 	ldr.w	r1, [pc, #1168]	; 8000aec <.text_18>
 800065c:	680b      	ldr	r3, [r1, #0]
 800065e:	085b      	lsrs	r3, r3, #1
 8000660:	005b      	lsls	r3, r3, #1
 8000662:	600b      	str	r3, [r1, #0]
 8000664:	2101      	movs	r1, #1
 8000666:	f8df 3488 	ldr.w	r3, [pc, #1160]	; 8000af0 <.text_19>
 800066a:	6099      	str	r1, [r3, #8]
 800066c:	6899      	ldr	r1, [r3, #8]
 800066e:	2900      	cmp	r1, #0
 8000670:	d1fc      	bne.n	800066c <ai_platform_network_destroy+0x26>
 8000672:	f8df c480 	ldr.w	ip, [pc, #1152]	; 8000af4 <.text_20>
 8000676:	f8c3 c000 	str.w	ip, [r3]
 800067a:	6819      	ldr	r1, [r3, #0]
 800067c:	f8df 3478 	ldr.w	r3, [pc, #1144]	; 8000af8 <.text_21>
 8000680:	4299      	cmp	r1, r3
 8000682:	d000      	beq.n	8000686 <ai_platform_network_destroy+0x40>
 8000684:	e7fe      	b.n	8000684 <ai_platform_network_destroy+0x3e>
 8000686:	b102      	cbz	r2, 800068a <ai_platform_network_destroy+0x44>
 8000688:	2000      	movs	r0, #0
 800068a:	4770      	bx	lr

0800068c <ai_platform_network_init>:
 800068c:	e92d 4ff0 	stmdb	sp!, {r4, r5, r6, r7, r8, r9, sl, fp, lr}
 8000690:	b081      	sub	sp, #4
 8000692:	460a      	mov	r2, r1
 8000694:	b120      	cbz	r0, 80006a0 <ai_platform_network_init+0x14>
 8000696:	6801      	ldr	r1, [r0, #0]
 8000698:	f8df 3460 	ldr.w	r3, [pc, #1120]	; 8000afc <.text_22>
 800069c:	4299      	cmp	r1, r3
 800069e:	d000      	beq.n	80006a2 <ai_platform_network_init+0x16>
 80006a0:	2000      	movs	r0, #0
 80006a2:	f8df 1448 	ldr.w	r1, [pc, #1096]	; 8000aec <.text_18>
 80006a6:	680b      	ldr	r3, [r1, #0]
 80006a8:	085b      	lsrs	r3, r3, #1
 80006aa:	005b      	lsls	r3, r3, #1
 80006ac:	600b      	str	r3, [r1, #0]
 80006ae:	2101      	movs	r1, #1
 80006b0:	f8df 343c 	ldr.w	r3, [pc, #1084]	; 8000af0 <.text_19>
 80006b4:	6099      	str	r1, [r3, #8]
 80006b6:	6899      	ldr	r1, [r3, #8]
 80006b8:	2900      	cmp	r1, #0
 80006ba:	d1fc      	bne.n	80006b6 <ai_platform_network_init+0x2a>
 80006bc:	f8df 4434 	ldr.w	r4, [pc, #1076]	; 8000af4 <.text_20>
 80006c0:	601c      	str	r4, [r3, #0]
 80006c2:	6819      	ldr	r1, [r3, #0]
 80006c4:	f8df 3430 	ldr.w	r3, [pc, #1072]	; 8000af8 <.text_21>
 80006c8:	4299      	cmp	r1, r3
 80006ca:	d000      	beq.n	80006ce <ai_platform_network_init+0x42>
 80006cc:	e7fe      	b.n	80006cc <ai_platform_network_init+0x40>
 80006ce:	2800      	cmp	r0, #0
 80006d0:	d035      	beq.n	800073e <ai_platform_network_init+0xb2>
 80006d2:	b90a      	cbnz	r2, 80006d8 <ai_platform_network_init+0x4c>
 80006d4:	2211      	movs	r2, #17
 80006d6:	e012      	b.n	80006fe <ai_platform_network_init+0x72>
 80006d8:	6913      	ldr	r3, [r2, #16]
 80006da:	6a91      	ldr	r1, [r2, #40]	; 0x28
 80006dc:	b939      	cbnz	r1, 80006ee <ai_platform_network_init+0x62>
 80006de:	8c11      	ldrh	r1, [r2, #32]
 80006e0:	8bd5      	ldrh	r5, [r2, #30]
 80006e2:	6a54      	ldr	r4, [r2, #36]	; 0x24
 80006e4:	4369      	muls	r1, r5
 80006e6:	4361      	muls	r1, r4
 80006e8:	bf18      	it	ne
 80006ea:	2213      	movne	r2, #19
 80006ec:	d107      	bne.n	80006fe <ai_platform_network_init+0x72>
 80006ee:	b973      	cbnz	r3, 800070e <ai_platform_network_init+0x82>
 80006f0:	8911      	ldrh	r1, [r2, #8]
 80006f2:	88d4      	ldrh	r4, [r2, #6]
 80006f4:	68d3      	ldr	r3, [r2, #12]
 80006f6:	4361      	muls	r1, r4
 80006f8:	4359      	muls	r1, r3
 80006fa:	d008      	beq.n	800070e <ai_platform_network_init+0x82>
 80006fc:	2212      	movs	r2, #18
 80006fe:	2110      	movs	r1, #16
 8000700:	3010      	adds	r0, #16
 8000702:	f000 fa1a 	bl	8000b3a <core_set_error>
 8000706:	2000      	movs	r0, #0
 8000708:	b001      	add	sp, #4
 800070a:	e8bd 8ff0 	ldmia.w	sp!, {r4, r5, r6, r7, r8, r9, sl, fp, pc}
 800070e:	e8b2 10f8 	ldmia.w	r2!, {r3, r4, r5, r6, r7, ip}
 8000712:	f100 0118 	add.w	r1, r0, #24
 8000716:	f100 0e30 	add.w	lr, r0, #48	; 0x30
 800071a:	e881 10f8 	stmia.w	r1, {r3, r4, r5, r6, r7, ip}
 800071e:	e892 0f0a 	ldmia.w	r2, {r1, r3, r8, r9, sl, fp}
 8000722:	e88e 0f0a 	stmia.w	lr, {r1, r3, r8, r9, sl, fp}
 8000726:	2103      	movs	r1, #3
 8000728:	6d02      	ldr	r2, [r0, #80]	; 0x50
 800072a:	60c1      	str	r1, [r0, #12]
 800072c:	b13a      	cbz	r2, 800073e <ai_platform_network_init+0xb2>
 800072e:	e000      	b.n	8000732 <ai_platform_network_init+0xa6>
 8000730:	460a      	mov	r2, r1
 8000732:	68d1      	ldr	r1, [r2, #12]
 8000734:	6090      	str	r0, [r2, #8]
 8000736:	428a      	cmp	r2, r1
 8000738:	bf18      	it	ne
 800073a:	2900      	cmpne	r1, #0
 800073c:	d1f8      	bne.n	8000730 <ai_platform_network_init+0xa4>
 800073e:	b001      	add	sp, #4
 8000740:	e8bd 8ff0 	ldmia.w	sp!, {r4, r5, r6, r7, r8, r9, sl, fp, pc}

08000744 <ai_platform_network_process>:
 8000744:	e92d 4ff4 	stmdb	sp!, {r2, r4, r5, r6, r7, r8, r9, sl, fp, lr}
 8000748:	b082      	sub	sp, #8
 800074a:	460a      	mov	r2, r1
 800074c:	b120      	cbz	r0, 8000758 <ai_platform_network_process+0x14>
 800074e:	6801      	ldr	r1, [r0, #0]
 8000750:	f8df 33a8 	ldr.w	r3, [pc, #936]	; 8000afc <.text_22>
 8000754:	4299      	cmp	r1, r3
 8000756:	d000      	beq.n	800075a <ai_platform_network_process+0x16>
 8000758:	2000      	movs	r0, #0
 800075a:	f8df 1390 	ldr.w	r1, [pc, #912]	; 8000aec <.text_18>
 800075e:	680b      	ldr	r3, [r1, #0]
 8000760:	085b      	lsrs	r3, r3, #1
 8000762:	005b      	lsls	r3, r3, #1
 8000764:	600b      	str	r3, [r1, #0]
 8000766:	2101      	movs	r1, #1
 8000768:	f8df 3384 	ldr.w	r3, [pc, #900]	; 8000af0 <.text_19>
 800076c:	6099      	str	r1, [r3, #8]
 800076e:	6899      	ldr	r1, [r3, #8]
 8000770:	2900      	cmp	r1, #0
 8000772:	d1fc      	bne.n	800076e <ai_platform_network_process+0x2a>
 8000774:	f8df 437c 	ldr.w	r4, [pc, #892]	; 8000af4 <.text_20>
 8000778:	601c      	str	r4, [r3, #0]
 800077a:	6819      	ldr	r1, [r3, #0]
 800077c:	f8df 3378 	ldr.w	r3, [pc, #888]	; 8000af8 <.text_21>
 8000780:	4299      	cmp	r1, r3
 8000782:	d000      	beq.n	8000786 <ai_platform_network_process+0x42>
 8000784:	e7fe      	b.n	8000784 <ai_platform_network_process+0x40>
 8000786:	2800      	cmp	r0, #0
 8000788:	f000 8113 	beq.w	80009b2 <ai_platform_network_process+0x26e>
 800078c:	f8b0 1048 	ldrh.w	r1, [r0, #72]	; 0x48
 8000790:	b101      	cbz	r1, 8000794 <ai_platform_network_process+0x50>
 8000792:	6cc1      	ldr	r1, [r0, #76]	; 0x4c
 8000794:	2300      	movs	r3, #0
 8000796:	82c3      	strh	r3, [r0, #22]
 8000798:	2400      	movs	r4, #0
 800079a:	7b03      	ldrb	r3, [r0, #12]
 800079c:	8284      	strh	r4, [r0, #20]
 800079e:	f003 0303 	and.w	r3, r3, #3
 80007a2:	2b03      	cmp	r3, #3
 80007a4:	d002      	beq.n	80007ac <ai_platform_network_process+0x68>
 80007a6:	2230      	movs	r2, #48	; 0x30
 80007a8:	2111      	movs	r1, #17
 80007aa:	e0ff      	b.n	80009ac <ai_platform_network_process+0x268>
 80007ac:	2a00      	cmp	r2, #0
 80007ae:	bf1e      	ittt	ne
 80007b0:	2900      	cmpne	r1, #0
 80007b2:	880b      	ldrhne	r3, [r1, #0]
 80007b4:	2b00      	cmpne	r3, #0
 80007b6:	f000 80f7 	beq.w	80009a8 <ai_platform_network_process+0x264>
 80007ba:	f8b2 b004 	ldrh.w	fp, [r2, #4]
 80007be:	9100      	str	r1, [sp, #0]
 80007c0:	46a0      	mov	r8, r4
 80007c2:	46a1      	mov	r9, r4
 80007c4:	2600      	movs	r6, #0
 80007c6:	1d17      	adds	r7, r2, #4
 80007c8:	4682      	mov	sl, r0
 80007ca:	e014      	b.n	80007f6 <ai_platform_network_process+0xb2>
 80007cc:	68f8      	ldr	r0, [r7, #12]
 80007ce:	2800      	cmp	r0, #0
 80007d0:	f000 80e9 	beq.w	80009a6 <ai_platform_network_process+0x262>
 80007d4:	8838      	ldrh	r0, [r7, #0]
 80007d6:	2800      	cmp	r0, #0
 80007d8:	d052      	beq.n	8000880 <ai_platform_network_process+0x13c>
 80007da:	4558      	cmp	r0, fp
 80007dc:	bf28      	it	cs
 80007de:	4683      	movcs	fp, r0
 80007e0:	4622      	mov	r2, r4
 80007e2:	1f39      	subs	r1, r7, #4
 80007e4:	4628      	mov	r0, r5
 80007e6:	f7ff fd59 	bl	800029c <_platform_network_state_setup>
 80007ea:	f108 0801 	add.w	r8, r8, #1
 80007ee:	3718      	adds	r7, #24
 80007f0:	3610      	adds	r6, #16
 80007f2:	f109 0904 	add.w	r9, r9, #4
 80007f6:	9800      	ldr	r0, [sp, #0]
 80007f8:	8801      	ldrh	r1, [r0, #0]
 80007fa:	4588      	cmp	r8, r1
 80007fc:	d24a      	bcs.n	8000894 <ai_platform_network_process+0x150>
 80007fe:	6840      	ldr	r0, [r0, #4]
 8000800:	2800      	cmp	r0, #0
 8000802:	bf1c      	itt	ne
 8000804:	f850 4009 	ldrne.w	r4, [r0, r9]
 8000808:	2c00      	cmpne	r4, #0
 800080a:	d043      	beq.n	8000894 <ai_platform_network_process+0x150>
 800080c:	9800      	ldr	r0, [sp, #0]
 800080e:	6881      	ldr	r1, [r0, #8]
 8000810:	680a      	ldr	r2, [r1, #0]
 8000812:	1995      	adds	r5, r2, r6
 8000814:	f000 80c7 	beq.w	80009a6 <ai_platform_network_process+0x262>
 8000818:	69a0      	ldr	r0, [r4, #24]
 800081a:	6841      	ldr	r1, [r0, #4]
 800081c:	887b      	ldrh	r3, [r7, #2]
 800081e:	88ba      	ldrh	r2, [r7, #4]
 8000820:	68b8      	ldr	r0, [r7, #8]
 8000822:	fb03 fc02 	mul.w	ip, r3, r2
 8000826:	fb00 fc0c 	mul.w	ip, r0, ip
 800082a:	4561      	cmp	r1, ip
 800082c:	d32d      	bcc.n	800088a <ai_platform_network_process+0x146>
 800082e:	f8d4 c00c 	ldr.w	ip, [r4, #12]
 8000832:	f8dc e00c 	ldr.w	lr, [ip, #12]
 8000836:	459e      	cmp	lr, r3
 8000838:	bf01      	itttt	eq
 800083a:	f8dc 3008 	ldreq.w	r3, [ip, #8]
 800083e:	4293      	cmpeq	r3, r2
 8000840:	f8dc 2004 	ldreq.w	r2, [ip, #4]
 8000844:	4282      	cmpeq	r2, r0
 8000846:	d120      	bne.n	800088a <ai_platform_network_process+0x146>
 8000848:	69a0      	ldr	r0, [r4, #24]
 800084a:	6800      	ldr	r0, [r0, #0]
 800084c:	f005 fb1a 	bl	8005e84 <ai_array_get_byte_size>
 8000850:	68e1      	ldr	r1, [r4, #12]
 8000852:	68ca      	ldr	r2, [r1, #12]
 8000854:	6961      	ldr	r1, [r4, #20]
 8000856:	68cb      	ldr	r3, [r1, #12]
 8000858:	435a      	muls	r2, r3
 800085a:	4290      	cmp	r0, r2
 800085c:	d315      	bcc.n	800088a <ai_platform_network_process+0x146>
 800085e:	69a0      	ldr	r0, [r4, #24]
 8000860:	6800      	ldr	r0, [r0, #0]
 8000862:	f005 fa37 	bl	8005cd4 <ai_array_to_buffer_fmt>
 8000866:	f857 1c04 	ldr.w	r1, [r7, #-4]
 800086a:	f020 407e 	bic.w	r0, r0, #4261412864	; 0xfe000000
 800086e:	f021 417e 	bic.w	r1, r1, #4261412864	; 0xfe000000
 8000872:	4288      	cmp	r0, r1
 8000874:	d0aa      	beq.n	80007cc <ai_platform_network_process+0x88>
 8000876:	2219      	movs	r2, #25
 8000878:	2112      	movs	r1, #18
 800087a:	f10a 0010 	add.w	r0, sl, #16
 800087e:	e096      	b.n	80009ae <ai_platform_network_process+0x26a>
 8000880:	2221      	movs	r2, #33	; 0x21
 8000882:	2112      	movs	r1, #18
 8000884:	f10a 0010 	add.w	r0, sl, #16
 8000888:	e091      	b.n	80009ae <ai_platform_network_process+0x26a>
 800088a:	2218      	movs	r2, #24
 800088c:	2112      	movs	r1, #18
 800088e:	f10a 0010 	add.w	r0, sl, #16
 8000892:	e08c      	b.n	80009ae <ai_platform_network_process+0x26a>
 8000894:	9902      	ldr	r1, [sp, #8]
 8000896:	2900      	cmp	r1, #0
 8000898:	4655      	mov	r5, sl
 800089a:	d075      	beq.n	8000988 <ai_platform_network_process+0x244>
 800089c:	f8b5 0048 	ldrh.w	r0, [r5, #72]	; 0x48
 80008a0:	2802      	cmp	r0, #2
 80008a2:	db7b      	blt.n	800099c <ai_platform_network_process+0x258>
 80008a4:	6ce8      	ldr	r0, [r5, #76]	; 0x4c
 80008a6:	300c      	adds	r0, #12
 80008a8:	bf1c      	itt	ne
 80008aa:	8802      	ldrhne	r2, [r0, #0]
 80008ac:	2a00      	cmpne	r2, #0
 80008ae:	d075      	beq.n	800099c <ai_platform_network_process+0x258>
 80008b0:	f04f 0800 	mov.w	r8, #0
 80008b4:	46c1      	mov	r9, r8
 80008b6:	2600      	movs	r6, #0
 80008b8:	1d0f      	adds	r7, r1, #4
 80008ba:	9000      	str	r0, [sp, #0]
 80008bc:	e013      	b.n	80008e6 <ai_platform_network_process+0x1a2>
 80008be:	68f8      	ldr	r0, [r7, #12]
 80008c0:	2800      	cmp	r0, #0
 80008c2:	d059      	beq.n	8000978 <ai_platform_network_process+0x234>
 80008c4:	8838      	ldrh	r0, [r7, #0]
 80008c6:	2800      	cmp	r0, #0
 80008c8:	d051      	beq.n	800096e <ai_platform_network_process+0x22a>
 80008ca:	4558      	cmp	r0, fp
 80008cc:	bf28      	it	cs
 80008ce:	4683      	movcs	fp, r0
 80008d0:	4622      	mov	r2, r4
 80008d2:	1f39      	subs	r1, r7, #4
 80008d4:	4628      	mov	r0, r5
 80008d6:	f7ff fce1 	bl	800029c <_platform_network_state_setup>
 80008da:	f108 0801 	add.w	r8, r8, #1
 80008de:	3718      	adds	r7, #24
 80008e0:	3610      	adds	r6, #16
 80008e2:	f109 0904 	add.w	r9, r9, #4
 80008e6:	9800      	ldr	r0, [sp, #0]
 80008e8:	8801      	ldrh	r1, [r0, #0]
 80008ea:	4588      	cmp	r8, r1
 80008ec:	d249      	bcs.n	8000982 <ai_platform_network_process+0x23e>
 80008ee:	6840      	ldr	r0, [r0, #4]
 80008f0:	2800      	cmp	r0, #0
 80008f2:	bf1c      	itt	ne
 80008f4:	f850 4009 	ldrne.w	r4, [r0, r9]
 80008f8:	2c00      	cmpne	r4, #0
 80008fa:	d042      	beq.n	8000982 <ai_platform_network_process+0x23e>
 80008fc:	9800      	ldr	r0, [sp, #0]
 80008fe:	6881      	ldr	r1, [r0, #8]
 8000900:	680a      	ldr	r2, [r1, #0]
 8000902:	1995      	adds	r5, r2, r6
 8000904:	d038      	beq.n	8000978 <ai_platform_network_process+0x234>
 8000906:	69a0      	ldr	r0, [r4, #24]
 8000908:	6841      	ldr	r1, [r0, #4]
 800090a:	887b      	ldrh	r3, [r7, #2]
 800090c:	88ba      	ldrh	r2, [r7, #4]
 800090e:	68b8      	ldr	r0, [r7, #8]
 8000910:	fb03 fc02 	mul.w	ip, r3, r2
 8000914:	fb00 fc0c 	mul.w	ip, r0, ip
 8000918:	4561      	cmp	r1, ip
 800091a:	d33e      	bcc.n	800099a <ai_platform_network_process+0x256>
 800091c:	f8d4 c00c 	ldr.w	ip, [r4, #12]
 8000920:	f8dc e00c 	ldr.w	lr, [ip, #12]
 8000924:	459e      	cmp	lr, r3
 8000926:	bf01      	itttt	eq
 8000928:	f8dc 3008 	ldreq.w	r3, [ip, #8]
 800092c:	4293      	cmpeq	r3, r2
 800092e:	f8dc 2004 	ldreq.w	r2, [ip, #4]
 8000932:	4282      	cmpeq	r2, r0
 8000934:	d131      	bne.n	800099a <ai_platform_network_process+0x256>
 8000936:	69a0      	ldr	r0, [r4, #24]
 8000938:	6800      	ldr	r0, [r0, #0]
 800093a:	f005 faa3 	bl	8005e84 <ai_array_get_byte_size>
 800093e:	68e1      	ldr	r1, [r4, #12]
 8000940:	68ca      	ldr	r2, [r1, #12]
 8000942:	6961      	ldr	r1, [r4, #20]
 8000944:	68cb      	ldr	r3, [r1, #12]
 8000946:	435a      	muls	r2, r3
 8000948:	4290      	cmp	r0, r2
 800094a:	d326      	bcc.n	800099a <ai_platform_network_process+0x256>
 800094c:	69a0      	ldr	r0, [r4, #24]
 800094e:	6800      	ldr	r0, [r0, #0]
 8000950:	f005 f9c0 	bl	8005cd4 <ai_array_to_buffer_fmt>
 8000954:	f857 1c04 	ldr.w	r1, [r7, #-4]
 8000958:	f020 407e 	bic.w	r0, r0, #4261412864	; 0xfe000000
 800095c:	f021 417e 	bic.w	r1, r1, #4261412864	; 0xfe000000
 8000960:	4288      	cmp	r0, r1
 8000962:	d0ac      	beq.n	80008be <ai_platform_network_process+0x17a>
 8000964:	2219      	movs	r2, #25
 8000966:	2113      	movs	r1, #19
 8000968:	f10a 0010 	add.w	r0, sl, #16
 800096c:	e01f      	b.n	80009ae <ai_platform_network_process+0x26a>
 800096e:	2221      	movs	r2, #33	; 0x21
 8000970:	2113      	movs	r1, #19
 8000972:	f10a 0010 	add.w	r0, sl, #16
 8000976:	e01a      	b.n	80009ae <ai_platform_network_process+0x26a>
 8000978:	2217      	movs	r2, #23
 800097a:	2113      	movs	r1, #19
 800097c:	f10a 0010 	add.w	r0, sl, #16
 8000980:	e015      	b.n	80009ae <ai_platform_network_process+0x26a>
 8000982:	4655      	mov	r5, sl
 8000984:	f8a5 b014 	strh.w	fp, [r5, #20]
 8000988:	f8b5 0048 	ldrh.w	r0, [r5, #72]	; 0x48
 800098c:	2800      	cmp	r0, #0
 800098e:	bf14      	ite	ne
 8000990:	f8d5 a04c 	ldrne.w	sl, [r5, #76]	; 0x4c
 8000994:	f04f 0a00 	moveq.w	sl, #0
 8000998:	e00f      	b.n	80009ba <ai_platform_network_process+0x276>
 800099a:	4655      	mov	r5, sl
 800099c:	2218      	movs	r2, #24
 800099e:	2113      	movs	r1, #19
 80009a0:	f105 0010 	add.w	r0, r5, #16
 80009a4:	e003      	b.n	80009ae <ai_platform_network_process+0x26a>
 80009a6:	4650      	mov	r0, sl
 80009a8:	2217      	movs	r2, #23
 80009aa:	2112      	movs	r1, #18
 80009ac:	3010      	adds	r0, #16
 80009ae:	f000 f8c4 	bl	8000b3a <core_set_error>
 80009b2:	2000      	movs	r0, #0
 80009b4:	b003      	add	sp, #12
 80009b6:	e8bd 8ff0 	ldmia.w	sp!, {r4, r5, r6, r7, r8, r9, sl, fp, pc}
 80009ba:	2802      	cmp	r0, #2
 80009bc:	bfa6      	itte	ge
 80009be:	6ce8      	ldrge	r0, [r5, #76]	; 0x4c
 80009c0:	f100 0b0c 	addge.w	fp, r0, #12
 80009c4:	f04f 0b00 	movlt.w	fp, #0
 80009c8:	8ae8      	ldrh	r0, [r5, #22]
 80009ca:	8aa9      	ldrh	r1, [r5, #20]
 80009cc:	ebb0 0f01 	cmp.w	r0, r1
 80009d0:	f080 8087 	bcs.w	8000ae2 <ai_platform_network_process+0x39e>
 80009d4:	f04f 0800 	mov.w	r8, #0
 80009d8:	4654      	mov	r4, sl
 80009da:	46c1      	mov	r9, r8
 80009dc:	46c2      	mov	sl, r8
 80009de:	e018      	b.n	8000a12 <ai_platform_network_process+0x2ce>
 80009e0:	6882      	ldr	r2, [r0, #8]
 80009e2:	68c3      	ldr	r3, [r0, #12]
 80009e4:	6871      	ldr	r1, [r6, #4]
 80009e6:	1ad2      	subs	r2, r2, r3
 80009e8:	4411      	add	r1, r2
 80009ea:	6081      	str	r1, [r0, #8]
 80009ec:	6872      	ldr	r2, [r6, #4]
 80009ee:	60c2      	str	r2, [r0, #12]
 80009f0:	6870      	ldr	r0, [r6, #4]
 80009f2:	68b1      	ldr	r1, [r6, #8]
 80009f4:	4408      	add	r0, r1
 80009f6:	6070      	str	r0, [r6, #4]
 80009f8:	6831      	ldr	r1, [r6, #0]
 80009fa:	4288      	cmp	r0, r1
 80009fc:	d302      	bcc.n	8000a04 <ai_platform_network_process+0x2c0>
 80009fe:	68f0      	ldr	r0, [r6, #12]
 8000a00:	4240      	negs	r0, r0
 8000a02:	4408      	add	r0, r1
 8000a04:	6070      	str	r0, [r6, #4]
 8000a06:	f10a 0a01 	add.w	sl, sl, #1
 8000a0a:	f109 0910 	add.w	r9, r9, #16
 8000a0e:	f108 0804 	add.w	r8, r8, #4
 8000a12:	2c00      	cmp	r4, #0
 8000a14:	bf14      	ite	ne
 8000a16:	8820      	ldrhne	r0, [r4, #0]
 8000a18:	2000      	moveq	r0, #0
 8000a1a:	4582      	cmp	sl, r0
 8000a1c:	d212      	bcs.n	8000a44 <ai_platform_network_process+0x300>
 8000a1e:	6860      	ldr	r0, [r4, #4]
 8000a20:	b180      	cbz	r0, 8000a44 <ai_platform_network_process+0x300>
 8000a22:	f850 0008 	ldr.w	r0, [r0, r8]
 8000a26:	b168      	cbz	r0, 8000a44 <ai_platform_network_process+0x300>
 8000a28:	68a1      	ldr	r1, [r4, #8]
 8000a2a:	6980      	ldr	r0, [r0, #24]
 8000a2c:	680a      	ldr	r2, [r1, #0]
 8000a2e:	6801      	ldr	r1, [r0, #0]
 8000a30:	eb02 0609 	add.w	r6, r2, r9
 8000a34:	008a      	lsls	r2, r1, #2
 8000a36:	d5d3      	bpl.n	80009e0 <ai_platform_network_process+0x29c>
 8000a38:	68b2      	ldr	r2, [r6, #8]
 8000a3a:	6871      	ldr	r1, [r6, #4]
 8000a3c:	6880      	ldr	r0, [r0, #8]
 8000a3e:	f009 fa9e 	bl	8009f7e <__aeabi_memcpy>
 8000a42:	e7d5      	b.n	80009f0 <ai_platform_network_process+0x2ac>
 8000a44:	46a2      	mov	sl, r4
 8000a46:	4628      	mov	r0, r5
 8000a48:	f000 f936 	bl	8000cb8 <ai_layers_forward_all>
 8000a4c:	f04f 0800 	mov.w	r8, #0
 8000a50:	465c      	mov	r4, fp
 8000a52:	46c1      	mov	r9, r8
 8000a54:	46c3      	mov	fp, r8
 8000a56:	e017      	b.n	8000a88 <ai_platform_network_process+0x344>
 8000a58:	6871      	ldr	r1, [r6, #4]
 8000a5a:	68b2      	ldr	r2, [r6, #8]
 8000a5c:	4411      	add	r1, r2
 8000a5e:	6071      	str	r1, [r6, #4]
 8000a60:	6832      	ldr	r2, [r6, #0]
 8000a62:	4291      	cmp	r1, r2
 8000a64:	d302      	bcc.n	8000a6c <ai_platform_network_process+0x328>
 8000a66:	68f1      	ldr	r1, [r6, #12]
 8000a68:	4249      	negs	r1, r1
 8000a6a:	4411      	add	r1, r2
 8000a6c:	6071      	str	r1, [r6, #4]
 8000a6e:	6882      	ldr	r2, [r0, #8]
 8000a70:	68c3      	ldr	r3, [r0, #12]
 8000a72:	1ad2      	subs	r2, r2, r3
 8000a74:	4411      	add	r1, r2
 8000a76:	6081      	str	r1, [r0, #8]
 8000a78:	6872      	ldr	r2, [r6, #4]
 8000a7a:	60c2      	str	r2, [r0, #12]
 8000a7c:	f10b 0b01 	add.w	fp, fp, #1
 8000a80:	f109 0910 	add.w	r9, r9, #16
 8000a84:	f108 0804 	add.w	r8, r8, #4
 8000a88:	2c00      	cmp	r4, #0
 8000a8a:	bf14      	ite	ne
 8000a8c:	8820      	ldrhne	r0, [r4, #0]
 8000a8e:	2000      	moveq	r0, #0
 8000a90:	4583      	cmp	fp, r0
 8000a92:	d21d      	bcs.n	8000ad0 <ai_platform_network_process+0x38c>
 8000a94:	6860      	ldr	r0, [r4, #4]
 8000a96:	b1d8      	cbz	r0, 8000ad0 <ai_platform_network_process+0x38c>
 8000a98:	f850 0008 	ldr.w	r0, [r0, r8]
 8000a9c:	b1c0      	cbz	r0, 8000ad0 <ai_platform_network_process+0x38c>
 8000a9e:	68a1      	ldr	r1, [r4, #8]
 8000aa0:	6980      	ldr	r0, [r0, #24]
 8000aa2:	680a      	ldr	r2, [r1, #0]
 8000aa4:	6801      	ldr	r1, [r0, #0]
 8000aa6:	eb02 0609 	add.w	r6, r2, r9
 8000aaa:	008a      	lsls	r2, r1, #2
 8000aac:	d5d4      	bpl.n	8000a58 <ai_platform_network_process+0x314>
 8000aae:	6881      	ldr	r1, [r0, #8]
 8000ab0:	68b2      	ldr	r2, [r6, #8]
 8000ab2:	6870      	ldr	r0, [r6, #4]
 8000ab4:	f009 fa63 	bl	8009f7e <__aeabi_memcpy>
 8000ab8:	6870      	ldr	r0, [r6, #4]
 8000aba:	68b1      	ldr	r1, [r6, #8]
 8000abc:	4408      	add	r0, r1
 8000abe:	6070      	str	r0, [r6, #4]
 8000ac0:	6831      	ldr	r1, [r6, #0]
 8000ac2:	4288      	cmp	r0, r1
 8000ac4:	d302      	bcc.n	8000acc <ai_platform_network_process+0x388>
 8000ac6:	68f0      	ldr	r0, [r6, #12]
 8000ac8:	4240      	negs	r0, r0
 8000aca:	4408      	add	r0, r1
 8000acc:	6070      	str	r0, [r6, #4]
 8000ace:	e7d5      	b.n	8000a7c <ai_platform_network_process+0x338>
 8000ad0:	8ae8      	ldrh	r0, [r5, #22]
 8000ad2:	8aa9      	ldrh	r1, [r5, #20]
 8000ad4:	1c40      	adds	r0, r0, #1
 8000ad6:	82e8      	strh	r0, [r5, #22]
 8000ad8:	46a3      	mov	fp, r4
 8000ada:	b280      	uxth	r0, r0
 8000adc:	4288      	cmp	r0, r1
 8000ade:	f4ff af79 	bcc.w	80009d4 <ai_platform_network_process+0x290>
 8000ae2:	8ae8      	ldrh	r0, [r5, #22]
 8000ae4:	b003      	add	sp, #12
 8000ae6:	e8bd 8ff0 	ldmia.w	sp!, {r4, r5, r6, r7, r8, r9, sl, fp, pc}
	...

08000aec <.text_18>:
 8000aec:	e0002000 	.word	0xe0002000

08000af0 <.text_19>:
 8000af0:	40023000 	.word	0x40023000

08000af4 <.text_20>:
 8000af4:	f407a5c2 	.word	0xf407a5c2

08000af8 <.text_21>:
 8000af8:	b5e8b5cd 	.word	0xb5e8b5cd

08000afc <.text_22>:
 8000afc:	a1c00100 	.word	0xa1c00100

08000b00 <.text_23>:
 8000b00:	01030001 	.word	0x01030001

08000b04 <.text_24>:
 8000b04:	00000104 	.word	0x00000104

08000b08 <.text_25>:
 8000b08:	00000101 	.word	0x00000101

08000b0c <.text_26>:
 8000b0c:	00000301 	.word	0x00000301

08000b10 <.text_27>:
 8000b10:	00001030 	.word	0x00001030

08000b14 <.text_28>:
 8000b14:	00001001 	.word	0x00001001

08000b18 <_platform_network_sanity_check{5}::signatures>:
 8000b18:	84048403                                ....

08000b1c <.text_30>:
 8000b1c:	00001002 	.word	0x00001002

08000b20 <.text_31>:
 8000b20:	00001010 	.word	0x00001010

08000b24 <.text_32>:
 8000b24:	00000000 	.word	0x00000000

08000b28 <.text_33>:
 8000b28:	00001010 	.word	0x00001010

08000b2c <core_init>:
 8000b2c:	2001      	movs	r0, #1
 8000b2e:	4770      	bx	lr

08000b30 <core_get_error>:
 8000b30:	4601      	mov	r1, r0
 8000b32:	2200      	movs	r2, #0
 8000b34:	6808      	ldr	r0, [r1, #0]
 8000b36:	600a      	str	r2, [r1, #0]
 8000b38:	4770      	bx	lr

08000b3a <core_set_error>:
 8000b3a:	7803      	ldrb	r3, [r0, #0]
 8000b3c:	ea5f 6c03 	movs.w	ip, r3, lsl #24
 8000b40:	d104      	bne.n	8000b4c <core_set_error+0x12>
 8000b42:	ea41 2102 	orr.w	r1, r1, r2, lsl #8
 8000b46:	6001      	str	r1, [r0, #0]
 8000b48:	2001      	movs	r0, #1
 8000b4a:	4770      	bx	lr
 8000b4c:	2000      	movs	r0, #0
 8000b4e:	4770      	bx	lr

08000b50 <ai_layers_forward_layer>:
 8000b50:	b510      	push	{r4, lr}
 8000b52:	4604      	mov	r4, r0
 8000b54:	6921      	ldr	r1, [r4, #16]
 8000b56:	4788      	blx	r1
 8000b58:	68e0      	ldr	r0, [r4, #12]
 8000b5a:	42a0      	cmp	r0, r4
 8000b5c:	bf08      	it	eq
 8000b5e:	2000      	moveq	r0, #0
 8000b60:	bd10      	pop	{r4, pc}
	...

08000b64 <ai_check_custom_types>:
 8000b64:	b500      	push	{lr}
 8000b66:	b081      	sub	sp, #4
 8000b68:	b160      	cbz	r0, 8000b84 <ai_check_custom_types+0x20>
 8000b6a:	7801      	ldrb	r1, [r0, #0]
 8000b6c:	2903      	cmp	r1, #3
 8000b6e:	d109      	bne.n	8000b84 <ai_check_custom_types+0x20>
 8000b70:	f05f 0204 	movs.w	r2, #4
 8000b74:	a18d      	add	r1, pc, #564	; (adr r1, 8000dac <ai_check_custom_types::ref_signatures>)
 8000b76:	f009 fa2f 	bl	8009fd8 <memcmp>
 8000b7a:	1e40      	subs	r0, r0, #1
 8000b7c:	4180      	sbcs	r0, r0
 8000b7e:	0fc0      	lsrs	r0, r0, #31
 8000b80:	b001      	add	sp, #4
 8000b82:	bd00      	pop	{pc}
 8000b84:	2000      	movs	r0, #0
 8000b86:	b001      	add	sp, #4
 8000b88:	bd00      	pop	{pc}
	...

08000b8c <ai_layer_type_name>:
 8000b8c:	f242 7211 	movw	r2, #10001	; 0x2711
 8000b90:	1a81      	subs	r1, r0, r2
 8000b92:	2901      	cmp	r1, #1
 8000b94:	bf81      	itttt	hi
 8000b96:	1ec9      	subhi	r1, r1, #3
 8000b98:	290d      	cmphi	r1, #13
 8000b9a:	390f      	subhi	r1, #15
 8000b9c:	2909      	cmphi	r1, #9
 8000b9e:	f200 806b 	bhi.w	8000c78 <ai_layer_type_name+0xec>
 8000ba2:	1a80      	subs	r0, r0, r2
 8000ba4:	d033      	beq.n	8000c0e <ai_layer_type_name+0x82>
 8000ba6:	1e40      	subs	r0, r0, #1
 8000ba8:	d033      	beq.n	8000c12 <ai_layer_type_name+0x86>
 8000baa:	1e80      	subs	r0, r0, #2
 8000bac:	d033      	beq.n	8000c16 <ai_layer_type_name+0x8a>
 8000bae:	1e40      	subs	r0, r0, #1
 8000bb0:	d034      	beq.n	8000c1c <ai_layer_type_name+0x90>
 8000bb2:	1e40      	subs	r0, r0, #1
 8000bb4:	d034      	beq.n	8000c20 <ai_layer_type_name+0x94>
 8000bb6:	1e40      	subs	r0, r0, #1
 8000bb8:	d034      	beq.n	8000c24 <ai_layer_type_name+0x98>
 8000bba:	1e40      	subs	r0, r0, #1
 8000bbc:	d034      	beq.n	8000c28 <ai_layer_type_name+0x9c>
 8000bbe:	1e40      	subs	r0, r0, #1
 8000bc0:	d034      	beq.n	8000c2c <ai_layer_type_name+0xa0>
 8000bc2:	1e40      	subs	r0, r0, #1
 8000bc4:	d034      	beq.n	8000c30 <ai_layer_type_name+0xa4>
 8000bc6:	1e40      	subs	r0, r0, #1
 8000bc8:	d034      	beq.n	8000c34 <ai_layer_type_name+0xa8>
 8000bca:	1e40      	subs	r0, r0, #1
 8000bcc:	d034      	beq.n	8000c38 <ai_layer_type_name+0xac>
 8000bce:	1e40      	subs	r0, r0, #1
 8000bd0:	d034      	beq.n	8000c3c <ai_layer_type_name+0xb0>
 8000bd2:	1e40      	subs	r0, r0, #1
 8000bd4:	d034      	beq.n	8000c40 <ai_layer_type_name+0xb4>
 8000bd6:	1e40      	subs	r0, r0, #1
 8000bd8:	d034      	beq.n	8000c44 <ai_layer_type_name+0xb8>
 8000bda:	1e40      	subs	r0, r0, #1
 8000bdc:	d034      	beq.n	8000c48 <ai_layer_type_name+0xbc>
 8000bde:	1e40      	subs	r0, r0, #1
 8000be0:	d034      	beq.n	8000c4c <ai_layer_type_name+0xc0>
 8000be2:	1e80      	subs	r0, r0, #2
 8000be4:	d034      	beq.n	8000c50 <ai_layer_type_name+0xc4>
 8000be6:	1e40      	subs	r0, r0, #1
 8000be8:	d034      	beq.n	8000c54 <ai_layer_type_name+0xc8>
 8000bea:	1e40      	subs	r0, r0, #1
 8000bec:	d034      	beq.n	8000c58 <ai_layer_type_name+0xcc>
 8000bee:	1e40      	subs	r0, r0, #1
 8000bf0:	d034      	beq.n	8000c5c <ai_layer_type_name+0xd0>
 8000bf2:	1e40      	subs	r0, r0, #1
 8000bf4:	d034      	beq.n	8000c60 <ai_layer_type_name+0xd4>
 8000bf6:	1e40      	subs	r0, r0, #1
 8000bf8:	d034      	beq.n	8000c64 <ai_layer_type_name+0xd8>
 8000bfa:	1e40      	subs	r0, r0, #1
 8000bfc:	d034      	beq.n	8000c68 <ai_layer_type_name+0xdc>
 8000bfe:	1e40      	subs	r0, r0, #1
 8000c00:	d034      	beq.n	8000c6c <ai_layer_type_name+0xe0>
 8000c02:	1e40      	subs	r0, r0, #1
 8000c04:	d034      	beq.n	8000c70 <ai_layer_type_name+0xe4>
 8000c06:	1e40      	subs	r0, r0, #1
 8000c08:	d034      	beq.n	8000c74 <ai_layer_type_name+0xe8>
 8000c0a:	a01c      	add	r0, pc, #112	; (adr r0, 8000c7c <.text_5>)
 8000c0c:	4770      	bx	lr
 8000c0e:	a01c      	add	r0, pc, #112	; (adr r0, 8000c80 <.text_6>)
 8000c10:	4770      	bx	lr
 8000c12:	a01c      	add	r0, pc, #112	; (adr r0, 8000c84 <.text_7>)
 8000c14:	4770      	bx	lr
 8000c16:	bf00      	nop
 8000c18:	a031      	add	r0, pc, #196	; (adr r0, 8000ce0 <.text_15>)
 8000c1a:	4770      	bx	lr
 8000c1c:	a032      	add	r0, pc, #200	; (adr r0, 8000ce8 <.text_16>)
 8000c1e:	4770      	bx	lr
 8000c20:	a019      	add	r0, pc, #100	; (adr r0, 8000c88 <.text_8>)
 8000c22:	4770      	bx	lr
 8000c24:	a019      	add	r0, pc, #100	; (adr r0, 8000c8c <.text_9>)
 8000c26:	4770      	bx	lr
 8000c28:	a031      	add	r0, pc, #196	; (adr r0, 8000cf0 <.text_17>)
 8000c2a:	4770      	bx	lr
 8000c2c:	a018      	add	r0, pc, #96	; (adr r0, 8000c90 <.text_10>)
 8000c2e:	4770      	bx	lr
 8000c30:	a031      	add	r0, pc, #196	; (adr r0, 8000cf8 <.text_18>)
 8000c32:	4770      	bx	lr
 8000c34:	a032      	add	r0, pc, #200	; (adr r0, 8000d00 <.text_19>)
 8000c36:	4770      	bx	lr
 8000c38:	a036      	add	r0, pc, #216	; (adr r0, 8000d14 <.text_20>)
 8000c3a:	4770      	bx	lr
 8000c3c:	a038      	add	r0, pc, #224	; (adr r0, 8000d20 <.text_21>)
 8000c3e:	4770      	bx	lr
 8000c40:	a014      	add	r0, pc, #80	; (adr r0, 8000c94 <.text_11>)
 8000c42:	4770      	bx	lr
 8000c44:	a038      	add	r0, pc, #224	; (adr r0, 8000d28 <.text_22>)
 8000c46:	4770      	bx	lr
 8000c48:	a039      	add	r0, pc, #228	; (adr r0, 8000d30 <.text_23>)
 8000c4a:	4770      	bx	lr
 8000c4c:	a03b      	add	r0, pc, #236	; (adr r0, 8000d3c <.text_24>)
 8000c4e:	4770      	bx	lr
 8000c50:	a03f      	add	r0, pc, #252	; (adr r0, 8000d50 <.text_25>)
 8000c52:	4770      	bx	lr
 8000c54:	a040      	add	r0, pc, #256	; (adr r0, 8000d58 <.text_26>)
 8000c56:	4770      	bx	lr
 8000c58:	a041      	add	r0, pc, #260	; (adr r0, 8000d60 <.text_27>)
 8000c5a:	4770      	bx	lr
 8000c5c:	a043      	add	r0, pc, #268	; (adr r0, 8000d6c <.text_28>)
 8000c5e:	4770      	bx	lr
 8000c60:	a044      	add	r0, pc, #272	; (adr r0, 8000d74 <.text_29>)
 8000c62:	4770      	bx	lr
 8000c64:	a045      	add	r0, pc, #276	; (adr r0, 8000d7c <.text_30>)
 8000c66:	4770      	bx	lr
 8000c68:	a00b      	add	r0, pc, #44	; (adr r0, 8000c98 <.text_12>)
 8000c6a:	4770      	bx	lr
 8000c6c:	a049      	add	r0, pc, #292	; (adr r0, 8000d94 <.text_31>)
 8000c6e:	4770      	bx	lr
 8000c70:	a04a      	add	r0, pc, #296	; (adr r0, 8000d9c <.text_32>)
 8000c72:	4770      	bx	lr
 8000c74:	a04b      	add	r0, pc, #300	; (adr r0, 8000da4 <.text_33>)
 8000c76:	4770      	bx	lr
 8000c78:	a000      	add	r0, pc, #0	; (adr r0, 8000c7c <.text_5>)
 8000c7a:	4770      	bx	lr

08000c7c <.text_5>:
 8000c7c:	00000000 	.word	0x00000000

08000c80 <.text_6>:
 8000c80:	00444441 	.word	0x00444441

08000c84 <.text_7>:
 8000c84:	00004e42 	.word	0x00004e42

08000c88 <.text_8>:
 8000c88:	00555247 	.word	0x00555247

08000c8c <.text_9>:
 8000c8c:	004e524c 	.word	0x004e524c

08000c90 <.text_10>:
 8000c90:	00004c4e 	.word	0x00004c4e

08000c94 <.text_11>:
 8000c94:	00004d53 	.word	0x00004d53

08000c98 <.text_12>:
 8000c98:	00444150 	.word	0x00444150

08000c9c <ai_layer_type_is_valid>:
 8000c9c:	f242 7111 	movw	r1, #10001	; 0x2711
 8000ca0:	1a40      	subs	r0, r0, r1
 8000ca2:	2801      	cmp	r0, #1
 8000ca4:	bf81      	itttt	hi
 8000ca6:	1ec0      	subhi	r0, r0, #3
 8000ca8:	280d      	cmphi	r0, #13
 8000caa:	380f      	subhi	r0, #15
 8000cac:	2809      	cmphi	r0, #9
 8000cae:	d801      	bhi.n	8000cb4 <ai_layer_type_is_valid+0x18>
 8000cb0:	2001      	movs	r0, #1
 8000cb2:	4770      	bx	lr
 8000cb4:	2000      	movs	r0, #0
 8000cb6:	4770      	bx	lr

08000cb8 <ai_layers_forward_all>:
 8000cb8:	b530      	push	{r4, r5, lr}
 8000cba:	4604      	mov	r4, r0
 8000cbc:	b081      	sub	sp, #4
 8000cbe:	6d20      	ldr	r0, [r4, #80]	; 0x50
 8000cc0:	b158      	cbz	r0, 8000cda <ai_layers_forward_all+0x22>
 8000cc2:	6560      	str	r0, [r4, #84]	; 0x54
 8000cc4:	6d65      	ldr	r5, [r4, #84]	; 0x54
 8000cc6:	6929      	ldr	r1, [r5, #16]
 8000cc8:	4628      	mov	r0, r5
 8000cca:	4788      	blx	r1
 8000ccc:	68e8      	ldr	r0, [r5, #12]
 8000cce:	42a8      	cmp	r0, r5
 8000cd0:	bf08      	it	eq
 8000cd2:	2000      	moveq	r0, #0
 8000cd4:	2800      	cmp	r0, #0
 8000cd6:	6560      	str	r0, [r4, #84]	; 0x54
 8000cd8:	d1f4      	bne.n	8000cc4 <ai_layers_forward_all+0xc>
 8000cda:	b001      	add	sp, #4
 8000cdc:	bd30      	pop	{r4, r5, pc}
	...

08000ce0 <.text_15>:
 8000ce0:	564e4f43 	.word	0x564e4f43
 8000ce4:	00004432 	.word	0x00004432

08000ce8 <.text_16>:
 8000ce8:	534e4544 	.word	0x534e4544
 8000cec:	0045      	.short	0x0045
	...

08000cf0 <.text_17>:
 8000cf0:	4d54534c 	.word	0x4d54534c
 8000cf4:	00          	.byte	0x00
 8000cf5:	00          	.byte	0x00
	...

08000cf8 <.text_18>:
 8000cf8:	4d524f4e 	.word	0x4d524f4e
 8000cfc:	00          	.byte	0x00
 8000cfd:	00          	.byte	0x00
	...

08000d00 <.text_19>:
 8000d00:	4954504f 	.word	0x4954504f
 8000d04:	455a494d 	.word	0x455a494d
 8000d08:	4f435f44 	.word	0x4f435f44
 8000d0c:	4432564e 	.word	0x4432564e
 8000d10:	00          	.byte	0x00
 8000d11:	00          	.byte	0x00
	...

08000d14 <.text_20>:
 8000d14:	4e415254 	.word	0x4e415254
 8000d18:	534f5053 	.word	0x534f5053
 8000d1c:	0045      	.short	0x0045
	...

08000d20 <.text_21>:
 8000d20:	4c4f4f50 	.word	0x4c4f4f50
 8000d24:	00          	.byte	0x00
 8000d25:	00          	.byte	0x00
	...

08000d28 <.text_22>:
 8000d28:	494c5053 	.word	0x494c5053
 8000d2c:	0054      	.short	0x0054
	...

08000d30 <.text_23>:
 8000d30:	454d4954 	.word	0x454d4954
 8000d34:	4c45445f 	.word	0x4c45445f
 8000d38:	00005941 	.word	0x00005941

08000d3c <.text_24>:
 8000d3c:	454d4954 	.word	0x454d4954
 8000d40:	5349445f 	.word	0x5349445f
 8000d44:	42495254 	.word	0x42495254
 8000d48:	44455455 	.word	0x44455455
 8000d4c:	00          	.byte	0x00
 8000d4d:	00          	.byte	0x00
	...

08000d50 <.text_25>:
 8000d50:	434e4f43 	.word	0x434e4f43
 8000d54:	00005441 	.word	0x00005441

08000d58 <.text_26>:
 8000d58:	4d4d4547 	.word	0x4d4d4547
 8000d5c:	00          	.byte	0x00
 8000d5d:	00          	.byte	0x00
	...

08000d60 <.text_27>:
 8000d60:	41535055 	.word	0x41535055
 8000d64:	454c504d 	.word	0x454c504d
 8000d68:	00          	.byte	0x00
 8000d69:	00          	.byte	0x00
	...

08000d6c <.text_28>:
 8000d6c:	57544c45 	.word	0x57544c45
 8000d70:	00455349 	.word	0x00455349

08000d74 <.text_29>:
 8000d74:	454e4547 	.word	0x454e4547
 8000d78:	00434952 	.word	0x00434952

08000d7c <.text_30>:
 8000d7c:	54534e49 	.word	0x54534e49
 8000d80:	45434e41 	.word	0x45434e41
 8000d84:	4d524f4e 	.word	0x4d524f4e
 8000d88:	5a494c41 	.word	0x5a494c41
 8000d8c:	4f495441 	.word	0x4f495441
 8000d90:	004e      	.short	0x004e
	...

08000d94 <.text_31>:
 8000d94:	43494c53 	.word	0x43494c53
 8000d98:	0045      	.short	0x0045
	...

08000d9c <.text_32>:
 8000d9c:	454c4954 	.word	0x454c4954
 8000da0:	00          	.byte	0x00
 8000da1:	00          	.byte	0x00
	...

08000da4 <.text_33>:
 8000da4:	55444552 	.word	0x55444552
 8000da8:	00004543 	.word	0x00004543

08000dac <ai_check_custom_types::ref_signatures>:
 8000dac:	84048403                                ....

08000db0 <ai_conv2d_stripe_f32>:
 8000db0:	e92d 4ff0 	stmdb	sp!, {r4, r5, r6, r7, r8, r9, sl, fp, lr}
 8000db4:	b098      	sub	sp, #96	; 0x60
 8000db6:	9825      	ldr	r0, [sp, #148]	; 0x94
 8000db8:	2800      	cmp	r0, #0
 8000dba:	f000 82cb 	beq.w	8001354 <ai_conv2d_stripe_f32+0x5a4>
 8000dbe:	f9bd 40c0 	ldrsh.w	r4, [sp, #192]	; 0xc0
 8000dc2:	f8dd a0b4 	ldr.w	sl, [sp, #180]	; 0xb4
 8000dc6:	9d2b      	ldr	r5, [sp, #172]	; 0xac
 8000dc8:	9f24      	ldr	r7, [sp, #144]	; 0x90
 8000dca:	9e2c      	ldr	r6, [sp, #176]	; 0xb0
 8000dcc:	9004      	str	r0, [sp, #16]
 8000dce:	fb07 6a0a 	mla	sl, r7, sl, r6
 8000dd2:	982a      	ldr	r0, [sp, #168]	; 0xa8
 8000dd4:	f9bd 60c0 	ldrsh.w	r6, [sp, #192]	; 0xc0
 8000dd8:	f8cd a014 	str.w	sl, [sp, #20]
 8000ddc:	1904      	adds	r4, r0, r4
 8000dde:	1e64      	subs	r4, r4, #1
 8000de0:	9826      	ldr	r0, [sp, #152]	; 0x98
 8000de2:	9100      	str	r1, [sp, #0]
 8000de4:	fb94 f6f6 	sdiv	r6, r4, r6
 8000de8:	f9bd 40bc 	ldrsh.w	r4, [sp, #188]	; 0xbc
 8000dec:	9217      	str	r2, [sp, #92]	; 0x5c
 8000dee:	4346      	muls	r6, r0
 8000df0:	9616      	str	r6, [sp, #88]	; 0x58
 8000df2:	eeb7 0a00 	vmov.f32	s0, #112	; 0x3f800000  1.0
 8000df6:	9e2a      	ldr	r6, [sp, #168]	; 0xa8
 8000df8:	9822      	ldr	r0, [sp, #136]	; 0x88
 8000dfa:	9306      	str	r3, [sp, #24]
 8000dfc:	4344      	muls	r4, r0
 8000dfe:	9415      	str	r4, [sp, #84]	; 0x54
 8000e00:	437e      	muls	r6, r7
 8000e02:	f9bd 40c0 	ldrsh.w	r4, [sp, #192]	; 0xc0
 8000e06:	437c      	muls	r4, r7
 8000e08:	9414      	str	r4, [sp, #80]	; 0x50
 8000e0a:	4346      	muls	r6, r0
 8000e0c:	f9bd 40c0 	ldrsh.w	r4, [sp, #192]	; 0xc0
 8000e10:	982a      	ldr	r0, [sp, #168]	; 0xa8
 8000e12:	960b      	str	r6, [sp, #44]	; 0x2c
 8000e14:	1a24      	subs	r4, r4, r0
 8000e16:	9413      	str	r4, [sp, #76]	; 0x4c
 8000e18:	4604      	mov	r4, r0
 8000e1a:	9826      	ldr	r0, [sp, #152]	; 0x98
 8000e1c:	9e26      	ldr	r6, [sp, #152]	; 0x98
 8000e1e:	4344      	muls	r4, r0
 8000e20:	9412      	str	r4, [sp, #72]	; 0x48
 8000e22:	9c2a      	ldr	r4, [sp, #168]	; 0xa8
 8000e24:	4344      	muls	r4, r0
 8000e26:	9411      	str	r4, [sp, #68]	; 0x44
 8000e28:	f9bd 00c0 	ldrsh.w	r0, [sp, #192]	; 0xc0
 8000e2c:	f9bd 40bc 	ldrsh.w	r4, [sp, #188]	; 0xbc
 8000e30:	fb14 f000 	smulbb	r0, r4, r0
 8000e34:	900a      	str	r0, [sp, #40]	; 0x28
 8000e36:	9c23      	ldr	r4, [sp, #140]	; 0x8c
 8000e38:	9829      	ldr	r0, [sp, #164]	; 0xa4
 8000e3a:	fbb4 f0f0 	udiv	r0, r4, r0
 8000e3e:	9010      	str	r0, [sp, #64]	; 0x40
 8000e40:	9c22      	ldr	r4, [sp, #136]	; 0x88
 8000e42:	9829      	ldr	r0, [sp, #164]	; 0xa4
 8000e44:	fbb4 f0f0 	udiv	r0, r4, r0
 8000e48:	900f      	str	r0, [sp, #60]	; 0x3c
 8000e4a:	9c23      	ldr	r4, [sp, #140]	; 0x8c
 8000e4c:	9822      	ldr	r0, [sp, #136]	; 0x88
 8000e4e:	fbb4 f0f0 	udiv	r0, r4, r0
 8000e52:	9c22      	ldr	r4, [sp, #136]	; 0x88
 8000e54:	900e      	str	r0, [sp, #56]	; 0x38
 8000e56:	4374      	muls	r4, r6
 8000e58:	940d      	str	r4, [sp, #52]	; 0x34
 8000e5a:	9c2a      	ldr	r4, [sp, #168]	; 0xa8
 8000e5c:	1b2d      	subs	r5, r5, r4
 8000e5e:	950c      	str	r5, [sp, #48]	; 0x30
 8000e60:	9f2c      	ldr	r7, [sp, #176]	; 0xb0
 8000e62:	9924      	ldr	r1, [sp, #144]	; 0x90
 8000e64:	982c      	ldr	r0, [sp, #176]	; 0xb0
 8000e66:	9a2e      	ldr	r2, [sp, #184]	; 0xb8
 8000e68:	427f      	negs	r7, r7
 8000e6a:	bfd8      	it	le
 8000e6c:	2700      	movle	r7, #0
 8000e6e:	1a09      	subs	r1, r1, r0
 8000e70:	4291      	cmp	r1, r2
 8000e72:	bf3d      	ittte	cc
 8000e74:	9824      	ldrcc	r0, [sp, #144]	; 0x90
 8000e76:	9e2c      	ldrcc	r6, [sp, #176]	; 0xb0
 8000e78:	1b86      	subcc	r6, r0, r6
 8000e7a:	4616      	movcs	r6, r2
 8000e7c:	9a05      	ldr	r2, [sp, #20]
 8000e7e:	9922      	ldr	r1, [sp, #136]	; 0x88
 8000e80:	9817      	ldr	r0, [sp, #92]	; 0x5c
 8000e82:	18ba      	adds	r2, r7, r2
 8000e84:	434a      	muls	r2, r1
 8000e86:	eb00 0282 	add.w	r2, r0, r2, lsl #2
 8000e8a:	9821      	ldr	r0, [sp, #132]	; 0x84
 8000e8c:	b900      	cbnz	r0, 8000e90 <ai_conv2d_stripe_f32+0xe0>
 8000e8e:	9800      	ldr	r0, [sp, #0]
 8000e90:	9001      	str	r0, [sp, #4]
 8000e92:	1bf6      	subs	r6, r6, r7
 8000e94:	9829      	ldr	r0, [sp, #164]	; 0xa4
 8000e96:	9d0c      	ldr	r5, [sp, #48]	; 0x30
 8000e98:	2801      	cmp	r0, #1
 8000e9a:	bf04      	itt	eq
 8000e9c:	980a      	ldreq	r0, [sp, #40]	; 0x28
 8000e9e:	2801      	cmpeq	r0, #1
 8000ea0:	f040 80a9 	bne.w	8000ff6 <ai_conv2d_stripe_f32+0x246>
 8000ea4:	9c24      	ldr	r4, [sp, #144]	; 0x90
 8000ea6:	9826      	ldr	r0, [sp, #152]	; 0x98
 8000ea8:	9b0d      	ldr	r3, [sp, #52]	; 0x34
 8000eaa:	1ba4      	subs	r4, r4, r6
 8000eac:	434c      	muls	r4, r1
 8000eae:	1b80      	subs	r0, r0, r6
 8000eb0:	4341      	muls	r1, r0
 8000eb2:	9827      	ldr	r0, [sp, #156]	; 0x9c
 8000eb4:	1b40      	subs	r0, r0, r5
 8000eb6:	fb00 fc03 	mul.w	ip, r0, r3
 8000eba:	9811      	ldr	r0, [sp, #68]	; 0x44
 8000ebc:	9b06      	ldr	r3, [sp, #24]
 8000ebe:	4407      	add	r7, r0
 8000ec0:	9822      	ldr	r0, [sp, #136]	; 0x88
 8000ec2:	4347      	muls	r7, r0
 8000ec4:	eb03 0787 	add.w	r7, r3, r7, lsl #2
 8000ec8:	4370      	muls	r0, r6
 8000eca:	9e01      	ldr	r6, [sp, #4]
 8000ecc:	9b00      	ldr	r3, [sp, #0]
 8000ece:	429e      	cmp	r6, r3
 8000ed0:	9b0b      	ldr	r3, [sp, #44]	; 0x2c
 8000ed2:	eb02 0983 	add.w	r9, r2, r3, lsl #2
 8000ed6:	9a23      	ldr	r2, [sp, #140]	; 0x8c
 8000ed8:	bf0c      	ite	eq
 8000eda:	eddf 0aaf 	vldreq	s1, [pc, #700]	; 8001198 <ai_conv2d_stripe_f32+0x3e8>
 8000ede:	eef0 0a40 	vmovne.f32	s1, s0
 8000ee2:	2a00      	cmp	r2, #0
 8000ee4:	f000 8222 	beq.w	800132c <ai_conv2d_stripe_f32+0x57c>
 8000ee8:	46b0      	mov	r8, r6
 8000eea:	462e      	mov	r6, r5
 8000eec:	4613      	mov	r3, r2
 8000eee:	f8cd c008 	str.w	ip, [sp, #8]
 8000ef2:	461d      	mov	r5, r3
 8000ef4:	f8dd e000 	ldr.w	lr, [sp]
 8000ef8:	9b00      	ldr	r3, [sp, #0]
 8000efa:	463a      	mov	r2, r7
 8000efc:	4682      	mov	sl, r0
 8000efe:	f8cd 9004 	str.w	r9, [sp, #4]
 8000f02:	46c4      	mov	ip, r8
 8000f04:	f02a 0703 	bic.w	r7, sl, #3
 8000f08:	ed9c 1a00 	vldr	s2, [ip]
 8000f0c:	f8dd 8004 	ldr.w	r8, [sp, #4]
 8000f10:	2e00      	cmp	r6, #0
 8000f12:	ee21 1a20 	vmul.f32	s2, s2, s1
 8000f16:	dd61      	ble.n	8000fdc <ai_conv2d_stripe_f32+0x22c>
 8000f18:	4630      	mov	r0, r6
 8000f1a:	2f00      	cmp	r7, #0
 8000f1c:	f04f 0900 	mov.w	r9, #0
 8000f20:	f340 801f 	ble.w	8000f62 <ai_conv2d_stripe_f32+0x1b2>
 8000f24:	edd2 4a00 	vldr	s9, [r2]
 8000f28:	ed98 5a00 	vldr	s10, [r8]
 8000f2c:	edd2 3a01 	vldr	s7, [r2, #4]
 8000f30:	ed98 4a01 	vldr	s8, [r8, #4]
 8000f34:	edd2 2a02 	vldr	s5, [r2, #8]
 8000f38:	ed98 3a02 	vldr	s6, [r8, #8]
 8000f3c:	edd2 1a03 	vldr	s3, [r2, #12]
 8000f40:	ed98 2a03 	vldr	s4, [r8, #12]
 8000f44:	ee04 1a85 	vmla.f32	s2, s9, s10
 8000f48:	ee03 1a84 	vmla.f32	s2, s7, s8
 8000f4c:	3210      	adds	r2, #16
 8000f4e:	f109 0904 	add.w	r9, r9, #4
 8000f52:	ee02 1a83 	vmla.f32	s2, s5, s6
 8000f56:	45b9      	cmp	r9, r7
 8000f58:	ee01 1a82 	vmla.f32	s2, s3, s4
 8000f5c:	f108 0810 	add.w	r8, r8, #16
 8000f60:	dbe0      	blt.n	8000f24 <ai_conv2d_stripe_f32+0x174>
 8000f62:	45d1      	cmp	r9, sl
 8000f64:	f280 8034 	bge.w	8000fd0 <ai_conv2d_stripe_f32+0x220>
 8000f68:	f109 0901 	add.w	r9, r9, #1
 8000f6c:	edd2 2a00 	vldr	s5, [r2]
 8000f70:	edd8 1a00 	vldr	s3, [r8]
 8000f74:	1d12      	adds	r2, r2, #4
 8000f76:	45d1      	cmp	r9, sl
 8000f78:	ee02 1aa1 	vmla.f32	s2, s5, s3
 8000f7c:	f108 0804 	add.w	r8, r8, #4
 8000f80:	da26      	bge.n	8000fd0 <ai_conv2d_stripe_f32+0x220>
 8000f82:	f109 0901 	add.w	r9, r9, #1
 8000f86:	ed92 3a00 	vldr	s6, [r2]
 8000f8a:	ed98 2a00 	vldr	s4, [r8]
 8000f8e:	1d12      	adds	r2, r2, #4
 8000f90:	45d1      	cmp	r9, sl
 8000f92:	ee03 1a02 	vmla.f32	s2, s6, s4
 8000f96:	f108 0804 	add.w	r8, r8, #4
 8000f9a:	da19      	bge.n	8000fd0 <ai_conv2d_stripe_f32+0x220>
 8000f9c:	f109 0901 	add.w	r9, r9, #1
 8000fa0:	edd2 2a00 	vldr	s5, [r2]
 8000fa4:	edd8 1a00 	vldr	s3, [r8]
 8000fa8:	1d12      	adds	r2, r2, #4
 8000faa:	45d1      	cmp	r9, sl
 8000fac:	ee02 1aa1 	vmla.f32	s2, s5, s3
 8000fb0:	f108 0804 	add.w	r8, r8, #4
 8000fb4:	da0c      	bge.n	8000fd0 <ai_conv2d_stripe_f32+0x220>
 8000fb6:	f109 0901 	add.w	r9, r9, #1
 8000fba:	ed92 2a00 	vldr	s4, [r2]
 8000fbe:	ed98 3a00 	vldr	s6, [r8]
 8000fc2:	1d12      	adds	r2, r2, #4
 8000fc4:	45d1      	cmp	r9, sl
 8000fc6:	ee02 1a03 	vmla.f32	s2, s4, s6
 8000fca:	f108 0804 	add.w	r8, r8, #4
 8000fce:	dbcb      	blt.n	8000f68 <ai_conv2d_stripe_f32+0x1b8>
 8000fd0:	1e40      	subs	r0, r0, #1
 8000fd2:	eb08 0884 	add.w	r8, r8, r4, lsl #2
 8000fd6:	eb02 0281 	add.w	r2, r2, r1, lsl #2
 8000fda:	d19e      	bne.n	8000f1a <ai_conv2d_stripe_f32+0x16a>
 8000fdc:	9802      	ldr	r0, [sp, #8]
 8000fde:	ed8e 1a00 	vstr	s2, [lr]
 8000fe2:	1e6d      	subs	r5, r5, #1
 8000fe4:	eb02 0280 	add.w	r2, r2, r0, lsl #2
 8000fe8:	f10e 0e04 	add.w	lr, lr, #4
 8000fec:	f10c 0c04 	add.w	ip, ip, #4
 8000ff0:	d18a      	bne.n	8000f08 <ai_conv2d_stripe_f32+0x158>
 8000ff2:	9300      	str	r3, [sp, #0]
 8000ff4:	e19a      	b.n	800132c <ai_conv2d_stripe_f32+0x57c>
 8000ff6:	9829      	ldr	r0, [sp, #164]	; 0xa4
 8000ff8:	4288      	cmp	r0, r1
 8000ffa:	bf04      	itt	eq
 8000ffc:	980a      	ldreq	r0, [sp, #40]	; 0x28
 8000ffe:	2801      	cmpeq	r0, #1
 8001000:	f040 80cc 	bne.w	800119c <ai_conv2d_stripe_f32+0x3ec>
 8001004:	980e      	ldr	r0, [sp, #56]	; 0x38
 8001006:	9b06      	ldr	r3, [sp, #24]
 8001008:	9c00      	ldr	r4, [sp, #0]
 800100a:	9002      	str	r0, [sp, #8]
 800100c:	9824      	ldr	r0, [sp, #144]	; 0x90
 800100e:	1b81      	subs	r1, r0, r6
 8001010:	9822      	ldr	r0, [sp, #136]	; 0x88
 8001012:	fb01 fa00 	mul.w	sl, r1, r0
 8001016:	9826      	ldr	r0, [sp, #152]	; 0x98
 8001018:	9926      	ldr	r1, [sp, #152]	; 0x98
 800101a:	eba0 0c06 	sub.w	ip, r0, r6
 800101e:	9827      	ldr	r0, [sp, #156]	; 0x9c
 8001020:	1b40      	subs	r0, r0, r5
 8001022:	4341      	muls	r1, r0
 8001024:	9812      	ldr	r0, [sp, #72]	; 0x48
 8001026:	183f      	adds	r7, r7, r0
 8001028:	eb03 0087 	add.w	r0, r3, r7, lsl #2
 800102c:	9b01      	ldr	r3, [sp, #4]
 800102e:	42a3      	cmp	r3, r4
 8001030:	9b0b      	ldr	r3, [sp, #44]	; 0x2c
 8001032:	eb02 0e83 	add.w	lr, r2, r3, lsl #2
 8001036:	bf0c      	ite	eq
 8001038:	eddf 0a57 	vldreq	s1, [pc, #348]	; 8001198 <ai_conv2d_stripe_f32+0x3e8>
 800103c:	eef0 0a40 	vmovne.f32	s1, s0
 8001040:	9b22      	ldr	r3, [sp, #136]	; 0x88
 8001042:	2400      	movs	r4, #0
 8001044:	eb0e 0283 	add.w	r2, lr, r3, lsl #2
 8001048:	4596      	cmp	lr, r2
 800104a:	9203      	str	r2, [sp, #12]
 800104c:	f080 816e 	bcs.w	800132c <ai_conv2d_stripe_f32+0x57c>
 8001050:	9b00      	ldr	r3, [sp, #0]
 8001052:	9a02      	ldr	r2, [sp, #8]
 8001054:	2a00      	cmp	r2, #0
 8001056:	f000 8097 	beq.w	8001188 <ai_conv2d_stripe_f32+0x3d8>
 800105a:	9a01      	ldr	r2, [sp, #4]
 800105c:	9500      	str	r5, [sp, #0]
 800105e:	eb02 0784 	add.w	r7, r2, r4, lsl #2
 8001062:	eb03 0284 	add.w	r2, r3, r4, lsl #2
 8001066:	f8dd b008 	ldr.w	fp, [sp, #8]
 800106a:	9108      	str	r1, [sp, #32]
 800106c:	f8cd e01c 	str.w	lr, [sp, #28]
 8001070:	4615      	mov	r5, r2
 8001072:	9a00      	ldr	r2, [sp, #0]
 8001074:	ed97 1a00 	vldr	s2, [r7]
 8001078:	9907      	ldr	r1, [sp, #28]
 800107a:	2a00      	cmp	r2, #0
 800107c:	ee21 1a20 	vmul.f32	s2, s2, s1
 8001080:	f340 8072 	ble.w	8001168 <ai_conv2d_stripe_f32+0x3b8>
 8001084:	f026 0e03 	bic.w	lr, r6, #3
 8001088:	f1be 0f00 	cmp.w	lr, #0
 800108c:	f04f 0900 	mov.w	r9, #0
 8001090:	f340 8029 	ble.w	80010e6 <ai_conv2d_stripe_f32+0x336>
 8001094:	f8dd 8088 	ldr.w	r8, [sp, #136]	; 0x88
 8001098:	edd0 1a00 	vldr	s3, [r0]
 800109c:	ed91 2a00 	vldr	s4, [r1]
 80010a0:	eb01 0188 	add.w	r1, r1, r8, lsl #2
 80010a4:	ee01 1a82 	vmla.f32	s2, s3, s4
 80010a8:	edd0 1a01 	vldr	s3, [r0, #4]
 80010ac:	ed91 2a00 	vldr	s4, [r1]
 80010b0:	eb01 0188 	add.w	r1, r1, r8, lsl #2
 80010b4:	ee01 1a82 	vmla.f32	s2, s3, s4
 80010b8:	edd0 1a02 	vldr	s3, [r0, #8]
 80010bc:	ed91 2a00 	vldr	s4, [r1]
 80010c0:	eb01 0188 	add.w	r1, r1, r8, lsl #2
 80010c4:	ee01 1a82 	vmla.f32	s2, s3, s4
 80010c8:	f109 0904 	add.w	r9, r9, #4
 80010cc:	edd0 1a03 	vldr	s3, [r0, #12]
 80010d0:	ed91 2a00 	vldr	s4, [r1]
 80010d4:	3010      	adds	r0, #16
 80010d6:	45f1      	cmp	r9, lr
 80010d8:	ee01 1a82 	vmla.f32	s2, s3, s4
 80010dc:	eb01 0188 	add.w	r1, r1, r8, lsl #2
 80010e0:	dbda      	blt.n	8001098 <ai_conv2d_stripe_f32+0x2e8>
 80010e2:	f8cd 8088 	str.w	r8, [sp, #136]	; 0x88
 80010e6:	45b1      	cmp	r9, r6
 80010e8:	f280 8038 	bge.w	800115c <ai_conv2d_stripe_f32+0x3ac>
 80010ec:	f8dd e088 	ldr.w	lr, [sp, #136]	; 0x88
 80010f0:	f109 0901 	add.w	r9, r9, #1
 80010f4:	edd0 1a00 	vldr	s3, [r0]
 80010f8:	ed91 2a00 	vldr	s4, [r1]
 80010fc:	1d00      	adds	r0, r0, #4
 80010fe:	45b1      	cmp	r9, r6
 8001100:	ee01 1a82 	vmla.f32	s2, s3, s4
 8001104:	eb01 018e 	add.w	r1, r1, lr, lsl #2
 8001108:	da26      	bge.n	8001158 <ai_conv2d_stripe_f32+0x3a8>
 800110a:	f109 0901 	add.w	r9, r9, #1
 800110e:	ed90 2a00 	vldr	s4, [r0]
 8001112:	edd1 1a00 	vldr	s3, [r1]
 8001116:	1d00      	adds	r0, r0, #4
 8001118:	45b1      	cmp	r9, r6
 800111a:	ee02 1a21 	vmla.f32	s2, s4, s3
 800111e:	eb01 018e 	add.w	r1, r1, lr, lsl #2
 8001122:	da19      	bge.n	8001158 <ai_conv2d_stripe_f32+0x3a8>
 8001124:	f109 0901 	add.w	r9, r9, #1
 8001128:	edd0 1a00 	vldr	s3, [r0]
 800112c:	ed91 2a00 	vldr	s4, [r1]
 8001130:	1d00      	adds	r0, r0, #4
 8001132:	45b1      	cmp	r9, r6
 8001134:	ee01 1a82 	vmla.f32	s2, s3, s4
 8001138:	eb01 018e 	add.w	r1, r1, lr, lsl #2
 800113c:	da0c      	bge.n	8001158 <ai_conv2d_stripe_f32+0x3a8>
 800113e:	f109 0901 	add.w	r9, r9, #1
 8001142:	ed90 2a00 	vldr	s4, [r0]
 8001146:	edd1 1a00 	vldr	s3, [r1]
 800114a:	1d00      	adds	r0, r0, #4
 800114c:	45b1      	cmp	r9, r6
 800114e:	ee02 1a21 	vmla.f32	s2, s4, s3
 8001152:	eb01 018e 	add.w	r1, r1, lr, lsl #2
 8001156:	dbcb      	blt.n	80010f0 <ai_conv2d_stripe_f32+0x340>
 8001158:	f8cd e088 	str.w	lr, [sp, #136]	; 0x88
 800115c:	1e52      	subs	r2, r2, #1
 800115e:	eb01 018a 	add.w	r1, r1, sl, lsl #2
 8001162:	eb00 008c 	add.w	r0, r0, ip, lsl #2
 8001166:	d18d      	bne.n	8001084 <ai_conv2d_stripe_f32+0x2d4>
 8001168:	9908      	ldr	r1, [sp, #32]
 800116a:	ed85 1a00 	vstr	s2, [r5]
 800116e:	1c64      	adds	r4, r4, #1
 8001170:	1d2d      	adds	r5, r5, #4
 8001172:	1d3f      	adds	r7, r7, #4
 8001174:	f1bb 0b01 	subs.w	fp, fp, #1
 8001178:	eb00 0081 	add.w	r0, r0, r1, lsl #2
 800117c:	f47f af79 	bne.w	8001072 <ai_conv2d_stripe_f32+0x2c2>
 8001180:	9d00      	ldr	r5, [sp, #0]
 8001182:	9908      	ldr	r1, [sp, #32]
 8001184:	f8dd e01c 	ldr.w	lr, [sp, #28]
 8001188:	9a03      	ldr	r2, [sp, #12]
 800118a:	f10e 0e04 	add.w	lr, lr, #4
 800118e:	4596      	cmp	lr, r2
 8001190:	f4bf af2f 	bcs.w	8000ff2 <ai_conv2d_stripe_f32+0x242>
 8001194:	e75d      	b.n	8001052 <ai_conv2d_stripe_f32+0x2a2>
 8001196:	bf00      	nop
 8001198:	00000000 	.word	0x00000000
 800119c:	f9bd 10bc 	ldrsh.w	r1, [sp, #188]	; 0xbc
 80011a0:	f8dd 9050 	ldr.w	r9, [sp, #80]	; 0x50
 80011a4:	4608      	mov	r0, r1
 80011a6:	1bcb      	subs	r3, r1, r7
 80011a8:	fb97 f4f0 	sdiv	r4, r7, r0
 80011ac:	fb00 3004 	mla	r0, r0, r4, r3
 80011b0:	fb90 faf1 	sdiv	sl, r0, r1
 80011b4:	fb01 0a1a 	mls	sl, r1, sl, r0
 80011b8:	f9bd 30c0 	ldrsh.w	r3, [sp, #192]	; 0xc0
 80011bc:	982a      	ldr	r0, [sp, #168]	; 0xa8
 80011be:	9c13      	ldr	r4, [sp, #76]	; 0x4c
 80011c0:	fb90 f0f3 	sdiv	r0, r0, r3
 80011c4:	fb03 4000 	mla	r0, r3, r0, r4
 80011c8:	1876      	adds	r6, r6, r1
 80011ca:	fb90 fbf3 	sdiv	fp, r0, r3
 80011ce:	1e76      	subs	r6, r6, #1
 80011d0:	187f      	adds	r7, r7, r1
 80011d2:	fb03 0b1b 	mls	fp, r3, fp, r0
 80011d6:	eba6 060a 	sub.w	r6, r6, sl
 80011da:	eba5 050b 	sub.w	r5, r5, fp
 80011de:	1e7f      	subs	r7, r7, #1
 80011e0:	fb96 f0f1 	sdiv	r0, r6, r1
 80011e4:	9e27      	ldr	r6, [sp, #156]	; 0x9c
 80011e6:	9c22      	ldr	r4, [sp, #136]	; 0x88
 80011e8:	195d      	adds	r5, r3, r5
 80011ea:	1e6d      	subs	r5, r5, #1
 80011ec:	fb00 9911 	mls	r9, r0, r1, r9
 80011f0:	fb97 f1f1 	sdiv	r1, r7, r1
 80011f4:	fb95 fcf3 	sdiv	ip, r5, r3
 80011f8:	9d10      	ldr	r5, [sp, #64]	; 0x40
 80011fa:	9b0f      	ldr	r3, [sp, #60]	; 0x3c
 80011fc:	9509      	str	r5, [sp, #36]	; 0x24
 80011fe:	eba6 060c 	sub.w	r6, r6, ip
 8001202:	9d26      	ldr	r5, [sp, #152]	; 0x98
 8001204:	1a2d      	subs	r5, r5, r0
 8001206:	fb05 f803 	mul.w	r8, r5, r3
 800120a:	9d26      	ldr	r5, [sp, #152]	; 0x98
 800120c:	435d      	muls	r5, r3
 800120e:	fb06 fe05 	mul.w	lr, r6, r5
 8001212:	9d16      	ldr	r5, [sp, #88]	; 0x58
 8001214:	9e06      	ldr	r6, [sp, #24]
 8001216:	194d      	adds	r5, r1, r5
 8001218:	fb04 f909 	mul.w	r9, r4, r9
 800121c:	435d      	muls	r5, r3
 800121e:	9c15      	ldr	r4, [sp, #84]	; 0x54
 8001220:	eb06 0185 	add.w	r1, r6, r5, lsl #2
 8001224:	9d01      	ldr	r5, [sp, #4]
 8001226:	9e00      	ldr	r6, [sp, #0]
 8001228:	1ae4      	subs	r4, r4, r3
 800122a:	42b5      	cmp	r5, r6
 800122c:	9d2a      	ldr	r5, [sp, #168]	; 0xa8
 800122e:	9e24      	ldr	r6, [sp, #144]	; 0x90
 8001230:	445d      	add	r5, fp
 8001232:	fb06 aa05 	mla	sl, r6, r5, sl
 8001236:	9d22      	ldr	r5, [sp, #136]	; 0x88
 8001238:	fb0a f505 	mul.w	r5, sl, r5
 800123c:	bf0c      	ite	eq
 800123e:	eddf 0a9e 	vldreq	s1, [pc, #632]	; 80014b8 <.text_5>
 8001242:	eef0 0a40 	vmovne.f32	s1, s0
 8001246:	eb02 0785 	add.w	r7, r2, r5, lsl #2
 800124a:	9a29      	ldr	r2, [sp, #164]	; 0xa4
 800124c:	2500      	movs	r5, #0
 800124e:	2a00      	cmp	r2, #0
 8001250:	d06c      	beq.n	800132c <ai_conv2d_stripe_f32+0x57c>
 8001252:	9202      	str	r2, [sp, #8]
 8001254:	9a09      	ldr	r2, [sp, #36]	; 0x24
 8001256:	2a00      	cmp	r2, #0
 8001258:	d062      	beq.n	8001320 <ai_conv2d_stripe_f32+0x570>
 800125a:	9a01      	ldr	r2, [sp, #4]
 800125c:	eb02 0685 	add.w	r6, r2, r5, lsl #2
 8001260:	9a00      	ldr	r2, [sp, #0]
 8001262:	f8cd c00c 	str.w	ip, [sp, #12]
 8001266:	eb02 0a85 	add.w	sl, r2, r5, lsl #2
 800126a:	9a09      	ldr	r2, [sp, #36]	; 0x24
 800126c:	f8cd e020 	str.w	lr, [sp, #32]
 8001270:	f8cd 701c 	str.w	r7, [sp, #28]
 8001274:	f8dd e00c 	ldr.w	lr, [sp, #12]
 8001278:	ed96 1a00 	vldr	s2, [r6]
 800127c:	9f07      	ldr	r7, [sp, #28]
 800127e:	f1be 0f00 	cmp.w	lr, #0
 8001282:	ee21 1a20 	vmul.f32	s2, s2, s1
 8001286:	dd3b      	ble.n	8001300 <ai_conv2d_stripe_f32+0x550>
 8001288:	2800      	cmp	r0, #0
 800128a:	dd32      	ble.n	80012f2 <ai_conv2d_stripe_f32+0x542>
 800128c:	ea4f 0c00 	mov.w	ip, r0
 8001290:	eb07 0b83 	add.w	fp, r7, r3, lsl #2
 8001294:	455f      	cmp	r7, fp
 8001296:	d227      	bcs.n	80012e8 <ai_conv2d_stripe_f32+0x538>
 8001298:	edd1 2a00 	vldr	s5, [r1]
 800129c:	edd7 1a00 	vldr	s3, [r7]
 80012a0:	1d09      	adds	r1, r1, #4
 80012a2:	1d3f      	adds	r7, r7, #4
 80012a4:	455f      	cmp	r7, fp
 80012a6:	ee02 1aa1 	vmla.f32	s2, s5, s3
 80012aa:	d21d      	bcs.n	80012e8 <ai_conv2d_stripe_f32+0x538>
 80012ac:	ed91 3a00 	vldr	s6, [r1]
 80012b0:	ed97 2a00 	vldr	s4, [r7]
 80012b4:	1d09      	adds	r1, r1, #4
 80012b6:	1d3f      	adds	r7, r7, #4
 80012b8:	455f      	cmp	r7, fp
 80012ba:	ee03 1a02 	vmla.f32	s2, s6, s4
 80012be:	d213      	bcs.n	80012e8 <ai_conv2d_stripe_f32+0x538>
 80012c0:	edd1 2a00 	vldr	s5, [r1]
 80012c4:	edd7 1a00 	vldr	s3, [r7]
 80012c8:	1d09      	adds	r1, r1, #4
 80012ca:	1d3f      	adds	r7, r7, #4
 80012cc:	455f      	cmp	r7, fp
 80012ce:	ee02 1aa1 	vmla.f32	s2, s5, s3
 80012d2:	d209      	bcs.n	80012e8 <ai_conv2d_stripe_f32+0x538>
 80012d4:	ed91 2a00 	vldr	s4, [r1]
 80012d8:	ed97 3a00 	vldr	s6, [r7]
 80012dc:	1d09      	adds	r1, r1, #4
 80012de:	1d3f      	adds	r7, r7, #4
 80012e0:	455f      	cmp	r7, fp
 80012e2:	ee02 1a03 	vmla.f32	s2, s4, s6
 80012e6:	d3d7      	bcc.n	8001298 <ai_conv2d_stripe_f32+0x4e8>
 80012e8:	f1bc 0c01 	subs.w	ip, ip, #1
 80012ec:	eb07 0784 	add.w	r7, r7, r4, lsl #2
 80012f0:	d1ce      	bne.n	8001290 <ai_conv2d_stripe_f32+0x4e0>
 80012f2:	f1be 0e01 	subs.w	lr, lr, #1
 80012f6:	eb07 0789 	add.w	r7, r7, r9, lsl #2
 80012fa:	eb01 0188 	add.w	r1, r1, r8, lsl #2
 80012fe:	d1c3      	bne.n	8001288 <ai_conv2d_stripe_f32+0x4d8>
 8001300:	9f08      	ldr	r7, [sp, #32]
 8001302:	1c6d      	adds	r5, r5, #1
 8001304:	1d36      	adds	r6, r6, #4
 8001306:	ed8a 1a00 	vstr	s2, [sl]
 800130a:	1e52      	subs	r2, r2, #1
 800130c:	eb01 0187 	add.w	r1, r1, r7, lsl #2
 8001310:	f10a 0a04 	add.w	sl, sl, #4
 8001314:	d1ae      	bne.n	8001274 <ai_conv2d_stripe_f32+0x4c4>
 8001316:	f8dd c00c 	ldr.w	ip, [sp, #12]
 800131a:	f8dd e020 	ldr.w	lr, [sp, #32]
 800131e:	9f07      	ldr	r7, [sp, #28]
 8001320:	9a02      	ldr	r2, [sp, #8]
 8001322:	1e52      	subs	r2, r2, #1
 8001324:	eb07 0783 	add.w	r7, r7, r3, lsl #2
 8001328:	9202      	str	r2, [sp, #8]
 800132a:	d193      	bne.n	8001254 <ai_conv2d_stripe_f32+0x4a4>
 800132c:	9800      	ldr	r0, [sp, #0]
 800132e:	9923      	ldr	r1, [sp, #140]	; 0x8c
 8001330:	eb00 0281 	add.w	r2, r0, r1, lsl #2
 8001334:	982c      	ldr	r0, [sp, #176]	; 0xb0
 8001336:	f8bd 10a0 	ldrh.w	r1, [sp, #160]	; 0xa0
 800133a:	9200      	str	r2, [sp, #0]
 800133c:	1841      	adds	r1, r0, r1
 800133e:	912c      	str	r1, [sp, #176]	; 0xb0
 8001340:	9805      	ldr	r0, [sp, #20]
 8001342:	f8bd 10a0 	ldrh.w	r1, [sp, #160]	; 0xa0
 8001346:	1841      	adds	r1, r0, r1
 8001348:	9804      	ldr	r0, [sp, #16]
 800134a:	9105      	str	r1, [sp, #20]
 800134c:	1e40      	subs	r0, r0, #1
 800134e:	9004      	str	r0, [sp, #16]
 8001350:	f47f ad86 	bne.w	8000e60 <ai_conv2d_stripe_f32+0xb0>
 8001354:	b018      	add	sp, #96	; 0x60
 8001356:	e8bd 8ff0 	ldmia.w	sp!, {r4, r5, r6, r7, r8, r9, sl, fp, pc}

0800135a <func_dummy>:
 800135a:	4770      	bx	lr

0800135c <ai_dict8_dot_array_f32>:
 800135c:	e92d 4ff0 	stmdb	sp!, {r4, r5, r6, r7, r8, r9, sl, fp, lr}
 8001360:	b081      	sub	sp, #4
 8001362:	4682      	mov	sl, r0
 8001364:	ed2d 8b02 	vpush	{d8}
 8001368:	4615      	mov	r5, r2
 800136a:	9c0c      	ldr	r4, [sp, #48]	; 0x30
 800136c:	08e0      	lsrs	r0, r4, #3
 800136e:	460f      	mov	r7, r1
 8001370:	461a      	mov	r2, r3
 8001372:	ed9f 0a51 	vldr	s0, [pc, #324]	; 80014b8 <.text_5>
 8001376:	d052      	beq.n	800141e <ai_dict8_dot_array_f32+0xc2>
 8001378:	4629      	mov	r1, r5
 800137a:	783b      	ldrb	r3, [r7, #0]
 800137c:	787d      	ldrb	r5, [r7, #1]
 800137e:	78be      	ldrb	r6, [r7, #2]
 8001380:	f897 b003 	ldrb.w	fp, [r7, #3]
 8001384:	ed92 8a00 	vldr	s16, [r2]
 8001388:	ed92 7a01 	vldr	s14, [r2, #4]
 800138c:	f817 cf04 	ldrb.w	ip, [r7, #4]!
 8001390:	ed92 6a02 	vldr	s12, [r2, #8]
 8001394:	ed92 5a03 	vldr	s10, [r2, #12]
 8001398:	f897 e001 	ldrb.w	lr, [r7, #1]
 800139c:	f897 8002 	ldrb.w	r8, [r7, #2]
 80013a0:	f897 9003 	ldrb.w	r9, [r7, #3]
 80013a4:	ed92 4a04 	vldr	s8, [r2, #16]
 80013a8:	ed92 3a05 	vldr	s6, [r2, #20]
 80013ac:	ed92 2a06 	vldr	s4, [r2, #24]
 80013b0:	ed92 1a07 	vldr	s2, [r2, #28]
 80013b4:	eb01 0383 	add.w	r3, r1, r3, lsl #2
 80013b8:	eb01 0585 	add.w	r5, r1, r5, lsl #2
 80013bc:	eb01 0686 	add.w	r6, r1, r6, lsl #2
 80013c0:	edd3 7a00 	vldr	s15, [r3]
 80013c4:	edd5 6a00 	vldr	s13, [r5]
 80013c8:	eb01 0b8b 	add.w	fp, r1, fp, lsl #2
 80013cc:	ee07 0a88 	vmla.f32	s0, s15, s16
 80013d0:	eb01 0c8c 	add.w	ip, r1, ip, lsl #2
 80013d4:	edd6 5a00 	vldr	s11, [r6]
 80013d8:	eddb 4a00 	vldr	s9, [fp]
 80013dc:	eddc 3a00 	vldr	s7, [ip]
 80013e0:	ee06 0a87 	vmla.f32	s0, s13, s14
 80013e4:	eb01 0e8e 	add.w	lr, r1, lr, lsl #2
 80013e8:	ee05 0a86 	vmla.f32	s0, s11, s12
 80013ec:	eb01 0888 	add.w	r8, r1, r8, lsl #2
 80013f0:	ee04 0a85 	vmla.f32	s0, s9, s10
 80013f4:	eb01 0989 	add.w	r9, r1, r9, lsl #2
 80013f8:	edde 2a00 	vldr	s5, [lr]
 80013fc:	edd8 1a00 	vldr	s3, [r8]
 8001400:	edd9 0a00 	vldr	s1, [r9]
 8001404:	ee03 0a84 	vmla.f32	s0, s7, s8
 8001408:	1d3f      	adds	r7, r7, #4
 800140a:	ee02 0a83 	vmla.f32	s0, s5, s6
 800140e:	3220      	adds	r2, #32
 8001410:	ee01 0a82 	vmla.f32	s0, s3, s4
 8001414:	1e40      	subs	r0, r0, #1
 8001416:	ee00 0a81 	vmla.f32	s0, s1, s2
 800141a:	d1ae      	bne.n	800137a <ai_dict8_dot_array_f32+0x1e>
 800141c:	460d      	mov	r5, r1
 800141e:	f014 0007 	ands.w	r0, r4, #7
 8001422:	d03e      	beq.n	80014a2 <ai_dict8_dot_array_f32+0x146>
 8001424:	f010 0103 	ands.w	r1, r0, #3
 8001428:	f000 800d 	beq.w	8001446 <ai_dict8_dot_array_f32+0xea>
 800142c:	f817 3b01 	ldrb.w	r3, [r7], #1
 8001430:	ed92 1a00 	vldr	s2, [r2]
 8001434:	eb05 0683 	add.w	r6, r5, r3, lsl #2
 8001438:	1d12      	adds	r2, r2, #4
 800143a:	edd6 0a00 	vldr	s1, [r6]
 800143e:	1e49      	subs	r1, r1, #1
 8001440:	ee00 0a81 	vmla.f32	s0, s1, s2
 8001444:	d1f2      	bne.n	800142c <ai_dict8_dot_array_f32+0xd0>
 8001446:	0880      	lsrs	r0, r0, #2
 8001448:	f000 802b 	beq.w	80014a2 <ai_dict8_dot_array_f32+0x146>
 800144c:	f817 3b01 	ldrb.w	r3, [r7], #1
 8001450:	f817 1b01 	ldrb.w	r1, [r7], #1
 8001454:	ed92 1a00 	vldr	s2, [r2]
 8001458:	edd2 0a01 	vldr	s1, [r2, #4]
 800145c:	eb05 0383 	add.w	r3, r5, r3, lsl #2
 8001460:	eb05 0181 	add.w	r1, r5, r1, lsl #2
 8001464:	ed93 2a00 	vldr	s4, [r3]
 8001468:	edd1 1a00 	vldr	s3, [r1]
 800146c:	f817 1b01 	ldrb.w	r1, [r7], #1
 8001470:	f817 3b01 	ldrb.w	r3, [r7], #1
 8001474:	ee02 0a01 	vmla.f32	s0, s4, s2
 8001478:	eb05 0181 	add.w	r1, r5, r1, lsl #2
 800147c:	ee01 0aa0 	vmla.f32	s0, s3, s1
 8001480:	eb05 0383 	add.w	r3, r5, r3, lsl #2
 8001484:	edd2 0a02 	vldr	s1, [r2, #8]
 8001488:	ed91 2a00 	vldr	s4, [r1]
 800148c:	ed92 1a03 	vldr	s2, [r2, #12]
 8001490:	edd3 1a00 	vldr	s3, [r3]
 8001494:	3210      	adds	r2, #16
 8001496:	ee02 0a20 	vmla.f32	s0, s4, s1
 800149a:	1e40      	subs	r0, r0, #1
 800149c:	ee01 0a81 	vmla.f32	s0, s3, s2
 80014a0:	d1d4      	bne.n	800144c <ai_dict8_dot_array_f32+0xf0>
 80014a2:	edda 0a00 	vldr	s1, [sl]
 80014a6:	ee30 0a80 	vadd.f32	s0, s1, s0
 80014aa:	ed8a 0a00 	vstr	s0, [sl]
 80014ae:	ecbd 8b02 	vpop	{d8}
 80014b2:	b001      	add	sp, #4
 80014b4:	e8bd 8ff0 	ldmia.w	sp!, {r4, r5, r6, r7, r8, r9, sl, fp, pc}

080014b8 <.text_5>:
 80014b8:	00000000 	.word	0x00000000

080014bc <ai_dict4_dot_array_f32>:
 80014bc:	e92d 47f0 	stmdb	sp!, {r4, r5, r6, r7, r8, r9, sl, lr}
 80014c0:	ed2d 8b02 	vpush	{d8}
 80014c4:	4680      	mov	r8, r0
 80014c6:	f8dd c028 	ldr.w	ip, [sp, #40]	; 0x28
 80014ca:	ea4f 005c 	mov.w	r0, ip, lsr #1
 80014ce:	461e      	mov	r6, r3
 80014d0:	0040      	lsls	r0, r0, #1
 80014d2:	ea5f 03dc 	movs.w	r3, ip, lsr #3
 80014d6:	460c      	mov	r4, r1
 80014d8:	4615      	mov	r5, r2
 80014da:	eb06 0e80 	add.w	lr, r6, r0, lsl #2
 80014de:	ed9f 0a50 	vldr	s0, [pc, #320]	; 8001620 <.text_7>
 80014e2:	d053      	beq.n	800158c <ai_dict4_dot_array_f32+0xd0>
 80014e4:	ed96 8a00 	vldr	s16, [r6]
 80014e8:	ed96 7a01 	vldr	s14, [r6, #4]
 80014ec:	ed96 6a02 	vldr	s12, [r6, #8]
 80014f0:	ed96 5a03 	vldr	s10, [r6, #12]
 80014f4:	7820      	ldrb	r0, [r4, #0]
 80014f6:	7861      	ldrb	r1, [r4, #1]
 80014f8:	78a2      	ldrb	r2, [r4, #2]
 80014fa:	78e7      	ldrb	r7, [r4, #3]
 80014fc:	ed96 4a04 	vldr	s8, [r6, #16]
 8001500:	ed96 3a05 	vldr	s6, [r6, #20]
 8001504:	ed96 2a06 	vldr	s4, [r6, #24]
 8001508:	ed96 1a07 	vldr	s2, [r6, #28]
 800150c:	f007 090f 	and.w	r9, r7, #15
 8001510:	093f      	lsrs	r7, r7, #4
 8001512:	eb05 0787 	add.w	r7, r5, r7, lsl #2
 8001516:	eb05 0a89 	add.w	sl, r5, r9, lsl #2
 800151a:	edd7 1a00 	vldr	s3, [r7]
 800151e:	edda 0a00 	vldr	s1, [sl]
 8001522:	f002 070f 	and.w	r7, r2, #15
 8001526:	0912      	lsrs	r2, r2, #4
 8001528:	eb05 0282 	add.w	r2, r5, r2, lsl #2
 800152c:	eb05 0787 	add.w	r7, r5, r7, lsl #2
 8001530:	edd2 3a00 	vldr	s7, [r2]
 8001534:	edd7 2a00 	vldr	s5, [r7]
 8001538:	f001 020f 	and.w	r2, r1, #15
 800153c:	0909      	lsrs	r1, r1, #4
 800153e:	eb05 0181 	add.w	r1, r5, r1, lsl #2
 8001542:	eb05 0782 	add.w	r7, r5, r2, lsl #2
 8001546:	edd1 5a00 	vldr	s11, [r1]
 800154a:	edd7 4a00 	vldr	s9, [r7]
 800154e:	f000 010f 	and.w	r1, r0, #15
 8001552:	0900      	lsrs	r0, r0, #4
 8001554:	eb05 0080 	add.w	r0, r5, r0, lsl #2
 8001558:	eb05 0281 	add.w	r2, r5, r1, lsl #2
 800155c:	edd0 7a00 	vldr	s15, [r0]
 8001560:	edd2 6a00 	vldr	s13, [r2]
 8001564:	ee07 0a88 	vmla.f32	s0, s15, s16
 8001568:	ee06 0a87 	vmla.f32	s0, s13, s14
 800156c:	ee05 0a86 	vmla.f32	s0, s11, s12
 8001570:	ee04 0a85 	vmla.f32	s0, s9, s10
 8001574:	ee03 0a84 	vmla.f32	s0, s7, s8
 8001578:	1d24      	adds	r4, r4, #4
 800157a:	ee02 0a83 	vmla.f32	s0, s5, s6
 800157e:	3620      	adds	r6, #32
 8001580:	ee01 0a82 	vmla.f32	s0, s3, s4
 8001584:	1e5b      	subs	r3, r3, #1
 8001586:	ee00 0a81 	vmla.f32	s0, s1, s2
 800158a:	d1ab      	bne.n	80014e4 <ai_dict4_dot_array_f32+0x28>
 800158c:	4576      	cmp	r6, lr
 800158e:	d22f      	bcs.n	80015f0 <ai_dict4_dot_array_f32+0x134>
 8001590:	f814 0b01 	ldrb.w	r0, [r4], #1
 8001594:	edd6 1a00 	vldr	s3, [r6]
 8001598:	edd6 0a01 	vldr	s1, [r6, #4]
 800159c:	f000 010f 	and.w	r1, r0, #15
 80015a0:	0900      	lsrs	r0, r0, #4
 80015a2:	eb05 0080 	add.w	r0, r5, r0, lsl #2
 80015a6:	eb05 0281 	add.w	r2, r5, r1, lsl #2
 80015aa:	ed90 2a00 	vldr	s4, [r0]
 80015ae:	ed92 1a00 	vldr	s2, [r2]
 80015b2:	3608      	adds	r6, #8
 80015b4:	ee02 0a21 	vmla.f32	s0, s4, s3
 80015b8:	4576      	cmp	r6, lr
 80015ba:	ee01 0a20 	vmla.f32	s0, s2, s1
 80015be:	d217      	bcs.n	80015f0 <ai_dict4_dot_array_f32+0x134>
 80015c0:	f814 0b01 	ldrb.w	r0, [r4], #1
 80015c4:	ed96 1a00 	vldr	s2, [r6]
 80015c8:	ed96 2a01 	vldr	s4, [r6, #4]
 80015cc:	f000 010f 	and.w	r1, r0, #15
 80015d0:	0900      	lsrs	r0, r0, #4
 80015d2:	eb05 0080 	add.w	r0, r5, r0, lsl #2
 80015d6:	eb05 0281 	add.w	r2, r5, r1, lsl #2
 80015da:	edd0 1a00 	vldr	s3, [r0]
 80015de:	edd2 0a00 	vldr	s1, [r2]
 80015e2:	3608      	adds	r6, #8
 80015e4:	ee01 0a81 	vmla.f32	s0, s3, s2
 80015e8:	4576      	cmp	r6, lr
 80015ea:	ee00 0a82 	vmla.f32	s0, s1, s4
 80015ee:	d3cf      	bcc.n	8001590 <ai_dict4_dot_array_f32+0xd4>
 80015f0:	ea5f 70cc 	movs.w	r0, ip, lsl #31
 80015f4:	d509      	bpl.n	800160a <ai_dict4_dot_array_f32+0x14e>
 80015f6:	7821      	ldrb	r1, [r4, #0]
 80015f8:	ed96 1a00 	vldr	s2, [r6]
 80015fc:	0909      	lsrs	r1, r1, #4
 80015fe:	eb05 0081 	add.w	r0, r5, r1, lsl #2
 8001602:	edd0 0a00 	vldr	s1, [r0]
 8001606:	ee00 0a81 	vmla.f32	s0, s1, s2
 800160a:	edd8 1a00 	vldr	s3, [r8]
 800160e:	ee31 0a80 	vadd.f32	s0, s3, s0
 8001612:	ed88 0a00 	vstr	s0, [r8]
 8001616:	ecbd 8b02 	vpop	{d8}
 800161a:	e8bd 87f0 	ldmia.w	sp!, {r4, r5, r6, r7, r8, r9, sl, pc}
	...

08001620 <.text_7>:
 8001620:	00000000 	.word	0x00000000

08001624 <ai_dict_decompress_f32>:
 8001624:	b4f0      	push	{r4, r5, r6, r7}
 8001626:	4604      	mov	r4, r0
 8001628:	9805      	ldr	r0, [sp, #20]
 800162a:	9e04      	ldr	r6, [sp, #16]
 800162c:	2b04      	cmp	r3, #4
 800162e:	eb04 0580 	add.w	r5, r4, r0, lsl #2
 8001632:	d003      	beq.n	800163c <ai_dict_decompress_f32+0x18>
 8001634:	2b08      	cmp	r3, #8
 8001636:	d03e      	beq.n	80016b6 <ai_dict_decompress_f32+0x92>
 8001638:	bcf0      	pop	{r4, r5, r6, r7}
 800163a:	4770      	bx	lr
 800163c:	42ac      	cmp	r4, r5
 800163e:	d259      	bcs.n	80016f4 <ai_dict_decompress_f32+0xd0>
 8001640:	0870      	lsrs	r0, r6, #1
 8001642:	d02e      	beq.n	80016a2 <ai_dict_decompress_f32+0x7e>
 8001644:	07c3      	lsls	r3, r0, #31
 8001646:	d50c      	bpl.n	8001662 <ai_dict_decompress_f32+0x3e>
 8001648:	780f      	ldrb	r7, [r1, #0]
 800164a:	093f      	lsrs	r7, r7, #4
 800164c:	f852 3027 	ldr.w	r3, [r2, r7, lsl #2]
 8001650:	6023      	str	r3, [r4, #0]
 8001652:	f811 7b01 	ldrb.w	r7, [r1], #1
 8001656:	f007 070f 	and.w	r7, r7, #15
 800165a:	f852 3027 	ldr.w	r3, [r2, r7, lsl #2]
 800165e:	6063      	str	r3, [r4, #4]
 8001660:	3408      	adds	r4, #8
 8001662:	0840      	lsrs	r0, r0, #1
 8001664:	d01d      	beq.n	80016a2 <ai_dict_decompress_f32+0x7e>
 8001666:	780b      	ldrb	r3, [r1, #0]
 8001668:	091b      	lsrs	r3, r3, #4
 800166a:	f852 7023 	ldr.w	r7, [r2, r3, lsl #2]
 800166e:	6027      	str	r7, [r4, #0]
 8001670:	f811 3b01 	ldrb.w	r3, [r1], #1
 8001674:	f003 030f 	and.w	r3, r3, #15
 8001678:	f852 7023 	ldr.w	r7, [r2, r3, lsl #2]
 800167c:	6067      	str	r7, [r4, #4]
 800167e:	f104 0308 	add.w	r3, r4, #8
 8001682:	780c      	ldrb	r4, [r1, #0]
 8001684:	0924      	lsrs	r4, r4, #4
 8001686:	f852 7024 	ldr.w	r7, [r2, r4, lsl #2]
 800168a:	601f      	str	r7, [r3, #0]
 800168c:	1e40      	subs	r0, r0, #1
 800168e:	f811 4b01 	ldrb.w	r4, [r1], #1
 8001692:	f004 040f 	and.w	r4, r4, #15
 8001696:	f852 7024 	ldr.w	r7, [r2, r4, lsl #2]
 800169a:	605f      	str	r7, [r3, #4]
 800169c:	f103 0408 	add.w	r4, r3, #8
 80016a0:	d1e1      	bne.n	8001666 <ai_dict_decompress_f32+0x42>
 80016a2:	07f0      	lsls	r0, r6, #31
 80016a4:	d5ca      	bpl.n	800163c <ai_dict_decompress_f32+0x18>
 80016a6:	f811 3b01 	ldrb.w	r3, [r1], #1
 80016aa:	091b      	lsrs	r3, r3, #4
 80016ac:	f852 0023 	ldr.w	r0, [r2, r3, lsl #2]
 80016b0:	f844 0b04 	str.w	r0, [r4], #4
 80016b4:	e7c2      	b.n	800163c <ai_dict_decompress_f32+0x18>
 80016b6:	42ac      	cmp	r4, r5
 80016b8:	d21c      	bcs.n	80016f4 <ai_dict_decompress_f32+0xd0>
 80016ba:	7808      	ldrb	r0, [r1, #0]
 80016bc:	f852 0020 	ldr.w	r0, [r2, r0, lsl #2]
 80016c0:	6020      	str	r0, [r4, #0]
 80016c2:	1d20      	adds	r0, r4, #4
 80016c4:	42a8      	cmp	r0, r5
 80016c6:	bf3f      	itttt	cc
 80016c8:	784c      	ldrbcc	r4, [r1, #1]
 80016ca:	f852 3024 	ldrcc.w	r3, [r2, r4, lsl #2]
 80016ce:	f840 3b04 	strcc.w	r3, [r0], #4
 80016d2:	42a8      	cmpcc	r0, r5
 80016d4:	d20e      	bcs.n	80016f4 <ai_dict_decompress_f32+0xd0>
 80016d6:	788b      	ldrb	r3, [r1, #2]
 80016d8:	f852 3023 	ldr.w	r3, [r2, r3, lsl #2]
 80016dc:	f840 3b04 	str.w	r3, [r0], #4
 80016e0:	42a8      	cmp	r0, r5
 80016e2:	d207      	bcs.n	80016f4 <ai_dict_decompress_f32+0xd0>
 80016e4:	78cc      	ldrb	r4, [r1, #3]
 80016e6:	f852 3024 	ldr.w	r3, [r2, r4, lsl #2]
 80016ea:	1d09      	adds	r1, r1, #4
 80016ec:	1d04      	adds	r4, r0, #4
 80016ee:	42ac      	cmp	r4, r5
 80016f0:	6003      	str	r3, [r0, #0]
 80016f2:	d3e2      	bcc.n	80016ba <ai_dict_decompress_f32+0x96>
 80016f4:	bcf0      	pop	{r4, r5, r6, r7}
 80016f6:	4770      	bx	lr

080016f8 <forward_conv2d>:
 80016f8:	e92d 4ff0 	stmdb	sp!, {r4, r5, r6, r7, r8, r9, sl, fp, lr}
 80016fc:	4605      	mov	r5, r0
 80016fe:	b0a9      	sub	sp, #164	; 0xa4
 8001700:	696b      	ldr	r3, [r5, #20]
 8001702:	8819      	ldrh	r1, [r3, #0]
 8001704:	2900      	cmp	r1, #0
 8001706:	bf1a      	itte	ne
 8001708:	6858      	ldrne	r0, [r3, #4]
 800170a:	1d00      	addne	r0, r0, #4
 800170c:	2004      	moveq	r0, #4
 800170e:	6800      	ldr	r0, [r0, #0]
 8001710:	2800      	cmp	r0, #0
 8001712:	bf14      	ite	ne
 8001714:	6802      	ldrne	r2, [r0, #0]
 8001716:	2200      	moveq	r2, #0
 8001718:	2901      	cmp	r1, #1
 800171a:	bfc6      	itte	gt
 800171c:	6858      	ldrgt	r0, [r3, #4]
 800171e:	3010      	addgt	r0, #16
 8001720:	2004      	movle	r0, #4
 8001722:	6800      	ldr	r0, [r0, #0]
 8001724:	2800      	cmp	r0, #0
 8001726:	bf14      	ite	ne
 8001728:	f8d0 a000 	ldrne.w	sl, [r0]
 800172c:	f04f 0a00 	moveq.w	sl, #0
 8001730:	2902      	cmp	r1, #2
 8001732:	bfc6      	itte	gt
 8001734:	6858      	ldrgt	r0, [r3, #4]
 8001736:	f100 041c 	addgt.w	r4, r0, #28
 800173a:	2404      	movle	r4, #4
 800173c:	6820      	ldr	r0, [r4, #0]
 800173e:	2800      	cmp	r0, #0
 8001740:	bf14      	ite	ne
 8001742:	6806      	ldrne	r6, [r0, #0]
 8001744:	2600      	moveq	r6, #0
 8001746:	2902      	cmp	r1, #2
 8001748:	dd0a      	ble.n	8001760 <forward_conv2d+0x68>
 800174a:	685b      	ldr	r3, [r3, #4]
 800174c:	f113 0118 	adds.w	r1, r3, #24
 8001750:	d006      	beq.n	8001760 <forward_conv2d+0x68>
 8001752:	8b19      	ldrh	r1, [r3, #24]
 8001754:	2901      	cmp	r1, #1
 8001756:	dd03      	ble.n	8001760 <forward_conv2d+0x68>
 8001758:	69d9      	ldr	r1, [r3, #28]
 800175a:	b109      	cbz	r1, 8001760 <forward_conv2d+0x68>
 800175c:	6849      	ldr	r1, [r1, #4]
 800175e:	e000      	b.n	8001762 <forward_conv2d+0x6a>
 8001760:	2100      	movs	r1, #0
 8001762:	b100      	cbz	r0, 8001766 <forward_conv2d+0x6e>
 8001764:	6880      	ldr	r0, [r0, #8]
 8001766:	68d7      	ldr	r7, [r2, #12]
 8001768:	687b      	ldr	r3, [r7, #4]
 800176a:	931b      	str	r3, [sp, #108]	; 0x6c
 800176c:	f8da 300c 	ldr.w	r3, [sl, #12]
 8001770:	685c      	ldr	r4, [r3, #4]
 8001772:	9404      	str	r4, [sp, #16]
 8001774:	68dc      	ldr	r4, [r3, #12]
 8001776:	689b      	ldr	r3, [r3, #8]
 8001778:	9314      	str	r3, [sp, #80]	; 0x50
 800177a:	68fb      	ldr	r3, [r7, #12]
 800177c:	931a      	str	r3, [sp, #104]	; 0x68
 800177e:	68bf      	ldr	r7, [r7, #8]
 8001780:	9720      	str	r7, [sp, #128]	; 0x80
 8001782:	6a6b      	ldr	r3, [r5, #36]	; 0x24
 8001784:	f8ad 3040 	strh.w	r3, [sp, #64]	; 0x40
 8001788:	8d2f      	ldrh	r7, [r5, #40]	; 0x28
 800178a:	971f      	str	r7, [sp, #124]	; 0x7c
 800178c:	6bab      	ldr	r3, [r5, #56]	; 0x38
 800178e:	681f      	ldr	r7, [r3, #0]
 8001790:	f8b3 8004 	ldrh.w	r8, [r3, #4]
 8001794:	6aeb      	ldr	r3, [r5, #44]	; 0x2c
 8001796:	9319      	str	r3, [sp, #100]	; 0x64
 8001798:	6b2b      	ldr	r3, [r5, #48]	; 0x30
 800179a:	9318      	str	r3, [sp, #96]	; 0x60
 800179c:	68f3      	ldr	r3, [r6, #12]
 800179e:	f8d3 e008 	ldr.w	lr, [r3, #8]
 80017a2:	f8cd e04c 	str.w	lr, [sp, #76]	; 0x4c
 80017a6:	685b      	ldr	r3, [r3, #4]
 80017a8:	9312      	str	r3, [sp, #72]	; 0x48
 80017aa:	69ab      	ldr	r3, [r5, #24]
 80017ac:	931e      	str	r3, [sp, #120]	; 0x78
 80017ae:	6992      	ldr	r2, [r2, #24]
 80017b0:	6893      	ldr	r3, [r2, #8]
 80017b2:	931d      	str	r3, [sp, #116]	; 0x74
 80017b4:	69b2      	ldr	r2, [r6, #24]
 80017b6:	f8d2 9008 	ldr.w	r9, [r2, #8]
 80017ba:	b119      	cbz	r1, 80017c4 <forward_conv2d+0xcc>
 80017bc:	698a      	ldr	r2, [r1, #24]
 80017be:	6893      	ldr	r3, [r2, #8]
 80017c0:	9317      	str	r3, [sp, #92]	; 0x5c
 80017c2:	e001      	b.n	80017c8 <forward_conv2d+0xd0>
 80017c4:	2200      	movs	r2, #0
 80017c6:	9217      	str	r2, [sp, #92]	; 0x5c
 80017c8:	f8da 1018 	ldr.w	r1, [sl, #24]
 80017cc:	688a      	ldr	r2, [r1, #8]
 80017ce:	9203      	str	r2, [sp, #12]
 80017d0:	69e9      	ldr	r1, [r5, #28]
 80017d2:	b118      	cbz	r0, 80017dc <forward_conv2d+0xe4>
 80017d4:	6981      	ldr	r1, [r0, #24]
 80017d6:	688a      	ldr	r2, [r1, #8]
 80017d8:	9215      	str	r2, [sp, #84]	; 0x54
 80017da:	e005      	b.n	80017e8 <forward_conv2d+0xf0>
 80017dc:	b111      	cbz	r1, 80017e4 <forward_conv2d+0xec>
 80017de:	688a      	ldr	r2, [r1, #8]
 80017e0:	9215      	str	r2, [sp, #84]	; 0x54
 80017e2:	e001      	b.n	80017e8 <forward_conv2d+0xf0>
 80017e4:	2300      	movs	r3, #0
 80017e6:	9315      	str	r3, [sp, #84]	; 0x54
 80017e8:	9915      	ldr	r1, [sp, #84]	; 0x54
 80017ea:	9102      	str	r1, [sp, #8]
 80017ec:	b920      	cbnz	r0, 80017f8 <forward_conv2d+0x100>
 80017ee:	2100      	movs	r1, #0
 80017f0:	2201      	movs	r2, #1
 80017f2:	9124      	str	r1, [sp, #144]	; 0x90
 80017f4:	9223      	str	r2, [sp, #140]	; 0x8c
 80017f6:	e008      	b.n	800180a <forward_conv2d+0x112>
 80017f8:	6941      	ldr	r1, [r0, #20]
 80017fa:	688a      	ldr	r2, [r1, #8]
 80017fc:	9224      	str	r2, [sp, #144]	; 0x90
 80017fe:	6980      	ldr	r0, [r0, #24]
 8001800:	6841      	ldr	r1, [r0, #4]
 8001802:	6800      	ldr	r0, [r0, #0]
 8001804:	f004 fb3e 	bl	8005e84 <ai_array_get_byte_size>
 8001808:	9023      	str	r0, [sp, #140]	; 0x8c
 800180a:	aa18      	add	r2, sp, #96	; 0x60
 800180c:	6a28      	ldr	r0, [r5, #32]
 800180e:	2800      	cmp	r0, #0
 8001810:	bf12      	itee	ne
 8001812:	9022      	strne	r0, [sp, #136]	; 0x88
 8001814:	f8df 1d28 	ldreq.w	r1, [pc, #3368]	; 8002540 <.text_15>
 8001818:	9122      	streq	r1, [sp, #136]	; 0x88
 800181a:	9913      	ldr	r1, [sp, #76]	; 0x4c
 800181c:	8813      	ldrh	r3, [r2, #0]
 800181e:	1e48      	subs	r0, r1, #1
 8001820:	1e5b      	subs	r3, r3, #1
 8001822:	aa19      	add	r2, sp, #100	; 0x64
 8001824:	fb03 1100 	mla	r1, r3, r0, r1
 8001828:	9116      	str	r1, [sp, #88]	; 0x58
 800182a:	9812      	ldr	r0, [sp, #72]	; 0x48
 800182c:	8813      	ldrh	r3, [r2, #0]
 800182e:	1e41      	subs	r1, r0, #1
 8001830:	1e5b      	subs	r3, r3, #1
 8001832:	fb03 0001 	mla	r0, r3, r1, r0
 8001836:	901c      	str	r0, [sp, #112]	; 0x70
 8001838:	2200      	movs	r2, #0
 800183a:	69b6      	ldr	r6, [r6, #24]
 800183c:	6831      	ldr	r1, [r6, #0]
 800183e:	11cb      	asrs	r3, r1, #7
 8001840:	ea4f 5c61 	mov.w	ip, r1, asr #21
 8001844:	1449      	asrs	r1, r1, #17
 8001846:	f001 010f 	and.w	r1, r1, #15
 800184a:	2000      	movs	r0, #0
 800184c:	f003 037f 	and.w	r3, r3, #127	; 0x7f
 8001850:	f00c 0c03 	and.w	ip, ip, #3
 8001854:	2904      	cmp	r1, #4
 8001856:	4683      	mov	fp, r0
 8001858:	fa23 f30c 	lsr.w	r3, r3, ip
 800185c:	bf14      	ite	ne
 800185e:	2908      	cmpne	r1, #8
 8001860:	68f2      	ldreq	r2, [r6, #12]
 8001862:	b1da      	cbz	r2, 800189c <forward_conv2d+0x1a4>
 8001864:	6969      	ldr	r1, [r5, #20]
 8001866:	880d      	ldrh	r5, [r1, #0]
 8001868:	2d04      	cmp	r5, #4
 800186a:	bfa6      	itte	ge
 800186c:	6849      	ldrge	r1, [r1, #4]
 800186e:	3128      	addge	r1, #40	; 0x28
 8001870:	2104      	movlt	r1, #4
 8001872:	6809      	ldr	r1, [r1, #0]
 8001874:	2900      	cmp	r1, #0
 8001876:	bf1f      	itttt	ne
 8001878:	6808      	ldrne	r0, [r1, #0]
 800187a:	2800      	cmpne	r0, #0
 800187c:	6981      	ldrne	r1, [r0, #24]
 800187e:	f8d1 b008 	ldrne.w	fp, [r1, #8]
 8001882:	6980      	ldr	r0, [r0, #24]
 8001884:	6841      	ldr	r1, [r0, #4]
 8001886:	981b      	ldr	r0, [sp, #108]	; 0x6c
 8001888:	9101      	str	r1, [sp, #4]
 800188a:	9000      	str	r0, [sp, #0]
 800188c:	4658      	mov	r0, fp
 800188e:	68b1      	ldr	r1, [r6, #8]
 8001890:	f7ff fec8 	bl	8001624 <ai_dict_decompress_f32>
 8001894:	f1bb 0f00 	cmp.w	fp, #0
 8001898:	bf18      	it	ne
 800189a:	46d9      	movne	r9, fp
 800189c:	b2bf      	uxth	r7, r7
 800189e:	427f      	negs	r7, r7
 80018a0:	2c00      	cmp	r4, #0
 80018a2:	d073      	beq.n	800198c <forward_conv2d+0x294>
 80018a4:	4622      	mov	r2, r4
 80018a6:	f1c8 0800 	rsb	r8, r8, #0
 80018aa:	9c04      	ldr	r4, [sp, #16]
 80018ac:	f8dd b00c 	ldr.w	fp, [sp, #12]
 80018b0:	9e02      	ldr	r6, [sp, #8]
 80018b2:	f8cd 8098 	str.w	r8, [sp, #152]	; 0x98
 80018b6:	f8cd 909c 	str.w	r9, [sp, #156]	; 0x9c
 80018ba:	9711      	str	r7, [sp, #68]	; 0x44
 80018bc:	9221      	str	r2, [sp, #132]	; 0x84
 80018be:	9826      	ldr	r0, [sp, #152]	; 0x98
 80018c0:	991a      	ldr	r1, [sp, #104]	; 0x68
 80018c2:	9a11      	ldr	r2, [sp, #68]	; 0x44
 80018c4:	9b16      	ldr	r3, [sp, #88]	; 0x58
 80018c6:	9025      	str	r0, [sp, #148]	; 0x94
 80018c8:	9811      	ldr	r0, [sp, #68]	; 0x44
 80018ca:	4240      	negs	r0, r0
 80018cc:	bfd8      	it	le
 80018ce:	2000      	movle	r0, #0
 80018d0:	1a89      	subs	r1, r1, r2
 80018d2:	4299      	cmp	r1, r3
 80018d4:	bf3d      	ittte	cc
 80018d6:	9a1a      	ldrcc	r2, [sp, #104]	; 0x68
 80018d8:	9911      	ldrcc	r1, [sp, #68]	; 0x44
 80018da:	1a51      	subcc	r1, r2, r1
 80018dc:	4619      	movcs	r1, r3
 80018de:	910a      	str	r1, [sp, #40]	; 0x28
 80018e0:	9009      	str	r0, [sp, #36]	; 0x24
 80018e2:	9402      	str	r4, [sp, #8]
 80018e4:	981e      	ldr	r0, [sp, #120]	; 0x78
 80018e6:	f8bd 1040 	ldrh.w	r1, [sp, #64]	; 0x40
 80018ea:	9a18      	ldr	r2, [sp, #96]	; 0x60
 80018ec:	9008      	str	r0, [sp, #32]
 80018ee:	9107      	str	r1, [sp, #28]
 80018f0:	b212      	sxth	r2, r2
 80018f2:	9813      	ldr	r0, [sp, #76]	; 0x4c
 80018f4:	9912      	ldr	r1, [sp, #72]	; 0x48
 80018f6:	9b19      	ldr	r3, [sp, #100]	; 0x64
 80018f8:	920f      	str	r2, [sp, #60]	; 0x3c
 80018fa:	9006      	str	r0, [sp, #24]
 80018fc:	9105      	str	r1, [sp, #20]
 80018fe:	b21b      	sxth	r3, r3
 8001900:	9a1c      	ldr	r2, [sp, #112]	; 0x70
 8001902:	9814      	ldr	r0, [sp, #80]	; 0x50
 8001904:	9920      	ldr	r1, [sp, #128]	; 0x80
 8001906:	930e      	str	r3, [sp, #56]	; 0x38
 8001908:	920d      	str	r2, [sp, #52]	; 0x34
 800190a:	9004      	str	r0, [sp, #16]
 800190c:	9103      	str	r1, [sp, #12]
 800190e:	9b11      	ldr	r3, [sp, #68]	; 0x44
 8001910:	9a25      	ldr	r2, [sp, #148]	; 0x94
 8001912:	981b      	ldr	r0, [sp, #108]	; 0x6c
 8001914:	9917      	ldr	r1, [sp, #92]	; 0x5c
 8001916:	930c      	str	r3, [sp, #48]	; 0x30
 8001918:	920b      	str	r2, [sp, #44]	; 0x2c
 800191a:	9001      	str	r0, [sp, #4]
 800191c:	9100      	str	r1, [sp, #0]
 800191e:	9b27      	ldr	r3, [sp, #156]	; 0x9c
 8001920:	9a1d      	ldr	r2, [sp, #116]	; 0x74
 8001922:	4659      	mov	r1, fp
 8001924:	2000      	movs	r0, #0
 8001926:	f7ff fa43 	bl	8000db0 <ai_conv2d_stripe_f32>
 800192a:	9814      	ldr	r0, [sp, #80]	; 0x50
 800192c:	b310      	cbz	r0, 8001974 <forward_conv2d+0x27c>
 800192e:	f8cd a000 	str.w	sl, [sp]
 8001932:	9d15      	ldr	r5, [sp, #84]	; 0x54
 8001934:	9f24      	ldr	r7, [sp, #144]	; 0x90
 8001936:	f8dd 808c 	ldr.w	r8, [sp, #140]	; 0x8c
 800193a:	f8dd 9088 	ldr.w	r9, [sp, #136]	; 0x88
 800193e:	4682      	mov	sl, r0
 8001940:	9800      	ldr	r0, [sp, #0]
 8001942:	6981      	ldr	r1, [r0, #24]
 8001944:	f8c1 b008 	str.w	fp, [r1, #8]
 8001948:	462b      	mov	r3, r5
 800194a:	4622      	mov	r2, r4
 800194c:	4608      	mov	r0, r1
 800194e:	47c8      	blx	r9
 8001950:	443d      	add	r5, r7
 8001952:	1ba8      	subs	r0, r5, r6
 8001954:	4540      	cmp	r0, r8
 8001956:	bfa8      	it	ge
 8001958:	4635      	movge	r5, r6
 800195a:	f1ba 0a01 	subs.w	sl, sl, #1
 800195e:	eb0b 0b84 	add.w	fp, fp, r4, lsl #2
 8001962:	d1ed      	bne.n	8001940 <forward_conv2d+0x248>
 8001964:	f8dd a000 	ldr.w	sl, [sp]
 8001968:	9515      	str	r5, [sp, #84]	; 0x54
 800196a:	9724      	str	r7, [sp, #144]	; 0x90
 800196c:	f8cd 808c 	str.w	r8, [sp, #140]	; 0x8c
 8001970:	f8cd 9088 	str.w	r9, [sp, #136]	; 0x88
 8001974:	f8da 0018 	ldr.w	r0, [sl, #24]
 8001978:	68c1      	ldr	r1, [r0, #12]
 800197a:	6081      	str	r1, [r0, #8]
 800197c:	9811      	ldr	r0, [sp, #68]	; 0x44
 800197e:	991f      	ldr	r1, [sp, #124]	; 0x7c
 8001980:	1808      	adds	r0, r1, r0
 8001982:	9011      	str	r0, [sp, #68]	; 0x44
 8001984:	9821      	ldr	r0, [sp, #132]	; 0x84
 8001986:	1e40      	subs	r0, r0, #1
 8001988:	9021      	str	r0, [sp, #132]	; 0x84
 800198a:	d198      	bne.n	80018be <forward_conv2d+0x1c6>
 800198c:	b029      	add	sp, #164	; 0xa4
 800198e:	e8bd 8ff0 	ldmia.w	sp!, {r4, r5, r6, r7, r8, r9, sl, fp, pc}
	...

08001994 <forward_conv2d_nl_pool>:
 8001994:	e92d 4ff0 	stmdb	sp!, {r4, r5, r6, r7, r8, r9, sl, fp, lr}
 8001998:	4604      	mov	r4, r0
 800199a:	b0b9      	sub	sp, #228	; 0xe4
 800199c:	6963      	ldr	r3, [r4, #20]
 800199e:	8819      	ldrh	r1, [r3, #0]
 80019a0:	2900      	cmp	r1, #0
 80019a2:	bf1a      	itte	ne
 80019a4:	6858      	ldrne	r0, [r3, #4]
 80019a6:	1d00      	addne	r0, r0, #4
 80019a8:	2004      	moveq	r0, #4
 80019aa:	6800      	ldr	r0, [r0, #0]
 80019ac:	2800      	cmp	r0, #0
 80019ae:	bf14      	ite	ne
 80019b0:	6802      	ldrne	r2, [r0, #0]
 80019b2:	2200      	moveq	r2, #0
 80019b4:	2901      	cmp	r1, #1
 80019b6:	bfc6      	itte	gt
 80019b8:	6858      	ldrgt	r0, [r3, #4]
 80019ba:	3010      	addgt	r0, #16
 80019bc:	2004      	movle	r0, #4
 80019be:	6800      	ldr	r0, [r0, #0]
 80019c0:	2800      	cmp	r0, #0
 80019c2:	bf14      	ite	ne
 80019c4:	f8d0 9000 	ldrne.w	r9, [r0]
 80019c8:	f04f 0900 	moveq.w	r9, #0
 80019cc:	2902      	cmp	r1, #2
 80019ce:	bfc6      	itte	gt
 80019d0:	6858      	ldrgt	r0, [r3, #4]
 80019d2:	f100 071c 	addgt.w	r7, r0, #28
 80019d6:	2704      	movle	r7, #4
 80019d8:	6838      	ldr	r0, [r7, #0]
 80019da:	2800      	cmp	r0, #0
 80019dc:	bf14      	ite	ne
 80019de:	6806      	ldrne	r6, [r0, #0]
 80019e0:	2600      	moveq	r6, #0
 80019e2:	2902      	cmp	r1, #2
 80019e4:	dd0a      	ble.n	80019fc <forward_conv2d_nl_pool+0x68>
 80019e6:	685b      	ldr	r3, [r3, #4]
 80019e8:	f113 0118 	adds.w	r1, r3, #24
 80019ec:	d006      	beq.n	80019fc <forward_conv2d_nl_pool+0x68>
 80019ee:	8b19      	ldrh	r1, [r3, #24]
 80019f0:	2901      	cmp	r1, #1
 80019f2:	dd03      	ble.n	80019fc <forward_conv2d_nl_pool+0x68>
 80019f4:	69d9      	ldr	r1, [r3, #28]
 80019f6:	b109      	cbz	r1, 80019fc <forward_conv2d_nl_pool+0x68>
 80019f8:	6849      	ldr	r1, [r1, #4]
 80019fa:	e000      	b.n	80019fe <forward_conv2d_nl_pool+0x6a>
 80019fc:	2100      	movs	r1, #0
 80019fe:	b100      	cbz	r0, 8001a02 <forward_conv2d_nl_pool+0x6e>
 8001a00:	6880      	ldr	r0, [r0, #8]
 8001a02:	68d7      	ldr	r7, [r2, #12]
 8001a04:	687b      	ldr	r3, [r7, #4]
 8001a06:	9323      	str	r3, [sp, #140]	; 0x8c
 8001a08:	f8d9 500c 	ldr.w	r5, [r9, #12]
 8001a0c:	686b      	ldr	r3, [r5, #4]
 8001a0e:	9310      	str	r3, [sp, #64]	; 0x40
 8001a10:	68eb      	ldr	r3, [r5, #12]
 8001a12:	9322      	str	r3, [sp, #136]	; 0x88
 8001a14:	68ab      	ldr	r3, [r5, #8]
 8001a16:	9321      	str	r3, [sp, #132]	; 0x84
 8001a18:	68fb      	ldr	r3, [r7, #12]
 8001a1a:	931b      	str	r3, [sp, #108]	; 0x6c
 8001a1c:	68bf      	ldr	r7, [r7, #8]
 8001a1e:	972d      	str	r7, [sp, #180]	; 0xb4
 8001a20:	6a63      	ldr	r3, [r4, #36]	; 0x24
 8001a22:	f8ad 304c 	strh.w	r3, [sp, #76]	; 0x4c
 8001a26:	8d27      	ldrh	r7, [r4, #40]	; 0x28
 8001a28:	9720      	str	r7, [sp, #128]	; 0x80
 8001a2a:	6ba3      	ldr	r3, [r4, #56]	; 0x38
 8001a2c:	881f      	ldrh	r7, [r3, #0]
 8001a2e:	f8b3 8004 	ldrh.w	r8, [r3, #4]
 8001a32:	689d      	ldr	r5, [r3, #8]
 8001a34:	69a3      	ldr	r3, [r4, #24]
 8001a36:	932c      	str	r3, [sp, #176]	; 0xb0
 8001a38:	6ae3      	ldr	r3, [r4, #44]	; 0x2c
 8001a3a:	931f      	str	r3, [sp, #124]	; 0x7c
 8001a3c:	6b23      	ldr	r3, [r4, #48]	; 0x30
 8001a3e:	931e      	str	r3, [sp, #120]	; 0x78
 8001a40:	68f3      	ldr	r3, [r6, #12]
 8001a42:	f8d3 e004 	ldr.w	lr, [r3, #4]
 8001a46:	f8cd e068 	str.w	lr, [sp, #104]	; 0x68
 8001a4a:	689b      	ldr	r3, [r3, #8]
 8001a4c:	9319      	str	r3, [sp, #100]	; 0x64
 8001a4e:	6be3      	ldr	r3, [r4, #60]	; 0x3c
 8001a50:	932b      	str	r3, [sp, #172]	; 0xac
 8001a52:	6c63      	ldr	r3, [r4, #68]	; 0x44
 8001a54:	932a      	str	r3, [sp, #168]	; 0xa8
 8001a56:	6ca3      	ldr	r3, [r4, #72]	; 0x48
 8001a58:	9311      	str	r3, [sp, #68]	; 0x44
 8001a5a:	6d23      	ldr	r3, [r4, #80]	; 0x50
 8001a5c:	f8d3 a000 	ldr.w	sl, [r3]
 8001a60:	685b      	ldr	r3, [r3, #4]
 8001a62:	9329      	str	r3, [sp, #164]	; 0xa4
 8001a64:	6992      	ldr	r2, [r2, #24]
 8001a66:	6893      	ldr	r3, [r2, #8]
 8001a68:	9328      	str	r3, [sp, #160]	; 0xa0
 8001a6a:	69b2      	ldr	r2, [r6, #24]
 8001a6c:	f8d2 b008 	ldr.w	fp, [r2, #8]
 8001a70:	b119      	cbz	r1, 8001a7a <forward_conv2d_nl_pool+0xe6>
 8001a72:	698a      	ldr	r2, [r1, #24]
 8001a74:	6893      	ldr	r3, [r2, #8]
 8001a76:	931d      	str	r3, [sp, #116]	; 0x74
 8001a78:	e001      	b.n	8001a7e <forward_conv2d_nl_pool+0xea>
 8001a7a:	2200      	movs	r2, #0
 8001a7c:	921d      	str	r2, [sp, #116]	; 0x74
 8001a7e:	69e1      	ldr	r1, [r4, #28]
 8001a80:	b118      	cbz	r0, 8001a8a <forward_conv2d_nl_pool+0xf6>
 8001a82:	6981      	ldr	r1, [r0, #24]
 8001a84:	688a      	ldr	r2, [r1, #8]
 8001a86:	921c      	str	r2, [sp, #112]	; 0x70
 8001a88:	e005      	b.n	8001a96 <forward_conv2d_nl_pool+0x102>
 8001a8a:	b111      	cbz	r1, 8001a92 <forward_conv2d_nl_pool+0xfe>
 8001a8c:	688a      	ldr	r2, [r1, #8]
 8001a8e:	921c      	str	r2, [sp, #112]	; 0x70
 8001a90:	e001      	b.n	8001a96 <forward_conv2d_nl_pool+0x102>
 8001a92:	2300      	movs	r3, #0
 8001a94:	931c      	str	r3, [sp, #112]	; 0x70
 8001a96:	991c      	ldr	r1, [sp, #112]	; 0x70
 8001a98:	9102      	str	r1, [sp, #8]
 8001a9a:	b920      	cbnz	r0, 8001aa6 <forward_conv2d_nl_pool+0x112>
 8001a9c:	2100      	movs	r1, #0
 8001a9e:	2201      	movs	r2, #1
 8001aa0:	9116      	str	r1, [sp, #88]	; 0x58
 8001aa2:	9215      	str	r2, [sp, #84]	; 0x54
 8001aa4:	e008      	b.n	8001ab8 <forward_conv2d_nl_pool+0x124>
 8001aa6:	6941      	ldr	r1, [r0, #20]
 8001aa8:	688a      	ldr	r2, [r1, #8]
 8001aaa:	9216      	str	r2, [sp, #88]	; 0x58
 8001aac:	6980      	ldr	r0, [r0, #24]
 8001aae:	6841      	ldr	r1, [r0, #4]
 8001ab0:	6800      	ldr	r0, [r0, #0]
 8001ab2:	f004 f9e7 	bl	8005e84 <ai_array_get_byte_size>
 8001ab6:	9015      	str	r0, [sp, #84]	; 0x54
 8001ab8:	aa1e      	add	r2, sp, #120	; 0x78
 8001aba:	6a20      	ldr	r0, [r4, #32]
 8001abc:	2800      	cmp	r0, #0
 8001abe:	bf12      	itee	ne
 8001ac0:	9030      	strne	r0, [sp, #192]	; 0xc0
 8001ac2:	f8df 1a7c 	ldreq.w	r1, [pc, #2684]	; 8002540 <.text_15>
 8001ac6:	9130      	streq	r1, [sp, #192]	; 0xc0
 8001ac8:	6d61      	ldr	r1, [r4, #84]	; 0x54
 8001aca:	9819      	ldr	r0, [sp, #100]	; 0x64
 8001acc:	8813      	ldrh	r3, [r2, #0]
 8001ace:	9127      	str	r1, [sp, #156]	; 0x9c
 8001ad0:	1e5b      	subs	r3, r3, #1
 8001ad2:	1e41      	subs	r1, r0, #1
 8001ad4:	aa1f      	add	r2, sp, #124	; 0x7c
 8001ad6:	fb03 0001 	mla	r0, r3, r1, r0
 8001ada:	9018      	str	r0, [sp, #96]	; 0x60
 8001adc:	991a      	ldr	r1, [sp, #104]	; 0x68
 8001ade:	8813      	ldrh	r3, [r2, #0]
 8001ae0:	1e48      	subs	r0, r1, #1
 8001ae2:	1e5b      	subs	r3, r3, #1
 8001ae4:	fb03 1100 	mla	r1, r3, r0, r1
 8001ae8:	9126      	str	r1, [sp, #152]	; 0x98
 8001aea:	6c21      	ldr	r1, [r4, #64]	; 0x40
 8001aec:	9a1b      	ldr	r2, [sp, #108]	; 0x6c
 8001aee:	9818      	ldr	r0, [sp, #96]	; 0x60
 8001af0:	9112      	str	r1, [sp, #72]	; 0x48
 8001af2:	1a12      	subs	r2, r2, r0
 8001af4:	18ba      	adds	r2, r7, r2
 8001af6:	9920      	ldr	r1, [sp, #128]	; 0x80
 8001af8:	fa12 f085 	uxtah	r0, r2, r5
 8001afc:	fbb0 f1f1 	udiv	r1, r0, r1
 8001b00:	1c49      	adds	r1, r1, #1
 8001b02:	9114      	str	r1, [sp, #80]	; 0x50
 8001b04:	2000      	movs	r0, #0
 8001b06:	69b6      	ldr	r6, [r6, #24]
 8001b08:	6831      	ldr	r1, [r6, #0]
 8001b0a:	2500      	movs	r5, #0
 8001b0c:	2200      	movs	r2, #0
 8001b0e:	11cb      	asrs	r3, r1, #7
 8001b10:	ea4f 5c61 	mov.w	ip, r1, asr #21
 8001b14:	1449      	asrs	r1, r1, #17
 8001b16:	f001 010f 	and.w	r1, r1, #15
 8001b1a:	f003 037f 	and.w	r3, r3, #127	; 0x7f
 8001b1e:	f00c 0c03 	and.w	ip, ip, #3
 8001b22:	2904      	cmp	r1, #4
 8001b24:	fa23 f30c 	lsr.w	r3, r3, ip
 8001b28:	bf14      	ite	ne
 8001b2a:	2908      	cmpne	r1, #8
 8001b2c:	68f2      	ldreq	r2, [r6, #12]
 8001b2e:	b1da      	cbz	r2, 8001b68 <forward_conv2d_nl_pool+0x1d4>
 8001b30:	6961      	ldr	r1, [r4, #20]
 8001b32:	f8b1 c000 	ldrh.w	ip, [r1]
 8001b36:	f1bc 0f04 	cmp.w	ip, #4
 8001b3a:	bfa6      	itte	ge
 8001b3c:	6849      	ldrge	r1, [r1, #4]
 8001b3e:	3128      	addge	r1, #40	; 0x28
 8001b40:	2104      	movlt	r1, #4
 8001b42:	6809      	ldr	r1, [r1, #0]
 8001b44:	2900      	cmp	r1, #0
 8001b46:	bf1f      	itttt	ne
 8001b48:	6848      	ldrne	r0, [r1, #4]
 8001b4a:	2800      	cmpne	r0, #0
 8001b4c:	6981      	ldrne	r1, [r0, #24]
 8001b4e:	688d      	ldrne	r5, [r1, #8]
 8001b50:	6980      	ldr	r0, [r0, #24]
 8001b52:	6841      	ldr	r1, [r0, #4]
 8001b54:	9823      	ldr	r0, [sp, #140]	; 0x8c
 8001b56:	9101      	str	r1, [sp, #4]
 8001b58:	9000      	str	r0, [sp, #0]
 8001b5a:	4628      	mov	r0, r5
 8001b5c:	68b1      	ldr	r1, [r6, #8]
 8001b5e:	f7ff fd61 	bl	8001624 <ai_dict_decompress_f32>
 8001b62:	b10d      	cbz	r5, 8001b68 <forward_conv2d_nl_pool+0x1d4>
 8001b64:	4628      	mov	r0, r5
 8001b66:	e000      	b.n	8001b6a <forward_conv2d_nl_pool+0x1d6>
 8001b68:	4658      	mov	r0, fp
 8001b6a:	6963      	ldr	r3, [r4, #20]
 8001b6c:	f8dd c040 	ldr.w	ip, [sp, #64]	; 0x40
 8001b70:	881c      	ldrh	r4, [r3, #0]
 8001b72:	f8d9 1018 	ldr.w	r1, [r9, #24]
 8001b76:	2600      	movs	r6, #0
 8001b78:	2c04      	cmp	r4, #4
 8001b7a:	bfa6      	itte	ge
 8001b7c:	685b      	ldrge	r3, [r3, #4]
 8001b7e:	3328      	addge	r3, #40	; 0x28
 8001b80:	2304      	movlt	r3, #4
 8001b82:	f10d 0e44 	add.w	lr, sp, #68	; 0x44
 8001b86:	681b      	ldr	r3, [r3, #0]
 8001b88:	2b00      	cmp	r3, #0
 8001b8a:	bf14      	ite	ne
 8001b8c:	681d      	ldrne	r5, [r3, #0]
 8001b8e:	2500      	moveq	r5, #0
 8001b90:	427f      	negs	r7, r7
 8001b92:	69ac      	ldr	r4, [r5, #24]
 8001b94:	68eb      	ldr	r3, [r5, #12]
 8001b96:	f8d4 b008 	ldr.w	fp, [r4, #8]
 8001b9a:	689b      	ldr	r3, [r3, #8]
 8001b9c:	9c11      	ldr	r4, [sp, #68]	; 0x44
 8001b9e:	435c      	muls	r4, r3
 8001ba0:	fb0c f404 	mul.w	r4, ip, r4
 8001ba4:	9437      	str	r4, [sp, #220]	; 0xdc
 8001ba6:	fa0f f28a 	sxth.w	r2, sl
 8001baa:	f9be 4000 	ldrsh.w	r4, [lr]
 8001bae:	f8dd c084 	ldr.w	ip, [sp, #132]	; 0x84
 8001bb2:	9436      	str	r4, [sp, #216]	; 0xd8
 8001bb4:	f10d 0e48 	add.w	lr, sp, #72	; 0x48
 8001bb8:	9c10      	ldr	r4, [sp, #64]	; 0x40
 8001bba:	fb0c f404 	mul.w	r4, ip, r4
 8001bbe:	9435      	str	r4, [sp, #212]	; 0xd4
 8001bc0:	f1c8 0800 	rsb	r8, r8, #0
 8001bc4:	f9be 4000 	ldrsh.w	r4, [lr]
 8001bc8:	9434      	str	r4, [sp, #208]	; 0xd0
 8001bca:	4691      	mov	r9, r2
 8001bcc:	9c10      	ldr	r4, [sp, #64]	; 0x40
 8001bce:	f8cd 80c8 	str.w	r8, [sp, #200]	; 0xc8
 8001bd2:	435c      	muls	r4, r3
 8001bd4:	9433      	str	r4, [sp, #204]	; 0xcc
 8001bd6:	9c22      	ldr	r4, [sp, #136]	; 0x88
 8001bd8:	2c00      	cmp	r4, #0
 8001bda:	f000 812e 	beq.w	8001e3a <forward_conv2d_nl_pool+0x4a6>
 8001bde:	f8dd a008 	ldr.w	sl, [sp, #8]
 8001be2:	9038      	str	r0, [sp, #224]	; 0xe0
 8001be4:	9125      	str	r1, [sp, #148]	; 0x94
 8001be6:	4614      	mov	r4, r2
 8001be8:	962f      	str	r6, [sp, #188]	; 0xbc
 8001bea:	962e      	str	r6, [sp, #184]	; 0xb8
 8001bec:	9324      	str	r3, [sp, #144]	; 0x90
 8001bee:	9717      	str	r7, [sp, #92]	; 0x5c
 8001bf0:	9814      	ldr	r0, [sp, #80]	; 0x50
 8001bf2:	2800      	cmp	r0, #0
 8001bf4:	dd6a      	ble.n	8001ccc <forward_conv2d_nl_pool+0x338>
 8001bf6:	9832      	ldr	r0, [sp, #200]	; 0xc8
 8001bf8:	991b      	ldr	r1, [sp, #108]	; 0x6c
 8001bfa:	9a17      	ldr	r2, [sp, #92]	; 0x5c
 8001bfc:	9b18      	ldr	r3, [sp, #96]	; 0x60
 8001bfe:	9031      	str	r0, [sp, #196]	; 0xc4
 8001c00:	9817      	ldr	r0, [sp, #92]	; 0x5c
 8001c02:	4240      	negs	r0, r0
 8001c04:	bfd8      	it	le
 8001c06:	2000      	movle	r0, #0
 8001c08:	1a89      	subs	r1, r1, r2
 8001c0a:	4299      	cmp	r1, r3
 8001c0c:	bf3d      	ittte	cc
 8001c0e:	9a1b      	ldrcc	r2, [sp, #108]	; 0x6c
 8001c10:	9917      	ldrcc	r1, [sp, #92]	; 0x5c
 8001c12:	1a51      	subcc	r1, r2, r1
 8001c14:	4619      	movcs	r1, r3
 8001c16:	9009      	str	r0, [sp, #36]	; 0x24
 8001c18:	910a      	str	r1, [sp, #40]	; 0x28
 8001c1a:	982c      	ldr	r0, [sp, #176]	; 0xb0
 8001c1c:	f8bd 104c 	ldrh.w	r1, [sp, #76]	; 0x4c
 8001c20:	9a1e      	ldr	r2, [sp, #120]	; 0x78
 8001c22:	9b1f      	ldr	r3, [sp, #124]	; 0x7c
 8001c24:	9008      	str	r0, [sp, #32]
 8001c26:	9107      	str	r1, [sp, #28]
 8001c28:	b212      	sxth	r2, r2
 8001c2a:	9819      	ldr	r0, [sp, #100]	; 0x64
 8001c2c:	991a      	ldr	r1, [sp, #104]	; 0x68
 8001c2e:	9006      	str	r0, [sp, #24]
 8001c30:	920f      	str	r2, [sp, #60]	; 0x3c
 8001c32:	9105      	str	r1, [sp, #20]
 8001c34:	b21b      	sxth	r3, r3
 8001c36:	9824      	ldr	r0, [sp, #144]	; 0x90
 8001c38:	9a26      	ldr	r2, [sp, #152]	; 0x98
 8001c3a:	992d      	ldr	r1, [sp, #180]	; 0xb4
 8001c3c:	9004      	str	r0, [sp, #16]
 8001c3e:	930e      	str	r3, [sp, #56]	; 0x38
 8001c40:	920d      	str	r2, [sp, #52]	; 0x34
 8001c42:	9103      	str	r1, [sp, #12]
 8001c44:	9810      	ldr	r0, [sp, #64]	; 0x40
 8001c46:	9b17      	ldr	r3, [sp, #92]	; 0x5c
 8001c48:	9a31      	ldr	r2, [sp, #196]	; 0xc4
 8001c4a:	9923      	ldr	r1, [sp, #140]	; 0x8c
 8001c4c:	9002      	str	r0, [sp, #8]
 8001c4e:	930c      	str	r3, [sp, #48]	; 0x30
 8001c50:	920b      	str	r2, [sp, #44]	; 0x2c
 8001c52:	9101      	str	r1, [sp, #4]
 8001c54:	4659      	mov	r1, fp
 8001c56:	981d      	ldr	r0, [sp, #116]	; 0x74
 8001c58:	9b38      	ldr	r3, [sp, #224]	; 0xe0
 8001c5a:	9a28      	ldr	r2, [sp, #160]	; 0xa0
 8001c5c:	9000      	str	r0, [sp, #0]
 8001c5e:	2000      	movs	r0, #0
 8001c60:	f7ff f8a6 	bl	8000db0 <ai_conv2d_stripe_f32>
 8001c64:	9824      	ldr	r0, [sp, #144]	; 0x90
 8001c66:	b350      	cbz	r0, 8001cbe <forward_conv2d_nl_pool+0x32a>
 8001c68:	f8cd a008 	str.w	sl, [sp, #8]
 8001c6c:	9e10      	ldr	r6, [sp, #64]	; 0x40
 8001c6e:	9f1c      	ldr	r7, [sp, #112]	; 0x70
 8001c70:	f8dd 80c0 	ldr.w	r8, [sp, #192]	; 0xc0
 8001c74:	4682      	mov	sl, r0
 8001c76:	69a9      	ldr	r1, [r5, #24]
 8001c78:	463b      	mov	r3, r7
 8001c7a:	f8c1 b008 	str.w	fp, [r1, #8]
 8001c7e:	4632      	mov	r2, r6
 8001c80:	4608      	mov	r0, r1
 8001c82:	47c0      	blx	r8
 8001c84:	9816      	ldr	r0, [sp, #88]	; 0x58
 8001c86:	9902      	ldr	r1, [sp, #8]
 8001c88:	4407      	add	r7, r0
 8001c8a:	9815      	ldr	r0, [sp, #84]	; 0x54
 8001c8c:	1a79      	subs	r1, r7, r1
 8001c8e:	4281      	cmp	r1, r0
 8001c90:	69a8      	ldr	r0, [r5, #24]
 8001c92:	6841      	ldr	r1, [r0, #4]
 8001c94:	68c0      	ldr	r0, [r0, #12]
 8001c96:	bfa8      	it	ge
 8001c98:	9f02      	ldrge	r7, [sp, #8]
 8001c9a:	eb0b 0b86 	add.w	fp, fp, r6, lsl #2
 8001c9e:	eb00 0281 	add.w	r2, r0, r1, lsl #2
 8001ca2:	4593      	cmp	fp, r2
 8001ca4:	d302      	bcc.n	8001cac <forward_conv2d_nl_pool+0x318>
 8001ca6:	0089      	lsls	r1, r1, #2
 8001ca8:	4249      	negs	r1, r1
 8001caa:	448b      	add	fp, r1
 8001cac:	f1ba 0a01 	subs.w	sl, sl, #1
 8001cb0:	d1e1      	bne.n	8001c76 <forward_conv2d_nl_pool+0x2e2>
 8001cb2:	f8dd a008 	ldr.w	sl, [sp, #8]
 8001cb6:	9610      	str	r6, [sp, #64]	; 0x40
 8001cb8:	971c      	str	r7, [sp, #112]	; 0x70
 8001cba:	f8cd 80c0 	str.w	r8, [sp, #192]	; 0xc0
 8001cbe:	69a8      	ldr	r0, [r5, #24]
 8001cc0:	68c1      	ldr	r1, [r0, #12]
 8001cc2:	6081      	str	r1, [r0, #8]
 8001cc4:	f109 0001 	add.w	r0, r9, #1
 8001cc8:	fa0f f980 	sxth.w	r9, r0
 8001ccc:	9814      	ldr	r0, [sp, #80]	; 0x50
 8001cce:	1e40      	subs	r0, r0, #1
 8001cd0:	9014      	str	r0, [sp, #80]	; 0x50
 8001cd2:	d56b      	bpl.n	8001dac <forward_conv2d_nl_pool+0x418>
 8001cd4:	9833      	ldr	r0, [sp, #204]	; 0xcc
 8001cd6:	fb00 f009 	mul.w	r0, r0, r9
 8001cda:	0080      	lsls	r0, r0, #2
 8001cdc:	4240      	negs	r0, r0
 8001cde:	eb0b 0200 	add.w	r2, fp, r0
 8001ce2:	69a8      	ldr	r0, [r5, #24]
 8001ce4:	68c3      	ldr	r3, [r0, #12]
 8001ce6:	429a      	cmp	r2, r3
 8001ce8:	bf3c      	itt	cc
 8001cea:	6847      	ldrcc	r7, [r0, #4]
 8001cec:	eb02 0287 	addcc.w	r2, r2, r7, lsl #2
 8001cf0:	4293      	cmp	r3, r2
 8001cf2:	4659      	mov	r1, fp
 8001cf4:	d236      	bcs.n	8001d64 <forward_conv2d_nl_pool+0x3d0>
 8001cf6:	9e34      	ldr	r6, [sp, #208]	; 0xd0
 8001cf8:	45b1      	cmp	r9, r6
 8001cfa:	d033      	beq.n	8001d64 <forward_conv2d_nl_pool+0x3d0>
 8001cfc:	6846      	ldr	r6, [r0, #4]
 8001cfe:	eb03 0386 	add.w	r3, r3, r6, lsl #2
 8001d02:	429a      	cmp	r2, r3
 8001d04:	f080 802e 	bcs.w	8001d64 <forward_conv2d_nl_pool+0x3d0>
 8001d08:	ed92 0a00 	vldr	s0, [r2]
 8001d0c:	ed8b 0a00 	vstr	s0, [fp]
 8001d10:	68c3      	ldr	r3, [r0, #12]
 8001d12:	6846      	ldr	r6, [r0, #4]
 8001d14:	1d12      	adds	r2, r2, #4
 8001d16:	eb03 0786 	add.w	r7, r3, r6, lsl #2
 8001d1a:	42ba      	cmp	r2, r7
 8001d1c:	d222      	bcs.n	8001d64 <forward_conv2d_nl_pool+0x3d0>
 8001d1e:	edd2 0a00 	vldr	s1, [r2]
 8001d22:	edcb 0a01 	vstr	s1, [fp, #4]
 8001d26:	68c3      	ldr	r3, [r0, #12]
 8001d28:	6846      	ldr	r6, [r0, #4]
 8001d2a:	1d12      	adds	r2, r2, #4
 8001d2c:	eb03 0786 	add.w	r7, r3, r6, lsl #2
 8001d30:	42ba      	cmp	r2, r7
 8001d32:	d217      	bcs.n	8001d64 <forward_conv2d_nl_pool+0x3d0>
 8001d34:	ed92 0a00 	vldr	s0, [r2]
 8001d38:	ed8b 0a02 	vstr	s0, [fp, #8]
 8001d3c:	68c3      	ldr	r3, [r0, #12]
 8001d3e:	6846      	ldr	r6, [r0, #4]
 8001d40:	1d12      	adds	r2, r2, #4
 8001d42:	eb03 0786 	add.w	r7, r3, r6, lsl #2
 8001d46:	42ba      	cmp	r2, r7
 8001d48:	d20c      	bcs.n	8001d64 <forward_conv2d_nl_pool+0x3d0>
 8001d4a:	edd2 0a00 	vldr	s1, [r2]
 8001d4e:	edcb 0a03 	vstr	s1, [fp, #12]
 8001d52:	68c3      	ldr	r3, [r0, #12]
 8001d54:	6846      	ldr	r6, [r0, #4]
 8001d56:	1d12      	adds	r2, r2, #4
 8001d58:	eb03 0786 	add.w	r7, r3, r6, lsl #2
 8001d5c:	42ba      	cmp	r2, r7
 8001d5e:	f10b 0b10 	add.w	fp, fp, #16
 8001d62:	d3d1      	bcc.n	8001d08 <forward_conv2d_nl_pool+0x374>
 8001d64:	9a2f      	ldr	r2, [sp, #188]	; 0xbc
 8001d66:	9b12      	ldr	r3, [sp, #72]	; 0x48
 8001d68:	189a      	adds	r2, r3, r2
 8001d6a:	eba2 0209 	sub.w	r2, r2, r9
 8001d6e:	922f      	str	r2, [sp, #188]	; 0xbc
 8001d70:	9a11      	ldr	r2, [sp, #68]	; 0x44
 8001d72:	9b37      	ldr	r3, [sp, #220]	; 0xdc
 8001d74:	444a      	add	r2, r9
 8001d76:	fa0f f982 	sxth.w	r9, r2
 8001d7a:	eb01 0b83 	add.w	fp, r1, r3, lsl #2
 8001d7e:	68c1      	ldr	r1, [r0, #12]
 8001d80:	6842      	ldr	r2, [r0, #4]
 8001d82:	eb01 0382 	add.w	r3, r1, r2, lsl #2
 8001d86:	459b      	cmp	fp, r3
 8001d88:	460b      	mov	r3, r1
 8001d8a:	d30f      	bcc.n	8001dac <forward_conv2d_nl_pool+0x418>
 8001d8c:	6841      	ldr	r1, [r0, #4]
 8001d8e:	008a      	lsls	r2, r1, #2
 8001d90:	4252      	negs	r2, r2
 8001d92:	4493      	add	fp, r2
 8001d94:	eb03 0181 	add.w	r1, r3, r1, lsl #2
 8001d98:	458b      	cmp	fp, r1
 8001d9a:	bf24      	itt	cs
 8001d9c:	4493      	addcs	fp, r2
 8001d9e:	458b      	cmpcs	fp, r1
 8001da0:	bf21      	itttt	cs
 8001da2:	4493      	addcs	fp, r2
 8001da4:	458b      	cmpcs	fp, r1
 8001da6:	4493      	addcs	fp, r2
 8001da8:	458b      	cmpcs	fp, r1
 8001daa:	d2ef      	bcs.n	8001d8c <forward_conv2d_nl_pool+0x3f8>
 8001dac:	9812      	ldr	r0, [sp, #72]	; 0x48
 8001dae:	4581      	cmp	r9, r0
 8001db0:	d339      	bcc.n	8001e26 <forward_conv2d_nl_pool+0x492>
 8001db2:	9911      	ldr	r1, [sp, #68]	; 0x44
 8001db4:	9a21      	ldr	r2, [sp, #132]	; 0x84
 8001db6:	9b10      	ldr	r3, [sp, #64]	; 0x40
 8001db8:	9e27      	ldr	r6, [sp, #156]	; 0x9c
 8001dba:	eba9 0001 	sub.w	r0, r9, r1
 8001dbe:	fa0f f980 	sxth.w	r9, r0
 8001dc2:	982e      	ldr	r0, [sp, #184]	; 0xb8
 8001dc4:	1c40      	adds	r0, r0, #1
 8001dc6:	902e      	str	r0, [sp, #184]	; 0xb8
 8001dc8:	2101      	movs	r1, #1
 8001dca:	9825      	ldr	r0, [sp, #148]	; 0x94
 8001dcc:	9008      	str	r0, [sp, #32]
 8001dce:	9107      	str	r1, [sp, #28]
 8001dd0:	b292      	uxth	r2, r2
 8001dd2:	9811      	ldr	r0, [sp, #68]	; 0x44
 8001dd4:	992a      	ldr	r1, [sp, #168]	; 0xa8
 8001dd6:	9206      	str	r2, [sp, #24]
 8001dd8:	b280      	uxth	r0, r0
 8001dda:	9005      	str	r0, [sp, #20]
 8001ddc:	b289      	uxth	r1, r1
 8001dde:	9829      	ldr	r0, [sp, #164]	; 0xa4
 8001de0:	9a12      	ldr	r2, [sp, #72]	; 0x48
 8001de2:	9104      	str	r1, [sp, #16]
 8001de4:	b280      	uxth	r0, r0
 8001de6:	b2a1      	uxth	r1, r4
 8001de8:	9002      	str	r0, [sp, #8]
 8001dea:	9103      	str	r1, [sp, #12]
 8001dec:	b29b      	uxth	r3, r3
 8001dee:	982b      	ldr	r0, [sp, #172]	; 0xac
 8001df0:	9912      	ldr	r1, [sp, #72]	; 0x48
 8001df2:	b280      	uxth	r0, r0
 8001df4:	b289      	uxth	r1, r1
 8001df6:	9000      	str	r0, [sp, #0]
 8001df8:	9101      	str	r1, [sp, #4]
 8001dfa:	982f      	ldr	r0, [sp, #188]	; 0xbc
 8001dfc:	9924      	ldr	r1, [sp, #144]	; 0x90
 8001dfe:	1a12      	subs	r2, r2, r0
 8001e00:	69a8      	ldr	r0, [r5, #24]
 8001e02:	b292      	uxth	r2, r2
 8001e04:	b289      	uxth	r1, r1
 8001e06:	47b0      	blx	r6
 8001e08:	9825      	ldr	r0, [sp, #148]	; 0x94
 8001e0a:	6881      	ldr	r1, [r0, #8]
 8001e0c:	9835      	ldr	r0, [sp, #212]	; 0xd4
 8001e0e:	eb01 0280 	add.w	r2, r1, r0, lsl #2
 8001e12:	9925      	ldr	r1, [sp, #148]	; 0x94
 8001e14:	608a      	str	r2, [r1, #8]
 8001e16:	9836      	ldr	r0, [sp, #216]	; 0xd8
 8001e18:	1a20      	subs	r0, r4, r0
 8001e1a:	2800      	cmp	r0, #0
 8001e1c:	bfc3      	ittte	gt
 8001e1e:	9811      	ldrgt	r0, [sp, #68]	; 0x44
 8001e20:	1a24      	subgt	r4, r4, r0
 8001e22:	b224      	sxthgt	r4, r4
 8001e24:	2400      	movle	r4, #0
 8001e26:	9817      	ldr	r0, [sp, #92]	; 0x5c
 8001e28:	9920      	ldr	r1, [sp, #128]	; 0x80
 8001e2a:	1808      	adds	r0, r1, r0
 8001e2c:	9017      	str	r0, [sp, #92]	; 0x5c
 8001e2e:	9922      	ldr	r1, [sp, #136]	; 0x88
 8001e30:	982e      	ldr	r0, [sp, #184]	; 0xb8
 8001e32:	4288      	cmp	r0, r1
 8001e34:	f4ff aedc 	bcc.w	8001bf0 <forward_conv2d_nl_pool+0x25c>
 8001e38:	9925      	ldr	r1, [sp, #148]	; 0x94
 8001e3a:	69a8      	ldr	r0, [r5, #24]
 8001e3c:	68c2      	ldr	r2, [r0, #12]
 8001e3e:	6082      	str	r2, [r0, #8]
 8001e40:	68c8      	ldr	r0, [r1, #12]
 8001e42:	6088      	str	r0, [r1, #8]
 8001e44:	b039      	add	sp, #228	; 0xe4
 8001e46:	e8bd 8ff0 	ldmia.w	sp!, {r4, r5, r6, r7, r8, r9, sl, fp, pc}
	...

08001e4c <forward_dense>:
 8001e4c:	e92d 4ff0 	stmdb	sp!, {r4, r5, r6, r7, r8, r9, sl, fp, lr}
 8001e50:	b081      	sub	sp, #4
 8001e52:	ed2d 8b02 	vpush	{d8}
 8001e56:	b088      	sub	sp, #32
 8001e58:	6944      	ldr	r4, [r0, #20]
 8001e5a:	8820      	ldrh	r0, [r4, #0]
 8001e5c:	2800      	cmp	r0, #0
 8001e5e:	bf1a      	itte	ne
 8001e60:	6861      	ldrne	r1, [r4, #4]
 8001e62:	1d09      	addne	r1, r1, #4
 8001e64:	2104      	moveq	r1, #4
 8001e66:	6809      	ldr	r1, [r1, #0]
 8001e68:	2900      	cmp	r1, #0
 8001e6a:	bf14      	ite	ne
 8001e6c:	680a      	ldrne	r2, [r1, #0]
 8001e6e:	2200      	moveq	r2, #0
 8001e70:	2802      	cmp	r0, #2
 8001e72:	bfa6      	itte	ge
 8001e74:	6861      	ldrge	r1, [r4, #4]
 8001e76:	3110      	addge	r1, #16
 8001e78:	2104      	movlt	r1, #4
 8001e7a:	6809      	ldr	r1, [r1, #0]
 8001e7c:	2900      	cmp	r1, #0
 8001e7e:	bf14      	ite	ne
 8001e80:	680f      	ldrne	r7, [r1, #0]
 8001e82:	2700      	moveq	r7, #0
 8001e84:	2802      	cmp	r0, #2
 8001e86:	bfc6      	itte	gt
 8001e88:	6861      	ldrgt	r1, [r4, #4]
 8001e8a:	311c      	addgt	r1, #28
 8001e8c:	2104      	movle	r1, #4
 8001e8e:	6809      	ldr	r1, [r1, #0]
 8001e90:	2900      	cmp	r1, #0
 8001e92:	bf14      	ite	ne
 8001e94:	680b      	ldrne	r3, [r1, #0]
 8001e96:	2300      	moveq	r3, #0
 8001e98:	2802      	cmp	r0, #2
 8001e9a:	dd0b      	ble.n	8001eb4 <forward_dense+0x68>
 8001e9c:	6861      	ldr	r1, [r4, #4]
 8001e9e:	f111 0018 	adds.w	r0, r1, #24
 8001ea2:	d007      	beq.n	8001eb4 <forward_dense+0x68>
 8001ea4:	8b08      	ldrh	r0, [r1, #24]
 8001ea6:	2802      	cmp	r0, #2
 8001ea8:	db04      	blt.n	8001eb4 <forward_dense+0x68>
 8001eaa:	69c8      	ldr	r0, [r1, #28]
 8001eac:	b110      	cbz	r0, 8001eb4 <forward_dense+0x68>
 8001eae:	f8d0 a004 	ldr.w	sl, [r0, #4]
 8001eb2:	e001      	b.n	8001eb8 <forward_dense+0x6c>
 8001eb4:	f04f 0a00 	mov.w	sl, #0
 8001eb8:	68d0      	ldr	r0, [r2, #12]
 8001eba:	6844      	ldr	r4, [r0, #4]
 8001ebc:	68f8      	ldr	r0, [r7, #12]
 8001ebe:	6845      	ldr	r5, [r0, #4]
 8001ec0:	6881      	ldr	r1, [r0, #8]
 8001ec2:	68c0      	ldr	r0, [r0, #12]
 8001ec4:	699e      	ldr	r6, [r3, #24]
 8001ec6:	69bf      	ldr	r7, [r7, #24]
 8001ec8:	f8d6 e000 	ldr.w	lr, [r6]
 8001ecc:	6992      	ldr	r2, [r2, #24]
 8001ece:	68bf      	ldr	r7, [r7, #8]
 8001ed0:	4341      	muls	r1, r0
 8001ed2:	2000      	movs	r0, #0
 8001ed4:	ea4f 19ee 	mov.w	r9, lr, asr #7
 8001ed8:	ea4f 586e 	mov.w	r8, lr, asr #21
 8001edc:	ea4f 4e6e 	mov.w	lr, lr, asr #17
 8001ee0:	f00e 0e0f 	and.w	lr, lr, #15
 8001ee4:	f1be 0f04 	cmp.w	lr, #4
 8001ee8:	bf14      	ite	ne
 8001eea:	f1be 0f08 	cmpne.w	lr, #8
 8001eee:	68f0      	ldreq	r0, [r6, #12]
 8001ef0:	f009 097f 	and.w	r9, r9, #127	; 0x7f
 8001ef4:	f008 0803 	and.w	r8, r8, #3
 8001ef8:	695e      	ldr	r6, [r3, #20]
 8001efa:	6876      	ldr	r6, [r6, #4]
 8001efc:	fa29 f908 	lsr.w	r9, r9, r8
 8001f00:	f8d2 8008 	ldr.w	r8, [r2, #8]
 8001f04:	2900      	cmp	r1, #0
 8001f06:	eb07 0285 	add.w	r2, r7, r5, lsl #2
 8001f0a:	f000 80ea 	beq.w	80020e2 <forward_dense+0x296>
 8001f0e:	9307      	str	r3, [sp, #28]
 8001f10:	f8cd a014 	str.w	sl, [sp, #20]
 8001f14:	9506      	str	r5, [sp, #24]
 8001f16:	9201      	str	r2, [sp, #4]
 8001f18:	9104      	str	r1, [sp, #16]
 8001f1a:	9907      	ldr	r1, [sp, #28]
 8001f1c:	698a      	ldr	r2, [r1, #24]
 8001f1e:	9905      	ldr	r1, [sp, #20]
 8001f20:	f8d2 b008 	ldr.w	fp, [r2, #8]
 8001f24:	9b01      	ldr	r3, [sp, #4]
 8001f26:	2900      	cmp	r1, #0
 8001f28:	bf1a      	itte	ne
 8001f2a:	698a      	ldrne	r2, [r1, #24]
 8001f2c:	6892      	ldrne	r2, [r2, #8]
 8001f2e:	2200      	moveq	r2, #0
 8001f30:	2800      	cmp	r0, #0
 8001f32:	f040 80ab 	bne.w	800208c <forward_dense+0x240>
 8001f36:	429f      	cmp	r7, r3
 8001f38:	f080 80c7 	bcs.w	80020ca <forward_dense+0x27e>
 8001f3c:	9003      	str	r0, [sp, #12]
 8001f3e:	2a00      	cmp	r2, #0
 8001f40:	bf0e      	itee	eq
 8001f42:	ed9f 0a6b 	vldreq	s0, [pc, #428]	; 80020f0 <.text_12>
 8001f46:	ed92 0a00 	vldrne	s0, [r2]
 8001f4a:	1d12      	addne	r2, r2, #4
 8001f4c:	2c04      	cmp	r4, #4
 8001f4e:	4620      	mov	r0, r4
 8001f50:	46c6      	mov	lr, r8
 8001f52:	46dc      	mov	ip, fp
 8001f54:	eddf 0a66 	vldr	s1, [pc, #408]	; 80020f0 <.text_12>
 8001f58:	d35d      	bcc.n	8002016 <forward_dense+0x1ca>
 8001f5a:	08a1      	lsrs	r1, r4, #2
 8001f5c:	07cd      	lsls	r5, r1, #31
 8001f5e:	d51c      	bpl.n	8001f9a <forward_dense+0x14e>
 8001f60:	ed9c 4a00 	vldr	s8, [ip]
 8001f64:	edde 4a00 	vldr	s9, [lr]
 8001f68:	ed9c 3a01 	vldr	s6, [ip, #4]
 8001f6c:	edde 3a01 	vldr	s7, [lr, #4]
 8001f70:	ed9c 2a02 	vldr	s4, [ip, #8]
 8001f74:	edde 2a02 	vldr	s5, [lr, #8]
 8001f78:	ed9c 1a03 	vldr	s2, [ip, #12]
 8001f7c:	edde 1a03 	vldr	s3, [lr, #12]
 8001f80:	ee44 0a24 	vmla.f32	s1, s8, s9
 8001f84:	ee43 0a23 	vmla.f32	s1, s6, s7
 8001f88:	ee42 0a22 	vmla.f32	s1, s4, s5
 8001f8c:	ee41 0a21 	vmla.f32	s1, s2, s3
 8001f90:	f10e 0e10 	add.w	lr, lr, #16
 8001f94:	f10c 0c10 	add.w	ip, ip, #16
 8001f98:	1f00      	subs	r0, r0, #4
 8001f9a:	0849      	lsrs	r1, r1, #1
 8001f9c:	f000 803b 	beq.w	8002016 <forward_dense+0x1ca>
 8001fa0:	edde 4a00 	vldr	s9, [lr]
 8001fa4:	edde 3a01 	vldr	s7, [lr, #4]
 8001fa8:	edde 2a02 	vldr	s5, [lr, #8]
 8001fac:	edde 1a03 	vldr	s3, [lr, #12]
 8001fb0:	ed9c 1a03 	vldr	s2, [ip, #12]
 8001fb4:	ed9c 2a02 	vldr	s4, [ip, #8]
 8001fb8:	ed9c 3a01 	vldr	s6, [ip, #4]
 8001fbc:	ed9c 4a00 	vldr	s8, [ip]
 8001fc0:	ee44 0a24 	vmla.f32	s1, s8, s9
 8001fc4:	ee43 0a23 	vmla.f32	s1, s6, s7
 8001fc8:	ee42 0a22 	vmla.f32	s1, s4, s5
 8001fcc:	ee41 0a21 	vmla.f32	s1, s2, s3
 8001fd0:	f10e 0510 	add.w	r5, lr, #16
 8001fd4:	f10c 0c10 	add.w	ip, ip, #16
 8001fd8:	edd5 8a00 	vldr	s17, [r5]
 8001fdc:	ed9c 8a00 	vldr	s16, [ip]
 8001fe0:	ed9c 7a01 	vldr	s14, [ip, #4]
 8001fe4:	edd5 7a01 	vldr	s15, [r5, #4]
 8001fe8:	ed9c 6a02 	vldr	s12, [ip, #8]
 8001fec:	edd5 6a02 	vldr	s13, [r5, #8]
 8001ff0:	ed9c 5a03 	vldr	s10, [ip, #12]
 8001ff4:	edd5 5a03 	vldr	s11, [r5, #12]
 8001ff8:	ee48 0a28 	vmla.f32	s1, s16, s17
 8001ffc:	ee47 0a27 	vmla.f32	s1, s14, s15
 8002000:	3808      	subs	r0, #8
 8002002:	ee46 0a26 	vmla.f32	s1, s12, s13
 8002006:	1e49      	subs	r1, r1, #1
 8002008:	ee45 0a25 	vmla.f32	s1, s10, s11
 800200c:	f105 0e10 	add.w	lr, r5, #16
 8002010:	f10c 0c10 	add.w	ip, ip, #16
 8002014:	d1c4      	bne.n	8001fa0 <forward_dense+0x154>
 8002016:	b378      	cbz	r0, 8002078 <forward_dense+0x22c>
 8002018:	f010 0103 	ands.w	r1, r0, #3
 800201c:	f000 800c 	beq.w	8002038 <forward_dense+0x1ec>
 8002020:	ed9c 1a00 	vldr	s2, [ip]
 8002024:	edde 1a00 	vldr	s3, [lr]
 8002028:	1e49      	subs	r1, r1, #1
 800202a:	ee41 0a21 	vmla.f32	s1, s2, s3
 800202e:	f10e 0e04 	add.w	lr, lr, #4
 8002032:	f10c 0c04 	add.w	ip, ip, #4
 8002036:	d1f3      	bne.n	8002020 <forward_dense+0x1d4>
 8002038:	0880      	lsrs	r0, r0, #2
 800203a:	d01d      	beq.n	8002078 <forward_dense+0x22c>
 800203c:	ed9c 2a00 	vldr	s4, [ip]
 8002040:	ed9e 1a00 	vldr	s2, [lr]
 8002044:	eddc 1a01 	vldr	s3, [ip, #4]
 8002048:	edde 2a01 	vldr	s5, [lr, #4]
 800204c:	ee42 0a01 	vmla.f32	s1, s4, s2
 8002050:	ee41 0aa2 	vmla.f32	s1, s3, s5
 8002054:	ed9c 2a02 	vldr	s4, [ip, #8]
 8002058:	ed9e 1a02 	vldr	s2, [lr, #8]
 800205c:	eddc 1a03 	vldr	s3, [ip, #12]
 8002060:	edde 2a03 	vldr	s5, [lr, #12]
 8002064:	ee42 0a01 	vmla.f32	s1, s4, s2
 8002068:	1e40      	subs	r0, r0, #1
 800206a:	ee41 0aa2 	vmla.f32	s1, s3, s5
 800206e:	f10e 0e10 	add.w	lr, lr, #16
 8002072:	f10c 0c10 	add.w	ip, ip, #16
 8002076:	d1e1      	bne.n	800203c <forward_dense+0x1f0>
 8002078:	ee30 0a20 	vadd.f32	s0, s0, s1
 800207c:	ed87 0a00 	vstr	s0, [r7]
 8002080:	1d3f      	adds	r7, r7, #4
 8002082:	429f      	cmp	r7, r3
 8002084:	44b3      	add	fp, r6
 8002086:	f4ff af5a 	bcc.w	8001f3e <forward_dense+0xf2>
 800208a:	e01d      	b.n	80020c8 <forward_dense+0x27c>
 800208c:	429f      	cmp	r7, r3
 800208e:	d21c      	bcs.n	80020ca <forward_dense+0x27e>
 8002090:	469a      	mov	sl, r3
 8002092:	9003      	str	r0, [sp, #12]
 8002094:	4615      	mov	r5, r2
 8002096:	2d00      	cmp	r5, #0
 8002098:	bf14      	ite	ne
 800209a:	f855 0b04 	ldrne.w	r0, [r5], #4
 800209e:	2000      	moveq	r0, #0
 80020a0:	9002      	str	r0, [sp, #8]
 80020a2:	f1b9 0f04 	cmp.w	r9, #4
 80020a6:	9a03      	ldr	r2, [sp, #12]
 80020a8:	9400      	str	r4, [sp, #0]
 80020aa:	4643      	mov	r3, r8
 80020ac:	4659      	mov	r1, fp
 80020ae:	a802      	add	r0, sp, #8
 80020b0:	d102      	bne.n	80020b8 <forward_dense+0x26c>
 80020b2:	f7ff fa03 	bl	80014bc <ai_dict4_dot_array_f32>
 80020b6:	e001      	b.n	80020bc <forward_dense+0x270>
 80020b8:	f7ff f950 	bl	800135c <ai_dict8_dot_array_f32>
 80020bc:	9802      	ldr	r0, [sp, #8]
 80020be:	f847 0b04 	str.w	r0, [r7], #4
 80020c2:	4557      	cmp	r7, sl
 80020c4:	44b3      	add	fp, r6
 80020c6:	d3e6      	bcc.n	8002096 <forward_dense+0x24a>
 80020c8:	9803      	ldr	r0, [sp, #12]
 80020ca:	9901      	ldr	r1, [sp, #4]
 80020cc:	9a06      	ldr	r2, [sp, #24]
 80020ce:	eb01 0382 	add.w	r3, r1, r2, lsl #2
 80020d2:	9904      	ldr	r1, [sp, #16]
 80020d4:	9301      	str	r3, [sp, #4]
 80020d6:	1e49      	subs	r1, r1, #1
 80020d8:	eb08 0884 	add.w	r8, r8, r4, lsl #2
 80020dc:	9104      	str	r1, [sp, #16]
 80020de:	f47f af1c 	bne.w	8001f1a <forward_dense+0xce>
 80020e2:	b008      	add	sp, #32
 80020e4:	ecbd 8b02 	vpop	{d8}
 80020e8:	b001      	add	sp, #4
 80020ea:	e8bd 8ff0 	ldmia.w	sp!, {r4, r5, r6, r7, r8, r9, sl, fp, pc}
	...

080020f0 <.text_12>:
 80020f0:	00000000 	.word	0x00000000

080020f4 <forward_gemm>:
 80020f4:	e92d 4ff0 	stmdb	sp!, {r4, r5, r6, r7, r8, r9, sl, fp, lr}
 80020f8:	4604      	mov	r4, r0
 80020fa:	b091      	sub	sp, #68	; 0x44
 80020fc:	6961      	ldr	r1, [r4, #20]
 80020fe:	8808      	ldrh	r0, [r1, #0]
 8002100:	2800      	cmp	r0, #0
 8002102:	bf1a      	itte	ne
 8002104:	6848      	ldrne	r0, [r1, #4]
 8002106:	1d02      	addne	r2, r0, #4
 8002108:	2204      	moveq	r2, #4
 800210a:	460b      	mov	r3, r1
 800210c:	6810      	ldr	r0, [r2, #0]
 800210e:	8819      	ldrh	r1, [r3, #0]
 8002110:	2800      	cmp	r0, #0
 8002112:	bf14      	ite	ne
 8002114:	6805      	ldrne	r5, [r0, #0]
 8002116:	2500      	moveq	r5, #0
 8002118:	2900      	cmp	r1, #0
 800211a:	bf1d      	ittte	ne
 800211c:	6858      	ldrne	r0, [r3, #4]
 800211e:	2800      	cmpne	r0, #0
 8002120:	f8b0 c000 	ldrhne.w	ip, [r0]
 8002124:	f04f 0c00 	moveq.w	ip, #0
 8002128:	2902      	cmp	r1, #2
 800212a:	bfa6      	itte	ge
 800212c:	6858      	ldrge	r0, [r3, #4]
 800212e:	3010      	addge	r0, #16
 8002130:	2004      	movlt	r0, #4
 8002132:	6800      	ldr	r0, [r0, #0]
 8002134:	2800      	cmp	r0, #0
 8002136:	bf14      	ite	ne
 8002138:	6801      	ldrne	r1, [r0, #0]
 800213a:	2100      	moveq	r1, #0
 800213c:	2600      	movs	r6, #0
 800213e:	f1bc 0f03 	cmp.w	ip, #3
 8002142:	46b2      	mov	sl, r6
 8002144:	d107      	bne.n	8002156 <forward_gemm+0x62>
 8002146:	6810      	ldr	r0, [r2, #0]
 8002148:	2800      	cmp	r0, #0
 800214a:	d026      	beq.n	800219a <forward_gemm+0xa6>
 800214c:	6846      	ldr	r6, [r0, #4]
 800214e:	d024      	beq.n	800219a <forward_gemm+0xa6>
 8002150:	f8d0 a008 	ldr.w	sl, [r0, #8]
 8002154:	e021      	b.n	800219a <forward_gemm+0xa6>
 8002156:	f1bc 0f02 	cmp.w	ip, #2
 800215a:	d10d      	bne.n	8002178 <forward_gemm+0x84>
 800215c:	6810      	ldr	r0, [r2, #0]
 800215e:	b100      	cbz	r0, 8002162 <forward_gemm+0x6e>
 8002160:	6846      	ldr	r6, [r0, #4]
 8002162:	881a      	ldrh	r2, [r3, #0]
 8002164:	2a02      	cmp	r2, #2
 8002166:	bfc6      	itte	gt
 8002168:	6858      	ldrgt	r0, [r3, #4]
 800216a:	301c      	addgt	r0, #28
 800216c:	2004      	movle	r0, #4
 800216e:	6800      	ldr	r0, [r0, #0]
 8002170:	b198      	cbz	r0, 800219a <forward_gemm+0xa6>
 8002172:	f8d0 a000 	ldr.w	sl, [r0]
 8002176:	e010      	b.n	800219a <forward_gemm+0xa6>
 8002178:	f1bc 0f01 	cmp.w	ip, #1
 800217c:	d10d      	bne.n	800219a <forward_gemm+0xa6>
 800217e:	881a      	ldrh	r2, [r3, #0]
 8002180:	2a02      	cmp	r2, #2
 8002182:	bfc6      	itte	gt
 8002184:	6858      	ldrgt	r0, [r3, #4]
 8002186:	f100 021c 	addgt.w	r2, r0, #28
 800218a:	2204      	movle	r2, #4
 800218c:	6810      	ldr	r0, [r2, #0]
 800218e:	2800      	cmp	r0, #0
 8002190:	d003      	beq.n	800219a <forward_gemm+0xa6>
 8002192:	6806      	ldr	r6, [r0, #0]
 8002194:	bf18      	it	ne
 8002196:	f8d0 a004 	ldrne.w	sl, [r0, #4]
 800219a:	68c8      	ldr	r0, [r1, #12]
 800219c:	6989      	ldr	r1, [r1, #24]
 800219e:	688b      	ldr	r3, [r1, #8]
 80021a0:	6842      	ldr	r2, [r0, #4]
 80021a2:	68c1      	ldr	r1, [r0, #12]
 80021a4:	b292      	uxth	r2, r2
 80021a6:	b289      	uxth	r1, r1
 80021a8:	a806      	add	r0, sp, #24
 80021aa:	f004 f831 	bl	8006210 <arm_mat_init_f32>
 80021ae:	69a9      	ldr	r1, [r5, #24]
 80021b0:	68e8      	ldr	r0, [r5, #12]
 80021b2:	688b      	ldr	r3, [r1, #8]
 80021b4:	6842      	ldr	r2, [r0, #4]
 80021b6:	68c1      	ldr	r1, [r0, #12]
 80021b8:	b292      	uxth	r2, r2
 80021ba:	b289      	uxth	r1, r1
 80021bc:	a804      	add	r0, sp, #16
 80021be:	f004 f827 	bl	8006210 <arm_mat_init_f32>
 80021c2:	69b1      	ldr	r1, [r6, #24]
 80021c4:	68f0      	ldr	r0, [r6, #12]
 80021c6:	688b      	ldr	r3, [r1, #8]
 80021c8:	6842      	ldr	r2, [r0, #4]
 80021ca:	68c1      	ldr	r1, [r0, #12]
 80021cc:	b292      	uxth	r2, r2
 80021ce:	b289      	uxth	r1, r1
 80021d0:	a802      	add	r0, sp, #8
 80021d2:	f004 f81d 	bl	8006210 <arm_mat_init_f32>
 80021d6:	f8da 1018 	ldr.w	r1, [sl, #24]
 80021da:	f8da 000c 	ldr.w	r0, [sl, #12]
 80021de:	688b      	ldr	r3, [r1, #8]
 80021e0:	6842      	ldr	r2, [r0, #4]
 80021e2:	68c1      	ldr	r1, [r0, #12]
 80021e4:	b292      	uxth	r2, r2
 80021e6:	b289      	uxth	r1, r1
 80021e8:	4668      	mov	r0, sp
 80021ea:	f004 f811 	bl	8006210 <arm_mat_init_f32>
 80021ee:	f994 5021 	ldrsb.w	r5, [r4, #33]	; 0x21
 80021f2:	f994 0020 	ldrsb.w	r0, [r4, #32]
 80021f6:	9905      	ldr	r1, [sp, #20]
 80021f8:	9a03      	ldr	r2, [sp, #12]
 80021fa:	ed94 0a07 	vldr	s0, [r4, #28]
 80021fe:	edd4 0a06 	vldr	s1, [r4, #24]
 8002202:	910b      	str	r1, [sp, #44]	; 0x2c
 8002204:	920e      	str	r2, [sp, #56]	; 0x38
 8002206:	920d      	str	r2, [sp, #52]	; 0x34
 8002208:	2300      	movs	r3, #0
 800220a:	f8bd e010 	ldrh.w	lr, [sp, #16]
 800220e:	f8bd 8012 	ldrh.w	r8, [sp, #18]
 8002212:	9901      	ldr	r1, [sp, #4]
 8002214:	f8bd 7002 	ldrh.w	r7, [sp, #2]
 8002218:	f8bd c000 	ldrh.w	ip, [sp]
 800221c:	9c07      	ldr	r4, [sp, #28]
 800221e:	f8bd a008 	ldrh.w	sl, [sp, #8]
 8002222:	f8bd 6018 	ldrh.w	r6, [sp, #24]
 8002226:	f8bd b01a 	ldrh.w	fp, [sp, #26]
 800222a:	9108      	str	r1, [sp, #32]
 800222c:	0002      	movs	r2, r0
 800222e:	bf0c      	ite	eq
 8002230:	4672      	moveq	r2, lr
 8002232:	4642      	movne	r2, r8
 8002234:	2f01      	cmp	r7, #1
 8002236:	bf0c      	ite	eq
 8002238:	4699      	moveq	r9, r3
 800223a:	f04f 0904 	movne.w	r9, #4
 800223e:	f8bd 100a 	ldrh.w	r1, [sp, #10]
 8002242:	f1bc 0f01 	cmp.w	ip, #1
 8002246:	d104      	bne.n	8002252 <forward_gemm+0x15e>
 8002248:	2f01      	cmp	r7, #1
 800224a:	d004      	beq.n	8002256 <forward_gemm+0x162>
 800224c:	f1cb 0700 	rsb	r7, fp, #0
 8002250:	e002      	b.n	8002258 <forward_gemm+0x164>
 8002252:	2f01      	cmp	r7, #1
 8002254:	d000      	beq.n	8002258 <forward_gemm+0x164>
 8002256:	2700      	movs	r7, #0
 8002258:	2800      	cmp	r0, #0
 800225a:	bf0c      	ite	eq
 800225c:	46f4      	moveq	ip, lr
 800225e:	46c4      	movne	ip, r8
 8002260:	b23f      	sxth	r7, r7
 8002262:	45b4      	cmp	ip, r6
 8002264:	970c      	str	r7, [sp, #48]	; 0x30
 8002266:	f040 808b 	bne.w	8002380 <forward_gemm+0x28c>
 800226a:	2d00      	cmp	r5, #0
 800226c:	bf0c      	ite	eq
 800226e:	9109      	streq	r1, [sp, #36]	; 0x24
 8002270:	f8cd a024 	strne.w	sl, [sp, #36]	; 0x24
 8002274:	9f09      	ldr	r7, [sp, #36]	; 0x24
 8002276:	455f      	cmp	r7, fp
 8002278:	f040 8082 	bne.w	8002380 <forward_gemm+0x28c>
 800227c:	2800      	cmp	r0, #0
 800227e:	bf0c      	ite	eq
 8002280:	46c4      	moveq	ip, r8
 8002282:	46f4      	movne	ip, lr
 8002284:	2d00      	cmp	r5, #0
 8002286:	bf0c      	ite	eq
 8002288:	4657      	moveq	r7, sl
 800228a:	460f      	movne	r7, r1
 800228c:	45bc      	cmp	ip, r7
 800228e:	d177      	bne.n	8002380 <forward_gemm+0x28c>
 8002290:	9e08      	ldr	r6, [sp, #32]
 8002292:	f8dd c02c 	ldr.w	ip, [sp, #44]	; 0x2c
 8002296:	9410      	str	r4, [sp, #64]	; 0x40
 8002298:	f8ad 3022 	strh.w	r3, [sp, #34]	; 0x22
 800229c:	f8ad 2020 	strh.w	r2, [sp, #32]
 80022a0:	9a10      	ldr	r2, [sp, #64]	; 0x40
 80022a2:	f8bd 3022 	ldrh.w	r3, [sp, #34]	; 0x22
 80022a6:	f8cd c02c 	str.w	ip, [sp, #44]	; 0x2c
 80022aa:	eb02 0783 	add.w	r7, r2, r3, lsl #2
 80022ae:	9a09      	ldr	r2, [sp, #36]	; 0x24
 80022b0:	9b0e      	ldr	r3, [sp, #56]	; 0x38
 80022b2:	f8dd c034 	ldr.w	ip, [sp, #52]	; 0x34
 80022b6:	f8ad e028 	strh.w	lr, [sp, #40]	; 0x28
 80022ba:	ea4f 0488 	mov.w	r4, r8, lsl #2
 80022be:	f8cd 803c 	str.w	r8, [sp, #60]	; 0x3c
 80022c2:	2800      	cmp	r0, #0
 80022c4:	bf0c      	ite	eq
 80022c6:	f8dd 803c 	ldreq.w	r8, [sp, #60]	; 0x3c
 80022ca:	f8bd 8028 	ldrhne.w	r8, [sp, #40]	; 0x28
 80022ce:	fa1f fb88 	uxth.w	fp, r8
 80022d2:	f8dd e02c 	ldr.w	lr, [sp, #44]	; 0x2c
 80022d6:	f1bb 0f00 	cmp.w	fp, #0
 80022da:	ed9f 1a9a 	vldr	s2, [pc, #616]	; 8002544 <.text_16>
 80022de:	d019      	beq.n	8002314 <forward_gemm+0x220>
 80022e0:	2800      	cmp	r0, #0
 80022e2:	bf0c      	ite	eq
 80022e4:	f04f 0b04 	moveq.w	fp, #4
 80022e8:	46a3      	movne	fp, r4
 80022ea:	2d00      	cmp	r5, #0
 80022ec:	f1a8 0801 	sub.w	r8, r8, #1
 80022f0:	edde 1a00 	vldr	s3, [lr]
 80022f4:	ed93 2a00 	vldr	s4, [r3]
 80022f8:	44de      	add	lr, fp
 80022fa:	bf0c      	ite	eq
 80022fc:	ea4f 0b81 	moveq.w	fp, r1, lsl #2
 8002300:	f04f 0b04 	movne.w	fp, #4
 8002304:	445b      	add	r3, fp
 8002306:	fa1f fb88 	uxth.w	fp, r8
 800230a:	f1bb 0f00 	cmp.w	fp, #0
 800230e:	ee01 1a82 	vmla.f32	s2, s3, s4
 8002312:	d1e5      	bne.n	80022e0 <forward_gemm+0x1ec>
 8002314:	ee20 1a81 	vmul.f32	s2, s1, s2
 8002318:	edd6 1a00 	vldr	s3, [r6]
 800231c:	ee00 1a21 	vmla.f32	s2, s0, s3
 8002320:	ed87 1a00 	vstr	s2, [r7]
 8002324:	1d3f      	adds	r7, r7, #4
 8002326:	1e52      	subs	r2, r2, #1
 8002328:	b292      	uxth	r2, r2
 800232a:	002b      	movs	r3, r5
 800232c:	bf0e      	itee	eq
 800232e:	1a8b      	subeq	r3, r1, r2
 8002330:	ebaa 0302 	subne.w	r3, sl, r2
 8002334:	434b      	mulne	r3, r1
 8002336:	2a00      	cmp	r2, #0
 8002338:	444e      	add	r6, r9
 800233a:	eb0c 0383 	add.w	r3, ip, r3, lsl #2
 800233e:	d1c0      	bne.n	80022c2 <forward_gemm+0x1ce>
 8002340:	f8bd 7022 	ldrh.w	r7, [sp, #34]	; 0x22
 8002344:	9b09      	ldr	r3, [sp, #36]	; 0x24
 8002346:	9a0b      	ldr	r2, [sp, #44]	; 0x2c
 8002348:	f8bd e028 	ldrh.w	lr, [sp, #40]	; 0x28
 800234c:	f8dd 803c 	ldr.w	r8, [sp, #60]	; 0x3c
 8002350:	f8cd c034 	str.w	ip, [sp, #52]	; 0x34
 8002354:	19df      	adds	r7, r3, r7
 8002356:	f8ad 7022 	strh.w	r7, [sp, #34]	; 0x22
 800235a:	b100      	cbz	r0, 800235e <forward_gemm+0x26a>
 800235c:	2404      	movs	r4, #4
 800235e:	eb02 0c04 	add.w	ip, r2, r4
 8002362:	f8bd 4020 	ldrh.w	r4, [sp, #32]
 8002366:	9a0c      	ldr	r2, [sp, #48]	; 0x30
 8002368:	1e67      	subs	r7, r4, #1
 800236a:	eb06 0682 	add.w	r6, r6, r2, lsl #2
 800236e:	f8ad 7020 	strh.w	r7, [sp, #32]
 8002372:	f8bd 2020 	ldrh.w	r2, [sp, #32]
 8002376:	2a00      	cmp	r2, #0
 8002378:	d192      	bne.n	80022a0 <forward_gemm+0x1ac>
 800237a:	b011      	add	sp, #68	; 0x44
 800237c:	e8bd 8ff0 	ldmia.w	sp!, {r4, r5, r6, r7, r8, r9, sl, fp, pc}
 8002380:	fb0b f606 	mul.w	r6, fp, r6
 8002384:	2e00      	cmp	r6, #0
 8002386:	ddf8      	ble.n	800237a <forward_gemm+0x286>
 8002388:	f016 0003 	ands.w	r0, r6, #3
 800238c:	d003      	beq.n	8002396 <forward_gemm+0x2a2>
 800238e:	1e40      	subs	r0, r0, #1
 8002390:	f844 3b04 	str.w	r3, [r4], #4
 8002394:	d1fb      	bne.n	800238e <forward_gemm+0x29a>
 8002396:	08b1      	lsrs	r1, r6, #2
 8002398:	d0ef      	beq.n	800237a <forward_gemm+0x286>
 800239a:	6023      	str	r3, [r4, #0]
 800239c:	6063      	str	r3, [r4, #4]
 800239e:	60a3      	str	r3, [r4, #8]
 80023a0:	60e3      	str	r3, [r4, #12]
 80023a2:	3410      	adds	r4, #16
 80023a4:	1e49      	subs	r1, r1, #1
 80023a6:	d1f8      	bne.n	800239a <forward_gemm+0x2a6>
 80023a8:	b011      	add	sp, #68	; 0x44
 80023aa:	e8bd 8ff0 	ldmia.w	sp!, {r4, r5, r6, r7, r8, r9, sl, fp, pc}
	...

080023b0 <forward_matmul>:
 80023b0:	e92d 4ff0 	stmdb	sp!, {r4, r5, r6, r7, r8, r9, sl, fp, lr}
 80023b4:	b08b      	sub	sp, #44	; 0x2c
 80023b6:	6944      	ldr	r4, [r0, #20]
 80023b8:	8822      	ldrh	r2, [r4, #0]
 80023ba:	2a00      	cmp	r2, #0
 80023bc:	bf1a      	itte	ne
 80023be:	6860      	ldrne	r0, [r4, #4]
 80023c0:	1d03      	addne	r3, r0, #4
 80023c2:	2304      	moveq	r3, #4
 80023c4:	6819      	ldr	r1, [r3, #0]
 80023c6:	2900      	cmp	r1, #0
 80023c8:	bf14      	ite	ne
 80023ca:	6808      	ldrne	r0, [r1, #0]
 80023cc:	2000      	moveq	r0, #0
 80023ce:	2900      	cmp	r1, #0
 80023d0:	bf14      	ite	ne
 80023d2:	f8d1 b004 	ldrne.w	fp, [r1, #4]
 80023d6:	f04f 0b00 	moveq.w	fp, #0
 80023da:	2a02      	cmp	r2, #2
 80023dc:	bfa6      	itte	ge
 80023de:	6861      	ldrge	r1, [r4, #4]
 80023e0:	3110      	addge	r1, #16
 80023e2:	2104      	movlt	r1, #4
 80023e4:	6809      	ldr	r1, [r1, #0]
 80023e6:	2900      	cmp	r1, #0
 80023e8:	bf14      	ite	ne
 80023ea:	680b      	ldrne	r3, [r1, #0]
 80023ec:	2300      	moveq	r3, #0
 80023ee:	f1bb 0f00 	cmp.w	fp, #0
 80023f2:	d108      	bne.n	8002406 <forward_matmul+0x56>
 80023f4:	2a02      	cmp	r2, #2
 80023f6:	bfc6      	itte	gt
 80023f8:	6861      	ldrgt	r1, [r4, #4]
 80023fa:	311c      	addgt	r1, #28
 80023fc:	2104      	movle	r1, #4
 80023fe:	6809      	ldr	r1, [r1, #0]
 8002400:	b109      	cbz	r1, 8002406 <forward_matmul+0x56>
 8002402:	f8d1 b000 	ldr.w	fp, [r1]
 8002406:	68dd      	ldr	r5, [r3, #12]
 8002408:	68c4      	ldr	r4, [r0, #12]
 800240a:	f8db 900c 	ldr.w	r9, [fp, #12]
 800240e:	686e      	ldr	r6, [r5, #4]
 8002410:	f8d4 e000 	ldr.w	lr, [r4]
 8002414:	f8d9 2000 	ldr.w	r2, [r9]
 8002418:	f8d5 a000 	ldr.w	sl, [r5]
 800241c:	68a1      	ldr	r1, [r4, #8]
 800241e:	f8d9 8008 	ldr.w	r8, [r9, #8]
 8002422:	f8d5 c008 	ldr.w	ip, [r5, #8]
 8002426:	68ef      	ldr	r7, [r5, #12]
 8002428:	9706      	str	r7, [sp, #24]
 800242a:	fb01 f50e 	mul.w	r5, r1, lr
 800242e:	699b      	ldr	r3, [r3, #24]
 8002430:	68e7      	ldr	r7, [r4, #12]
 8002432:	689b      	ldr	r3, [r3, #8]
 8002434:	434f      	muls	r7, r1
 8002436:	fb0e f707 	mul.w	r7, lr, r7
 800243a:	970a      	str	r7, [sp, #40]	; 0x28
 800243c:	f8d9 400c 	ldr.w	r4, [r9, #12]
 8002440:	fb08 f404 	mul.w	r4, r8, r4
 8002444:	4354      	muls	r4, r2
 8002446:	2e00      	cmp	r6, #0
 8002448:	9409      	str	r4, [sp, #36]	; 0x24
 800244a:	fb08 f802 	mul.w	r8, r8, r2
 800244e:	d074      	beq.n	800253a <forward_matmul+0x18a>
 8002450:	2400      	movs	r4, #0
 8002452:	46a1      	mov	r9, r4
 8002454:	9602      	str	r6, [sp, #8]
 8002456:	9e06      	ldr	r6, [sp, #24]
 8002458:	2e00      	cmp	r6, #0
 800245a:	d064      	beq.n	8002526 <forward_matmul+0x176>
 800245c:	9f06      	ldr	r7, [sp, #24]
 800245e:	9701      	str	r7, [sp, #4]
 8002460:	f8cd c00c 	str.w	ip, [sp, #12]
 8002464:	2600      	movs	r6, #0
 8002466:	9505      	str	r5, [sp, #20]
 8002468:	9d03      	ldr	r5, [sp, #12]
 800246a:	2d00      	cmp	r5, #0
 800246c:	d051      	beq.n	8002512 <forward_matmul+0x162>
 800246e:	9500      	str	r5, [sp, #0]
 8002470:	f8cd a010 	str.w	sl, [sp, #16]
 8002474:	9207      	str	r2, [sp, #28]
 8002476:	f04f 0a00 	mov.w	sl, #0
 800247a:	9a04      	ldr	r2, [sp, #16]
 800247c:	2a00      	cmp	r2, #0
 800247e:	d03f      	beq.n	8002500 <forward_matmul+0x150>
 8002480:	f04f 0c00 	mov.w	ip, #0
 8002484:	9008      	str	r0, [sp, #32]
 8002486:	9808      	ldr	r0, [sp, #32]
 8002488:	6985      	ldr	r5, [r0, #24]
 800248a:	68a8      	ldr	r0, [r5, #8]
 800248c:	f8db 7018 	ldr.w	r7, [fp, #24]
 8002490:	4420      	add	r0, r4
 8002492:	4430      	add	r0, r6
 8002494:	eb00 050c 	add.w	r5, r0, ip
 8002498:	68b8      	ldr	r0, [r7, #8]
 800249a:	4448      	add	r0, r9
 800249c:	4450      	add	r0, sl
 800249e:	eb00 070c 	add.w	r7, r0, ip
 80024a2:	ed9f 0a28 	vldr	s0, [pc, #160]	; 8002544 <.text_16>
 80024a6:	b319      	cbz	r1, 80024f0 <forward_matmul+0x140>
 80024a8:	07c8      	lsls	r0, r1, #31
 80024aa:	d509      	bpl.n	80024c0 <forward_matmul+0x110>
 80024ac:	edd5 0a00 	vldr	s1, [r5]
 80024b0:	ed97 1a00 	vldr	s2, [r7]
 80024b4:	ee00 0a81 	vmla.f32	s0, s1, s2
 80024b8:	eb05 058e 	add.w	r5, r5, lr, lsl #2
 80024bc:	eb07 0788 	add.w	r7, r7, r8, lsl #2
 80024c0:	0848      	lsrs	r0, r1, #1
 80024c2:	d015      	beq.n	80024f0 <forward_matmul+0x140>
 80024c4:	edd5 0a00 	vldr	s1, [r5]
 80024c8:	ed97 1a00 	vldr	s2, [r7]
 80024cc:	eb05 058e 	add.w	r5, r5, lr, lsl #2
 80024d0:	eb07 0788 	add.w	r7, r7, r8, lsl #2
 80024d4:	ee00 0a81 	vmla.f32	s0, s1, s2
 80024d8:	edd5 0a00 	vldr	s1, [r5]
 80024dc:	ed97 1a00 	vldr	s2, [r7]
 80024e0:	1e40      	subs	r0, r0, #1
 80024e2:	ee00 0a81 	vmla.f32	s0, s1, s2
 80024e6:	eb05 058e 	add.w	r5, r5, lr, lsl #2
 80024ea:	eb07 0788 	add.w	r7, r7, r8, lsl #2
 80024ee:	d1e9      	bne.n	80024c4 <forward_matmul+0x114>
 80024f0:	ed83 0a00 	vstr	s0, [r3]
 80024f4:	1d1b      	adds	r3, r3, #4
 80024f6:	1e52      	subs	r2, r2, #1
 80024f8:	f10c 0c04 	add.w	ip, ip, #4
 80024fc:	d1c3      	bne.n	8002486 <forward_matmul+0xd6>
 80024fe:	9808      	ldr	r0, [sp, #32]
 8002500:	9d00      	ldr	r5, [sp, #0]
 8002502:	9a07      	ldr	r2, [sp, #28]
 8002504:	1e6d      	subs	r5, r5, #1
 8002506:	eb0a 0a82 	add.w	sl, sl, r2, lsl #2
 800250a:	9500      	str	r5, [sp, #0]
 800250c:	d1b5      	bne.n	800247a <forward_matmul+0xca>
 800250e:	f8dd a010 	ldr.w	sl, [sp, #16]
 8002512:	9f01      	ldr	r7, [sp, #4]
 8002514:	9d05      	ldr	r5, [sp, #20]
 8002516:	1e7f      	subs	r7, r7, #1
 8002518:	eb06 0685 	add.w	r6, r6, r5, lsl #2
 800251c:	9701      	str	r7, [sp, #4]
 800251e:	d1a3      	bne.n	8002468 <forward_matmul+0xb8>
 8002520:	f8dd c00c 	ldr.w	ip, [sp, #12]
 8002524:	9d05      	ldr	r5, [sp, #20]
 8002526:	9e09      	ldr	r6, [sp, #36]	; 0x24
 8002528:	9f0a      	ldr	r7, [sp, #40]	; 0x28
 800252a:	eb09 0986 	add.w	r9, r9, r6, lsl #2
 800252e:	9e02      	ldr	r6, [sp, #8]
 8002530:	1e76      	subs	r6, r6, #1
 8002532:	eb04 0487 	add.w	r4, r4, r7, lsl #2
 8002536:	9602      	str	r6, [sp, #8]
 8002538:	d18d      	bne.n	8002456 <forward_matmul+0xa6>
 800253a:	b00b      	add	sp, #44	; 0x2c
 800253c:	e8bd 8ff0 	ldmia.w	sp!, {r4, r5, r6, r7, r8, r9, sl, fp, pc}

08002540 <.text_15>:
 8002540:	0800135b 	.word	0x0800135b

08002544 <.text_16>:
 8002544:	00000000 	.word	0x00000000

08002548 <ai_shape_get_size>:
 8002548:	b470      	push	{r4, r5, r6}
 800254a:	4601      	mov	r1, r0
 800254c:	f04f 0201 	mov.w	r2, #1
 8002550:	680b      	ldr	r3, [r1, #0]
 8002552:	0a1b      	lsrs	r3, r3, #8
 8002554:	d01e      	beq.n	8002594 <ai_shape_get_size+0x4c>
 8002556:	684c      	ldr	r4, [r1, #4]
 8002558:	eb04 0183 	add.w	r1, r4, r3, lsl #2
 800255c:	4618      	mov	r0, r3
 800255e:	1f0d      	subs	r5, r1, #4
 8002560:	f010 0103 	ands.w	r1, r0, #3
 8002564:	f000 8006 	beq.w	8002574 <ai_shape_get_size+0x2c>
 8002568:	f855 6904 	ldr.w	r6, [r5], #-4
 800256c:	1e5b      	subs	r3, r3, #1
 800256e:	4372      	muls	r2, r6
 8002570:	1e49      	subs	r1, r1, #1
 8002572:	d1f9      	bne.n	8002568 <ai_shape_get_size+0x20>
 8002574:	0880      	lsrs	r0, r0, #2
 8002576:	d00d      	beq.n	8002594 <ai_shape_get_size+0x4c>
 8002578:	eb04 0183 	add.w	r1, r4, r3, lsl #2
 800257c:	3910      	subs	r1, #16
 800257e:	68cb      	ldr	r3, [r1, #12]
 8002580:	688c      	ldr	r4, [r1, #8]
 8002582:	684d      	ldr	r5, [r1, #4]
 8002584:	f851 6910 	ldr.w	r6, [r1], #-16
 8002588:	4363      	muls	r3, r4
 800258a:	436b      	muls	r3, r5
 800258c:	4373      	muls	r3, r6
 800258e:	435a      	muls	r2, r3
 8002590:	1e40      	subs	r0, r0, #1
 8002592:	d1f4      	bne.n	800257e <ai_shape_get_size+0x36>
 8002594:	bc70      	pop	{r4, r5, r6}
 8002596:	4610      	mov	r0, r2
 8002598:	4770      	bx	lr
	...

0800259c <nl_func_acos_array_f32>:
 800259c:	b570      	push	{r4, r5, r6, lr}
 800259e:	688c      	ldr	r4, [r1, #8]
 80025a0:	6880      	ldr	r0, [r0, #8]
 80025a2:	eb04 0182 	add.w	r1, r4, r2, lsl #2
 80025a6:	1f0d      	subs	r5, r1, #4
 80025a8:	eb00 0182 	add.w	r1, r0, r2, lsl #2
 80025ac:	1f0e      	subs	r6, r1, #4
 80025ae:	42a5      	cmp	r5, r4
 80025b0:	f0c0 800a 	bcc.w	80025c8 <nl_func_acos_array_f32+0x2c>
 80025b4:	ed95 0a00 	vldr	s0, [r5]
 80025b8:	f008 fb00 	bl	800abbc <acosf>
 80025bc:	ed86 0a00 	vstr	s0, [r6]
 80025c0:	1f2d      	subs	r5, r5, #4
 80025c2:	1f36      	subs	r6, r6, #4
 80025c4:	42a5      	cmp	r5, r4
 80025c6:	d2f5      	bcs.n	80025b4 <nl_func_acos_array_f32+0x18>
 80025c8:	bd70      	pop	{r4, r5, r6, pc}
	...

080025cc <forward_acos>:
 80025cc:	b5f0      	push	{r4, r5, r6, r7, lr}
 80025ce:	b081      	sub	sp, #4
 80025d0:	6942      	ldr	r2, [r0, #20]
 80025d2:	8811      	ldrh	r1, [r2, #0]
 80025d4:	2900      	cmp	r1, #0
 80025d6:	bf1a      	itte	ne
 80025d8:	6850      	ldrne	r0, [r2, #4]
 80025da:	1d00      	addne	r0, r0, #4
 80025dc:	2004      	moveq	r0, #4
 80025de:	f04f 0501 	mov.w	r5, #1
 80025e2:	6800      	ldr	r0, [r0, #0]
 80025e4:	2800      	cmp	r0, #0
 80025e6:	bf14      	ite	ne
 80025e8:	6803      	ldrne	r3, [r0, #0]
 80025ea:	2300      	moveq	r3, #0
 80025ec:	2902      	cmp	r1, #2
 80025ee:	bfa6      	itte	ge
 80025f0:	6850      	ldrge	r0, [r2, #4]
 80025f2:	3010      	addge	r0, #16
 80025f4:	2004      	movlt	r0, #4
 80025f6:	6800      	ldr	r0, [r0, #0]
 80025f8:	2800      	cmp	r0, #0
 80025fa:	bf19      	ittee	ne
 80025fc:	6800      	ldrne	r0, [r0, #0]
 80025fe:	f100 0418 	addne.w	r4, r0, #24
 8002602:	2100      	moveq	r1, #0
 8002604:	f101 0418 	addeq.w	r4, r1, #24
 8002608:	f103 0108 	add.w	r1, r3, #8
 800260c:	680a      	ldr	r2, [r1, #0]
 800260e:	0a12      	lsrs	r2, r2, #8
 8002610:	d01e      	beq.n	8002650 <forward_acos+0x84>
 8002612:	684e      	ldr	r6, [r1, #4]
 8002614:	eb06 0182 	add.w	r1, r6, r2, lsl #2
 8002618:	4610      	mov	r0, r2
 800261a:	1f0f      	subs	r7, r1, #4
 800261c:	f010 0103 	ands.w	r1, r0, #3
 8002620:	d006      	beq.n	8002630 <forward_acos+0x64>
 8002622:	1e52      	subs	r2, r2, #1
 8002624:	f857 c904 	ldr.w	ip, [r7], #-4
 8002628:	1e49      	subs	r1, r1, #1
 800262a:	fb0c f505 	mul.w	r5, ip, r5
 800262e:	d1f8      	bne.n	8002622 <forward_acos+0x56>
 8002630:	0880      	lsrs	r0, r0, #2
 8002632:	d00d      	beq.n	8002650 <forward_acos+0x84>
 8002634:	eb06 0182 	add.w	r1, r6, r2, lsl #2
 8002638:	3910      	subs	r1, #16
 800263a:	68ca      	ldr	r2, [r1, #12]
 800263c:	688e      	ldr	r6, [r1, #8]
 800263e:	684f      	ldr	r7, [r1, #4]
 8002640:	4372      	muls	r2, r6
 8002642:	f851 6910 	ldr.w	r6, [r1], #-16
 8002646:	437a      	muls	r2, r7
 8002648:	4372      	muls	r2, r6
 800264a:	4355      	muls	r5, r2
 800264c:	1e40      	subs	r0, r0, #1
 800264e:	d1f4      	bne.n	800263a <forward_acos+0x6e>
 8002650:	6998      	ldr	r0, [r3, #24]
 8002652:	6886      	ldr	r6, [r0, #8]
 8002654:	6821      	ldr	r1, [r4, #0]
 8002656:	eb06 0085 	add.w	r0, r6, r5, lsl #2
 800265a:	1f07      	subs	r7, r0, #4
 800265c:	6888      	ldr	r0, [r1, #8]
 800265e:	eb00 0285 	add.w	r2, r0, r5, lsl #2
 8002662:	1f14      	subs	r4, r2, #4
 8002664:	42b7      	cmp	r7, r6
 8002666:	d309      	bcc.n	800267c <forward_acos+0xb0>
 8002668:	ed97 0a00 	vldr	s0, [r7]
 800266c:	f008 faa6 	bl	800abbc <acosf>
 8002670:	ed84 0a00 	vstr	s0, [r4]
 8002674:	1f3f      	subs	r7, r7, #4
 8002676:	1f24      	subs	r4, r4, #4
 8002678:	42b7      	cmp	r7, r6
 800267a:	d2f5      	bcs.n	8002668 <forward_acos+0x9c>
 800267c:	b001      	add	sp, #4
 800267e:	bdf0      	pop	{r4, r5, r6, r7, pc}

08002680 <nl_func_acosh_array_f32>:
 8002680:	b570      	push	{r4, r5, r6, lr}
 8002682:	688c      	ldr	r4, [r1, #8]
 8002684:	6880      	ldr	r0, [r0, #8]
 8002686:	eb04 0182 	add.w	r1, r4, r2, lsl #2
 800268a:	1f0d      	subs	r5, r1, #4
 800268c:	eb00 0182 	add.w	r1, r0, r2, lsl #2
 8002690:	1f0e      	subs	r6, r1, #4
 8002692:	42a5      	cmp	r5, r4
 8002694:	f0c0 800a 	bcc.w	80026ac <nl_func_acosh_array_f32+0x2c>
 8002698:	ed95 0a00 	vldr	s0, [r5]
 800269c:	f008 fae6 	bl	800ac6c <acoshf>
 80026a0:	ed86 0a00 	vstr	s0, [r6]
 80026a4:	1f2d      	subs	r5, r5, #4
 80026a6:	1f36      	subs	r6, r6, #4
 80026a8:	42a5      	cmp	r5, r4
 80026aa:	d2f5      	bcs.n	8002698 <nl_func_acosh_array_f32+0x18>
 80026ac:	bd70      	pop	{r4, r5, r6, pc}
	...

080026b0 <forward_acosh>:
 80026b0:	b5f0      	push	{r4, r5, r6, r7, lr}
 80026b2:	b081      	sub	sp, #4
 80026b4:	6942      	ldr	r2, [r0, #20]
 80026b6:	8811      	ldrh	r1, [r2, #0]
 80026b8:	2900      	cmp	r1, #0
 80026ba:	bf1a      	itte	ne
 80026bc:	6850      	ldrne	r0, [r2, #4]
 80026be:	1d00      	addne	r0, r0, #4
 80026c0:	2004      	moveq	r0, #4
 80026c2:	f04f 0501 	mov.w	r5, #1
 80026c6:	6800      	ldr	r0, [r0, #0]
 80026c8:	2800      	cmp	r0, #0
 80026ca:	bf14      	ite	ne
 80026cc:	6803      	ldrne	r3, [r0, #0]
 80026ce:	2300      	moveq	r3, #0
 80026d0:	2902      	cmp	r1, #2
 80026d2:	bfa6      	itte	ge
 80026d4:	6850      	ldrge	r0, [r2, #4]
 80026d6:	3010      	addge	r0, #16
 80026d8:	2004      	movlt	r0, #4
 80026da:	6800      	ldr	r0, [r0, #0]
 80026dc:	2800      	cmp	r0, #0
 80026de:	bf19      	ittee	ne
 80026e0:	6800      	ldrne	r0, [r0, #0]
 80026e2:	f100 0418 	addne.w	r4, r0, #24
 80026e6:	2100      	moveq	r1, #0
 80026e8:	f101 0418 	addeq.w	r4, r1, #24
 80026ec:	f103 0108 	add.w	r1, r3, #8
 80026f0:	680a      	ldr	r2, [r1, #0]
 80026f2:	0a12      	lsrs	r2, r2, #8
 80026f4:	d01e      	beq.n	8002734 <forward_acosh+0x84>
 80026f6:	684e      	ldr	r6, [r1, #4]
 80026f8:	eb06 0182 	add.w	r1, r6, r2, lsl #2
 80026fc:	4610      	mov	r0, r2
 80026fe:	1f0f      	subs	r7, r1, #4
 8002700:	f010 0103 	ands.w	r1, r0, #3
 8002704:	d006      	beq.n	8002714 <forward_acosh+0x64>
 8002706:	1e52      	subs	r2, r2, #1
 8002708:	f857 c904 	ldr.w	ip, [r7], #-4
 800270c:	1e49      	subs	r1, r1, #1
 800270e:	fb0c f505 	mul.w	r5, ip, r5
 8002712:	d1f8      	bne.n	8002706 <forward_acosh+0x56>
 8002714:	0880      	lsrs	r0, r0, #2
 8002716:	d00d      	beq.n	8002734 <forward_acosh+0x84>
 8002718:	eb06 0182 	add.w	r1, r6, r2, lsl #2
 800271c:	3910      	subs	r1, #16
 800271e:	68ca      	ldr	r2, [r1, #12]
 8002720:	688e      	ldr	r6, [r1, #8]
 8002722:	684f      	ldr	r7, [r1, #4]
 8002724:	4372      	muls	r2, r6
 8002726:	f851 6910 	ldr.w	r6, [r1], #-16
 800272a:	437a      	muls	r2, r7
 800272c:	4372      	muls	r2, r6
 800272e:	4355      	muls	r5, r2
 8002730:	1e40      	subs	r0, r0, #1
 8002732:	d1f4      	bne.n	800271e <forward_acosh+0x6e>
 8002734:	6998      	ldr	r0, [r3, #24]
 8002736:	6886      	ldr	r6, [r0, #8]
 8002738:	6821      	ldr	r1, [r4, #0]
 800273a:	eb06 0085 	add.w	r0, r6, r5, lsl #2
 800273e:	1f07      	subs	r7, r0, #4
 8002740:	6888      	ldr	r0, [r1, #8]
 8002742:	eb00 0285 	add.w	r2, r0, r5, lsl #2
 8002746:	1f14      	subs	r4, r2, #4
 8002748:	42b7      	cmp	r7, r6
 800274a:	d309      	bcc.n	8002760 <forward_acosh+0xb0>
 800274c:	ed97 0a00 	vldr	s0, [r7]
 8002750:	f008 fa8c 	bl	800ac6c <acoshf>
 8002754:	ed84 0a00 	vstr	s0, [r4]
 8002758:	1f3f      	subs	r7, r7, #4
 800275a:	1f24      	subs	r4, r4, #4
 800275c:	42b7      	cmp	r7, r6
 800275e:	d2f5      	bcs.n	800274c <forward_acosh+0x9c>
 8002760:	b001      	add	sp, #4
 8002762:	bdf0      	pop	{r4, r5, r6, r7, pc}

08002764 <nl_func_asin_array_f32>:
 8002764:	b570      	push	{r4, r5, r6, lr}
 8002766:	688c      	ldr	r4, [r1, #8]
 8002768:	6880      	ldr	r0, [r0, #8]
 800276a:	eb04 0182 	add.w	r1, r4, r2, lsl #2
 800276e:	1f0d      	subs	r5, r1, #4
 8002770:	eb00 0182 	add.w	r1, r0, r2, lsl #2
 8002774:	1f0e      	subs	r6, r1, #4
 8002776:	42a5      	cmp	r5, r4
 8002778:	f0c0 800a 	bcc.w	8002790 <nl_func_asin_array_f32+0x2c>
 800277c:	ed95 0a00 	vldr	s0, [r5]
 8002780:	f008 fac4 	bl	800ad0c <asinf>
 8002784:	ed86 0a00 	vstr	s0, [r6]
 8002788:	1f2d      	subs	r5, r5, #4
 800278a:	1f36      	subs	r6, r6, #4
 800278c:	42a5      	cmp	r5, r4
 800278e:	d2f5      	bcs.n	800277c <nl_func_asin_array_f32+0x18>
 8002790:	bd70      	pop	{r4, r5, r6, pc}
	...

08002794 <forward_asin>:
 8002794:	b5f0      	push	{r4, r5, r6, r7, lr}
 8002796:	b081      	sub	sp, #4
 8002798:	6942      	ldr	r2, [r0, #20]
 800279a:	8811      	ldrh	r1, [r2, #0]
 800279c:	2900      	cmp	r1, #0
 800279e:	bf1a      	itte	ne
 80027a0:	6850      	ldrne	r0, [r2, #4]
 80027a2:	1d00      	addne	r0, r0, #4
 80027a4:	2004      	moveq	r0, #4
 80027a6:	f04f 0501 	mov.w	r5, #1
 80027aa:	6800      	ldr	r0, [r0, #0]
 80027ac:	2800      	cmp	r0, #0
 80027ae:	bf14      	ite	ne
 80027b0:	6803      	ldrne	r3, [r0, #0]
 80027b2:	2300      	moveq	r3, #0
 80027b4:	2902      	cmp	r1, #2
 80027b6:	bfa6      	itte	ge
 80027b8:	6850      	ldrge	r0, [r2, #4]
 80027ba:	3010      	addge	r0, #16
 80027bc:	2004      	movlt	r0, #4
 80027be:	6800      	ldr	r0, [r0, #0]
 80027c0:	2800      	cmp	r0, #0
 80027c2:	bf19      	ittee	ne
 80027c4:	6800      	ldrne	r0, [r0, #0]
 80027c6:	f100 0418 	addne.w	r4, r0, #24
 80027ca:	2100      	moveq	r1, #0
 80027cc:	f101 0418 	addeq.w	r4, r1, #24
 80027d0:	f103 0108 	add.w	r1, r3, #8
 80027d4:	680a      	ldr	r2, [r1, #0]
 80027d6:	0a12      	lsrs	r2, r2, #8
 80027d8:	d01e      	beq.n	8002818 <forward_asin+0x84>
 80027da:	684e      	ldr	r6, [r1, #4]
 80027dc:	eb06 0182 	add.w	r1, r6, r2, lsl #2
 80027e0:	4610      	mov	r0, r2
 80027e2:	1f0f      	subs	r7, r1, #4
 80027e4:	f010 0103 	ands.w	r1, r0, #3
 80027e8:	d006      	beq.n	80027f8 <forward_asin+0x64>
 80027ea:	1e52      	subs	r2, r2, #1
 80027ec:	f857 c904 	ldr.w	ip, [r7], #-4
 80027f0:	1e49      	subs	r1, r1, #1
 80027f2:	fb0c f505 	mul.w	r5, ip, r5
 80027f6:	d1f8      	bne.n	80027ea <forward_asin+0x56>
 80027f8:	0880      	lsrs	r0, r0, #2
 80027fa:	d00d      	beq.n	8002818 <forward_asin+0x84>
 80027fc:	eb06 0182 	add.w	r1, r6, r2, lsl #2
 8002800:	3910      	subs	r1, #16
 8002802:	68ca      	ldr	r2, [r1, #12]
 8002804:	688e      	ldr	r6, [r1, #8]
 8002806:	684f      	ldr	r7, [r1, #4]
 8002808:	4372      	muls	r2, r6
 800280a:	f851 6910 	ldr.w	r6, [r1], #-16
 800280e:	437a      	muls	r2, r7
 8002810:	4372      	muls	r2, r6
 8002812:	4355      	muls	r5, r2
 8002814:	1e40      	subs	r0, r0, #1
 8002816:	d1f4      	bne.n	8002802 <forward_asin+0x6e>
 8002818:	6998      	ldr	r0, [r3, #24]
 800281a:	6886      	ldr	r6, [r0, #8]
 800281c:	6821      	ldr	r1, [r4, #0]
 800281e:	eb06 0085 	add.w	r0, r6, r5, lsl #2
 8002822:	1f07      	subs	r7, r0, #4
 8002824:	6888      	ldr	r0, [r1, #8]
 8002826:	eb00 0285 	add.w	r2, r0, r5, lsl #2
 800282a:	1f14      	subs	r4, r2, #4
 800282c:	42b7      	cmp	r7, r6
 800282e:	d309      	bcc.n	8002844 <forward_asin+0xb0>
 8002830:	ed97 0a00 	vldr	s0, [r7]
 8002834:	f008 fa6a 	bl	800ad0c <asinf>
 8002838:	ed84 0a00 	vstr	s0, [r4]
 800283c:	1f3f      	subs	r7, r7, #4
 800283e:	1f24      	subs	r4, r4, #4
 8002840:	42b7      	cmp	r7, r6
 8002842:	d2f5      	bcs.n	8002830 <forward_asin+0x9c>
 8002844:	b001      	add	sp, #4
 8002846:	bdf0      	pop	{r4, r5, r6, r7, pc}

08002848 <nl_func_asinh_array_f32>:
 8002848:	b570      	push	{r4, r5, r6, lr}
 800284a:	688c      	ldr	r4, [r1, #8]
 800284c:	6880      	ldr	r0, [r0, #8]
 800284e:	eb04 0182 	add.w	r1, r4, r2, lsl #2
 8002852:	1f0d      	subs	r5, r1, #4
 8002854:	eb00 0182 	add.w	r1, r0, r2, lsl #2
 8002858:	1f0e      	subs	r6, r1, #4
 800285a:	42a5      	cmp	r5, r4
 800285c:	f0c0 800a 	bcc.w	8002874 <nl_func_asinh_array_f32+0x2c>
 8002860:	ed95 0a00 	vldr	s0, [r5]
 8002864:	f007 fbda 	bl	800a01c <asinhf>
 8002868:	ed86 0a00 	vstr	s0, [r6]
 800286c:	1f2d      	subs	r5, r5, #4
 800286e:	1f36      	subs	r6, r6, #4
 8002870:	42a5      	cmp	r5, r4
 8002872:	d2f5      	bcs.n	8002860 <nl_func_asinh_array_f32+0x18>
 8002874:	bd70      	pop	{r4, r5, r6, pc}
	...

08002878 <forward_asinh>:
 8002878:	b5f0      	push	{r4, r5, r6, r7, lr}
 800287a:	b081      	sub	sp, #4
 800287c:	6942      	ldr	r2, [r0, #20]
 800287e:	8811      	ldrh	r1, [r2, #0]
 8002880:	2900      	cmp	r1, #0
 8002882:	bf1a      	itte	ne
 8002884:	6850      	ldrne	r0, [r2, #4]
 8002886:	1d00      	addne	r0, r0, #4
 8002888:	2004      	moveq	r0, #4
 800288a:	f04f 0501 	mov.w	r5, #1
 800288e:	6800      	ldr	r0, [r0, #0]
 8002890:	2800      	cmp	r0, #0
 8002892:	bf14      	ite	ne
 8002894:	6803      	ldrne	r3, [r0, #0]
 8002896:	2300      	moveq	r3, #0
 8002898:	2902      	cmp	r1, #2
 800289a:	bfa6      	itte	ge
 800289c:	6850      	ldrge	r0, [r2, #4]
 800289e:	3010      	addge	r0, #16
 80028a0:	2004      	movlt	r0, #4
 80028a2:	6800      	ldr	r0, [r0, #0]
 80028a4:	2800      	cmp	r0, #0
 80028a6:	bf19      	ittee	ne
 80028a8:	6800      	ldrne	r0, [r0, #0]
 80028aa:	f100 0418 	addne.w	r4, r0, #24
 80028ae:	2100      	moveq	r1, #0
 80028b0:	f101 0418 	addeq.w	r4, r1, #24
 80028b4:	f103 0108 	add.w	r1, r3, #8
 80028b8:	680a      	ldr	r2, [r1, #0]
 80028ba:	0a12      	lsrs	r2, r2, #8
 80028bc:	d01e      	beq.n	80028fc <forward_asinh+0x84>
 80028be:	684e      	ldr	r6, [r1, #4]
 80028c0:	eb06 0182 	add.w	r1, r6, r2, lsl #2
 80028c4:	4610      	mov	r0, r2
 80028c6:	1f0f      	subs	r7, r1, #4
 80028c8:	f010 0103 	ands.w	r1, r0, #3
 80028cc:	d006      	beq.n	80028dc <forward_asinh+0x64>
 80028ce:	1e52      	subs	r2, r2, #1
 80028d0:	f857 c904 	ldr.w	ip, [r7], #-4
 80028d4:	1e49      	subs	r1, r1, #1
 80028d6:	fb0c f505 	mul.w	r5, ip, r5
 80028da:	d1f8      	bne.n	80028ce <forward_asinh+0x56>
 80028dc:	0880      	lsrs	r0, r0, #2
 80028de:	d00d      	beq.n	80028fc <forward_asinh+0x84>
 80028e0:	eb06 0182 	add.w	r1, r6, r2, lsl #2
 80028e4:	3910      	subs	r1, #16
 80028e6:	68ca      	ldr	r2, [r1, #12]
 80028e8:	688e      	ldr	r6, [r1, #8]
 80028ea:	684f      	ldr	r7, [r1, #4]
 80028ec:	4372      	muls	r2, r6
 80028ee:	f851 6910 	ldr.w	r6, [r1], #-16
 80028f2:	437a      	muls	r2, r7
 80028f4:	4372      	muls	r2, r6
 80028f6:	4355      	muls	r5, r2
 80028f8:	1e40      	subs	r0, r0, #1
 80028fa:	d1f4      	bne.n	80028e6 <forward_asinh+0x6e>
 80028fc:	6998      	ldr	r0, [r3, #24]
 80028fe:	6886      	ldr	r6, [r0, #8]
 8002900:	6821      	ldr	r1, [r4, #0]
 8002902:	eb06 0085 	add.w	r0, r6, r5, lsl #2
 8002906:	1f07      	subs	r7, r0, #4
 8002908:	6888      	ldr	r0, [r1, #8]
 800290a:	eb00 0285 	add.w	r2, r0, r5, lsl #2
 800290e:	1f14      	subs	r4, r2, #4
 8002910:	42b7      	cmp	r7, r6
 8002912:	d309      	bcc.n	8002928 <forward_asinh+0xb0>
 8002914:	ed97 0a00 	vldr	s0, [r7]
 8002918:	f007 fb80 	bl	800a01c <asinhf>
 800291c:	ed84 0a00 	vstr	s0, [r4]
 8002920:	1f3f      	subs	r7, r7, #4
 8002922:	1f24      	subs	r4, r4, #4
 8002924:	42b7      	cmp	r7, r6
 8002926:	d2f5      	bcs.n	8002914 <forward_asinh+0x9c>
 8002928:	b001      	add	sp, #4
 800292a:	bdf0      	pop	{r4, r5, r6, r7, pc}

0800292c <nl_func_atan_array_f32>:
 800292c:	b570      	push	{r4, r5, r6, lr}
 800292e:	688c      	ldr	r4, [r1, #8]
 8002930:	6880      	ldr	r0, [r0, #8]
 8002932:	eb04 0182 	add.w	r1, r4, r2, lsl #2
 8002936:	1f0d      	subs	r5, r1, #4
 8002938:	eb00 0182 	add.w	r1, r0, r2, lsl #2
 800293c:	1f0e      	subs	r6, r1, #4
 800293e:	42a5      	cmp	r5, r4
 8002940:	f0c0 800a 	bcc.w	8002958 <nl_func_atan_array_f32+0x2c>
 8002944:	ed95 0a00 	vldr	s0, [r5]
 8002948:	f007 fbd0 	bl	800a0ec <atanf>
 800294c:	ed86 0a00 	vstr	s0, [r6]
 8002950:	1f2d      	subs	r5, r5, #4
 8002952:	1f36      	subs	r6, r6, #4
 8002954:	42a5      	cmp	r5, r4
 8002956:	d2f5      	bcs.n	8002944 <nl_func_atan_array_f32+0x18>
 8002958:	bd70      	pop	{r4, r5, r6, pc}
	...

0800295c <forward_atan>:
 800295c:	b5f0      	push	{r4, r5, r6, r7, lr}
 800295e:	b081      	sub	sp, #4
 8002960:	6942      	ldr	r2, [r0, #20]
 8002962:	8811      	ldrh	r1, [r2, #0]
 8002964:	2900      	cmp	r1, #0
 8002966:	bf1a      	itte	ne
 8002968:	6850      	ldrne	r0, [r2, #4]
 800296a:	1d00      	addne	r0, r0, #4
 800296c:	2004      	moveq	r0, #4
 800296e:	f04f 0501 	mov.w	r5, #1
 8002972:	6800      	ldr	r0, [r0, #0]
 8002974:	2800      	cmp	r0, #0
 8002976:	bf14      	ite	ne
 8002978:	6803      	ldrne	r3, [r0, #0]
 800297a:	2300      	moveq	r3, #0
 800297c:	2902      	cmp	r1, #2
 800297e:	bfa6      	itte	ge
 8002980:	6850      	ldrge	r0, [r2, #4]
 8002982:	3010      	addge	r0, #16
 8002984:	2004      	movlt	r0, #4
 8002986:	6800      	ldr	r0, [r0, #0]
 8002988:	2800      	cmp	r0, #0
 800298a:	bf19      	ittee	ne
 800298c:	6800      	ldrne	r0, [r0, #0]
 800298e:	f100 0418 	addne.w	r4, r0, #24
 8002992:	2100      	moveq	r1, #0
 8002994:	f101 0418 	addeq.w	r4, r1, #24
 8002998:	f103 0108 	add.w	r1, r3, #8
 800299c:	680a      	ldr	r2, [r1, #0]
 800299e:	0a12      	lsrs	r2, r2, #8
 80029a0:	d01e      	beq.n	80029e0 <forward_atan+0x84>
 80029a2:	684e      	ldr	r6, [r1, #4]
 80029a4:	eb06 0182 	add.w	r1, r6, r2, lsl #2
 80029a8:	4610      	mov	r0, r2
 80029aa:	1f0f      	subs	r7, r1, #4
 80029ac:	f010 0103 	ands.w	r1, r0, #3
 80029b0:	d006      	beq.n	80029c0 <forward_atan+0x64>
 80029b2:	1e52      	subs	r2, r2, #1
 80029b4:	f857 c904 	ldr.w	ip, [r7], #-4
 80029b8:	1e49      	subs	r1, r1, #1
 80029ba:	fb0c f505 	mul.w	r5, ip, r5
 80029be:	d1f8      	bne.n	80029b2 <forward_atan+0x56>
 80029c0:	0880      	lsrs	r0, r0, #2
 80029c2:	d00d      	beq.n	80029e0 <forward_atan+0x84>
 80029c4:	eb06 0182 	add.w	r1, r6, r2, lsl #2
 80029c8:	3910      	subs	r1, #16
 80029ca:	68ca      	ldr	r2, [r1, #12]
 80029cc:	688e      	ldr	r6, [r1, #8]
 80029ce:	684f      	ldr	r7, [r1, #4]
 80029d0:	4372      	muls	r2, r6
 80029d2:	f851 6910 	ldr.w	r6, [r1], #-16
 80029d6:	437a      	muls	r2, r7
 80029d8:	4372      	muls	r2, r6
 80029da:	4355      	muls	r5, r2
 80029dc:	1e40      	subs	r0, r0, #1
 80029de:	d1f4      	bne.n	80029ca <forward_atan+0x6e>
 80029e0:	6998      	ldr	r0, [r3, #24]
 80029e2:	6886      	ldr	r6, [r0, #8]
 80029e4:	6821      	ldr	r1, [r4, #0]
 80029e6:	eb06 0085 	add.w	r0, r6, r5, lsl #2
 80029ea:	1f07      	subs	r7, r0, #4
 80029ec:	6888      	ldr	r0, [r1, #8]
 80029ee:	eb00 0285 	add.w	r2, r0, r5, lsl #2
 80029f2:	1f14      	subs	r4, r2, #4
 80029f4:	42b7      	cmp	r7, r6
 80029f6:	d309      	bcc.n	8002a0c <forward_atan+0xb0>
 80029f8:	ed97 0a00 	vldr	s0, [r7]
 80029fc:	f007 fb76 	bl	800a0ec <atanf>
 8002a00:	ed84 0a00 	vstr	s0, [r4]
 8002a04:	1f3f      	subs	r7, r7, #4
 8002a06:	1f24      	subs	r4, r4, #4
 8002a08:	42b7      	cmp	r7, r6
 8002a0a:	d2f5      	bcs.n	80029f8 <forward_atan+0x9c>
 8002a0c:	b001      	add	sp, #4
 8002a0e:	bdf0      	pop	{r4, r5, r6, r7, pc}

08002a10 <nl_func_atanh_array_f32>:
 8002a10:	b570      	push	{r4, r5, r6, lr}
 8002a12:	688c      	ldr	r4, [r1, #8]
 8002a14:	6880      	ldr	r0, [r0, #8]
 8002a16:	eb04 0182 	add.w	r1, r4, r2, lsl #2
 8002a1a:	1f0d      	subs	r5, r1, #4
 8002a1c:	eb00 0182 	add.w	r1, r0, r2, lsl #2
 8002a20:	1f0e      	subs	r6, r1, #4
 8002a22:	42a5      	cmp	r5, r4
 8002a24:	f0c0 800a 	bcc.w	8002a3c <nl_func_atanh_array_f32+0x2c>
 8002a28:	ed95 0a00 	vldr	s0, [r5]
 8002a2c:	f008 f9c6 	bl	800adbc <atanhf>
 8002a30:	ed86 0a00 	vstr	s0, [r6]
 8002a34:	1f2d      	subs	r5, r5, #4
 8002a36:	1f36      	subs	r6, r6, #4
 8002a38:	42a5      	cmp	r5, r4
 8002a3a:	d2f5      	bcs.n	8002a28 <nl_func_atanh_array_f32+0x18>
 8002a3c:	bd70      	pop	{r4, r5, r6, pc}
	...

08002a40 <forward_atanh>:
 8002a40:	b5f0      	push	{r4, r5, r6, r7, lr}
 8002a42:	b081      	sub	sp, #4
 8002a44:	6942      	ldr	r2, [r0, #20]
 8002a46:	8811      	ldrh	r1, [r2, #0]
 8002a48:	2900      	cmp	r1, #0
 8002a4a:	bf1a      	itte	ne
 8002a4c:	6850      	ldrne	r0, [r2, #4]
 8002a4e:	1d00      	addne	r0, r0, #4
 8002a50:	2004      	moveq	r0, #4
 8002a52:	f04f 0501 	mov.w	r5, #1
 8002a56:	6800      	ldr	r0, [r0, #0]
 8002a58:	2800      	cmp	r0, #0
 8002a5a:	bf14      	ite	ne
 8002a5c:	6803      	ldrne	r3, [r0, #0]
 8002a5e:	2300      	moveq	r3, #0
 8002a60:	2902      	cmp	r1, #2
 8002a62:	bfa6      	itte	ge
 8002a64:	6850      	ldrge	r0, [r2, #4]
 8002a66:	3010      	addge	r0, #16
 8002a68:	2004      	movlt	r0, #4
 8002a6a:	6800      	ldr	r0, [r0, #0]
 8002a6c:	2800      	cmp	r0, #0
 8002a6e:	bf19      	ittee	ne
 8002a70:	6800      	ldrne	r0, [r0, #0]
 8002a72:	f100 0418 	addne.w	r4, r0, #24
 8002a76:	2100      	moveq	r1, #0
 8002a78:	f101 0418 	addeq.w	r4, r1, #24
 8002a7c:	f103 0108 	add.w	r1, r3, #8
 8002a80:	680a      	ldr	r2, [r1, #0]
 8002a82:	0a12      	lsrs	r2, r2, #8
 8002a84:	d01e      	beq.n	8002ac4 <forward_atanh+0x84>
 8002a86:	684e      	ldr	r6, [r1, #4]
 8002a88:	eb06 0182 	add.w	r1, r6, r2, lsl #2
 8002a8c:	4610      	mov	r0, r2
 8002a8e:	1f0f      	subs	r7, r1, #4
 8002a90:	f010 0103 	ands.w	r1, r0, #3
 8002a94:	d006      	beq.n	8002aa4 <forward_atanh+0x64>
 8002a96:	1e52      	subs	r2, r2, #1
 8002a98:	f857 c904 	ldr.w	ip, [r7], #-4
 8002a9c:	1e49      	subs	r1, r1, #1
 8002a9e:	fb0c f505 	mul.w	r5, ip, r5
 8002aa2:	d1f8      	bne.n	8002a96 <forward_atanh+0x56>
 8002aa4:	0880      	lsrs	r0, r0, #2
 8002aa6:	d00d      	beq.n	8002ac4 <forward_atanh+0x84>
 8002aa8:	eb06 0182 	add.w	r1, r6, r2, lsl #2
 8002aac:	3910      	subs	r1, #16
 8002aae:	68ca      	ldr	r2, [r1, #12]
 8002ab0:	688e      	ldr	r6, [r1, #8]
 8002ab2:	684f      	ldr	r7, [r1, #4]
 8002ab4:	4372      	muls	r2, r6
 8002ab6:	f851 6910 	ldr.w	r6, [r1], #-16
 8002aba:	437a      	muls	r2, r7
 8002abc:	4372      	muls	r2, r6
 8002abe:	4355      	muls	r5, r2
 8002ac0:	1e40      	subs	r0, r0, #1
 8002ac2:	d1f4      	bne.n	8002aae <forward_atanh+0x6e>
 8002ac4:	6998      	ldr	r0, [r3, #24]
 8002ac6:	6886      	ldr	r6, [r0, #8]
 8002ac8:	6821      	ldr	r1, [r4, #0]
 8002aca:	eb06 0085 	add.w	r0, r6, r5, lsl #2
 8002ace:	1f07      	subs	r7, r0, #4
 8002ad0:	6888      	ldr	r0, [r1, #8]
 8002ad2:	eb00 0285 	add.w	r2, r0, r5, lsl #2
 8002ad6:	1f14      	subs	r4, r2, #4
 8002ad8:	42b7      	cmp	r7, r6
 8002ada:	d309      	bcc.n	8002af0 <forward_atanh+0xb0>
 8002adc:	ed97 0a00 	vldr	s0, [r7]
 8002ae0:	f008 f96c 	bl	800adbc <atanhf>
 8002ae4:	ed84 0a00 	vstr	s0, [r4]
 8002ae8:	1f3f      	subs	r7, r7, #4
 8002aea:	1f24      	subs	r4, r4, #4
 8002aec:	42b7      	cmp	r7, r6
 8002aee:	d2f5      	bcs.n	8002adc <forward_atanh+0x9c>
 8002af0:	b001      	add	sp, #4
 8002af2:	bdf0      	pop	{r4, r5, r6, r7, pc}

08002af4 <nl_func_cos_array_f32>:
 8002af4:	b570      	push	{r4, r5, r6, lr}
 8002af6:	688c      	ldr	r4, [r1, #8]
 8002af8:	6880      	ldr	r0, [r0, #8]
 8002afa:	eb04 0182 	add.w	r1, r4, r2, lsl #2
 8002afe:	1f0d      	subs	r5, r1, #4
 8002b00:	eb00 0182 	add.w	r1, r0, r2, lsl #2
 8002b04:	1f0e      	subs	r6, r1, #4
 8002b06:	42a5      	cmp	r5, r4
 8002b08:	f0c0 800a 	bcc.w	8002b20 <nl_func_cos_array_f32+0x2c>
 8002b0c:	ed95 0a00 	vldr	s0, [r5]
 8002b10:	f007 fc00 	bl	800a314 <cosf>
 8002b14:	ed86 0a00 	vstr	s0, [r6]
 8002b18:	1f2d      	subs	r5, r5, #4
 8002b1a:	1f36      	subs	r6, r6, #4
 8002b1c:	42a5      	cmp	r5, r4
 8002b1e:	d2f5      	bcs.n	8002b0c <nl_func_cos_array_f32+0x18>
 8002b20:	bd70      	pop	{r4, r5, r6, pc}
	...

08002b24 <forward_cos>:
 8002b24:	b5f0      	push	{r4, r5, r6, r7, lr}
 8002b26:	b081      	sub	sp, #4
 8002b28:	6942      	ldr	r2, [r0, #20]
 8002b2a:	8811      	ldrh	r1, [r2, #0]
 8002b2c:	2900      	cmp	r1, #0
 8002b2e:	bf1a      	itte	ne
 8002b30:	6850      	ldrne	r0, [r2, #4]
 8002b32:	1d00      	addne	r0, r0, #4
 8002b34:	2004      	moveq	r0, #4
 8002b36:	f04f 0501 	mov.w	r5, #1
 8002b3a:	6800      	ldr	r0, [r0, #0]
 8002b3c:	2800      	cmp	r0, #0
 8002b3e:	bf14      	ite	ne
 8002b40:	6803      	ldrne	r3, [r0, #0]
 8002b42:	2300      	moveq	r3, #0
 8002b44:	2902      	cmp	r1, #2
 8002b46:	bfa6      	itte	ge
 8002b48:	6850      	ldrge	r0, [r2, #4]
 8002b4a:	3010      	addge	r0, #16
 8002b4c:	2004      	movlt	r0, #4
 8002b4e:	6800      	ldr	r0, [r0, #0]
 8002b50:	2800      	cmp	r0, #0
 8002b52:	bf19      	ittee	ne
 8002b54:	6800      	ldrne	r0, [r0, #0]
 8002b56:	f100 0418 	addne.w	r4, r0, #24
 8002b5a:	2100      	moveq	r1, #0
 8002b5c:	f101 0418 	addeq.w	r4, r1, #24
 8002b60:	f103 0108 	add.w	r1, r3, #8
 8002b64:	680a      	ldr	r2, [r1, #0]
 8002b66:	0a12      	lsrs	r2, r2, #8
 8002b68:	d01e      	beq.n	8002ba8 <forward_cos+0x84>
 8002b6a:	684e      	ldr	r6, [r1, #4]
 8002b6c:	eb06 0182 	add.w	r1, r6, r2, lsl #2
 8002b70:	4610      	mov	r0, r2
 8002b72:	1f0f      	subs	r7, r1, #4
 8002b74:	f010 0103 	ands.w	r1, r0, #3
 8002b78:	d006      	beq.n	8002b88 <forward_cos+0x64>
 8002b7a:	1e52      	subs	r2, r2, #1
 8002b7c:	f857 c904 	ldr.w	ip, [r7], #-4
 8002b80:	1e49      	subs	r1, r1, #1
 8002b82:	fb0c f505 	mul.w	r5, ip, r5
 8002b86:	d1f8      	bne.n	8002b7a <forward_cos+0x56>
 8002b88:	0880      	lsrs	r0, r0, #2
 8002b8a:	d00d      	beq.n	8002ba8 <forward_cos+0x84>
 8002b8c:	eb06 0182 	add.w	r1, r6, r2, lsl #2
 8002b90:	3910      	subs	r1, #16
 8002b92:	68ca      	ldr	r2, [r1, #12]
 8002b94:	688e      	ldr	r6, [r1, #8]
 8002b96:	684f      	ldr	r7, [r1, #4]
 8002b98:	4372      	muls	r2, r6
 8002b9a:	f851 6910 	ldr.w	r6, [r1], #-16
 8002b9e:	437a      	muls	r2, r7
 8002ba0:	4372      	muls	r2, r6
 8002ba2:	4355      	muls	r5, r2
 8002ba4:	1e40      	subs	r0, r0, #1
 8002ba6:	d1f4      	bne.n	8002b92 <forward_cos+0x6e>
 8002ba8:	6998      	ldr	r0, [r3, #24]
 8002baa:	6886      	ldr	r6, [r0, #8]
 8002bac:	6821      	ldr	r1, [r4, #0]
 8002bae:	eb06 0085 	add.w	r0, r6, r5, lsl #2
 8002bb2:	1f07      	subs	r7, r0, #4
 8002bb4:	6888      	ldr	r0, [r1, #8]
 8002bb6:	eb00 0285 	add.w	r2, r0, r5, lsl #2
 8002bba:	1f14      	subs	r4, r2, #4
 8002bbc:	42b7      	cmp	r7, r6
 8002bbe:	d309      	bcc.n	8002bd4 <forward_cos+0xb0>
 8002bc0:	ed97 0a00 	vldr	s0, [r7]
 8002bc4:	f007 fba6 	bl	800a314 <cosf>
 8002bc8:	ed84 0a00 	vstr	s0, [r4]
 8002bcc:	1f3f      	subs	r7, r7, #4
 8002bce:	1f24      	subs	r4, r4, #4
 8002bd0:	42b7      	cmp	r7, r6
 8002bd2:	d2f5      	bcs.n	8002bc0 <forward_cos+0x9c>
 8002bd4:	b001      	add	sp, #4
 8002bd6:	bdf0      	pop	{r4, r5, r6, r7, pc}

08002bd8 <nl_func_cosh_array_f32>:
 8002bd8:	b570      	push	{r4, r5, r6, lr}
 8002bda:	688c      	ldr	r4, [r1, #8]
 8002bdc:	6880      	ldr	r0, [r0, #8]
 8002bde:	eb04 0182 	add.w	r1, r4, r2, lsl #2
 8002be2:	1f0d      	subs	r5, r1, #4
 8002be4:	eb00 0182 	add.w	r1, r0, r2, lsl #2
 8002be8:	1f0e      	subs	r6, r1, #4
 8002bea:	42a5      	cmp	r5, r4
 8002bec:	f0c0 800a 	bcc.w	8002c04 <nl_func_cosh_array_f32+0x2c>
 8002bf0:	ed95 0a00 	vldr	s0, [r5]
 8002bf4:	f008 f956 	bl	800aea4 <coshf>
 8002bf8:	ed86 0a00 	vstr	s0, [r6]
 8002bfc:	1f2d      	subs	r5, r5, #4
 8002bfe:	1f36      	subs	r6, r6, #4
 8002c00:	42a5      	cmp	r5, r4
 8002c02:	d2f5      	bcs.n	8002bf0 <nl_func_cosh_array_f32+0x18>
 8002c04:	bd70      	pop	{r4, r5, r6, pc}
	...

08002c08 <forward_cosh>:
 8002c08:	b5f0      	push	{r4, r5, r6, r7, lr}
 8002c0a:	b081      	sub	sp, #4
 8002c0c:	6942      	ldr	r2, [r0, #20]
 8002c0e:	8811      	ldrh	r1, [r2, #0]
 8002c10:	2900      	cmp	r1, #0
 8002c12:	bf1a      	itte	ne
 8002c14:	6850      	ldrne	r0, [r2, #4]
 8002c16:	1d00      	addne	r0, r0, #4
 8002c18:	2004      	moveq	r0, #4
 8002c1a:	f04f 0501 	mov.w	r5, #1
 8002c1e:	6800      	ldr	r0, [r0, #0]
 8002c20:	2800      	cmp	r0, #0
 8002c22:	bf14      	ite	ne
 8002c24:	6803      	ldrne	r3, [r0, #0]
 8002c26:	2300      	moveq	r3, #0
 8002c28:	2902      	cmp	r1, #2
 8002c2a:	bfa6      	itte	ge
 8002c2c:	6850      	ldrge	r0, [r2, #4]
 8002c2e:	3010      	addge	r0, #16
 8002c30:	2004      	movlt	r0, #4
 8002c32:	6800      	ldr	r0, [r0, #0]
 8002c34:	2800      	cmp	r0, #0
 8002c36:	bf19      	ittee	ne
 8002c38:	6800      	ldrne	r0, [r0, #0]
 8002c3a:	f100 0418 	addne.w	r4, r0, #24
 8002c3e:	2100      	moveq	r1, #0
 8002c40:	f101 0418 	addeq.w	r4, r1, #24
 8002c44:	f103 0108 	add.w	r1, r3, #8
 8002c48:	680a      	ldr	r2, [r1, #0]
 8002c4a:	0a12      	lsrs	r2, r2, #8
 8002c4c:	d01e      	beq.n	8002c8c <forward_cosh+0x84>
 8002c4e:	684e      	ldr	r6, [r1, #4]
 8002c50:	eb06 0182 	add.w	r1, r6, r2, lsl #2
 8002c54:	4610      	mov	r0, r2
 8002c56:	1f0f      	subs	r7, r1, #4
 8002c58:	f010 0103 	ands.w	r1, r0, #3
 8002c5c:	d006      	beq.n	8002c6c <forward_cosh+0x64>
 8002c5e:	1e52      	subs	r2, r2, #1
 8002c60:	f857 c904 	ldr.w	ip, [r7], #-4
 8002c64:	1e49      	subs	r1, r1, #1
 8002c66:	fb0c f505 	mul.w	r5, ip, r5
 8002c6a:	d1f8      	bne.n	8002c5e <forward_cosh+0x56>
 8002c6c:	0880      	lsrs	r0, r0, #2
 8002c6e:	d00d      	beq.n	8002c8c <forward_cosh+0x84>
 8002c70:	eb06 0182 	add.w	r1, r6, r2, lsl #2
 8002c74:	3910      	subs	r1, #16
 8002c76:	68ca      	ldr	r2, [r1, #12]
 8002c78:	688e      	ldr	r6, [r1, #8]
 8002c7a:	684f      	ldr	r7, [r1, #4]
 8002c7c:	4372      	muls	r2, r6
 8002c7e:	f851 6910 	ldr.w	r6, [r1], #-16
 8002c82:	437a      	muls	r2, r7
 8002c84:	4372      	muls	r2, r6
 8002c86:	4355      	muls	r5, r2
 8002c88:	1e40      	subs	r0, r0, #1
 8002c8a:	d1f4      	bne.n	8002c76 <forward_cosh+0x6e>
 8002c8c:	6998      	ldr	r0, [r3, #24]
 8002c8e:	6886      	ldr	r6, [r0, #8]
 8002c90:	6821      	ldr	r1, [r4, #0]
 8002c92:	eb06 0085 	add.w	r0, r6, r5, lsl #2
 8002c96:	1f07      	subs	r7, r0, #4
 8002c98:	6888      	ldr	r0, [r1, #8]
 8002c9a:	eb00 0285 	add.w	r2, r0, r5, lsl #2
 8002c9e:	1f14      	subs	r4, r2, #4
 8002ca0:	42b7      	cmp	r7, r6
 8002ca2:	d309      	bcc.n	8002cb8 <forward_cosh+0xb0>
 8002ca4:	ed97 0a00 	vldr	s0, [r7]
 8002ca8:	f008 f8fc 	bl	800aea4 <coshf>
 8002cac:	ed84 0a00 	vstr	s0, [r4]
 8002cb0:	1f3f      	subs	r7, r7, #4
 8002cb2:	1f24      	subs	r4, r4, #4
 8002cb4:	42b7      	cmp	r7, r6
 8002cb6:	d2f5      	bcs.n	8002ca4 <forward_cosh+0x9c>
 8002cb8:	b001      	add	sp, #4
 8002cba:	bdf0      	pop	{r4, r5, r6, r7, pc}

08002cbc <nl_func_erf_array_f32>:
 8002cbc:	b570      	push	{r4, r5, r6, lr}
 8002cbe:	688c      	ldr	r4, [r1, #8]
 8002cc0:	6880      	ldr	r0, [r0, #8]
 8002cc2:	eb04 0182 	add.w	r1, r4, r2, lsl #2
 8002cc6:	1f0d      	subs	r5, r1, #4
 8002cc8:	eb00 0182 	add.w	r1, r0, r2, lsl #2
 8002ccc:	1f0e      	subs	r6, r1, #4
 8002cce:	42a5      	cmp	r5, r4
 8002cd0:	f0c0 800a 	bcc.w	8002ce8 <nl_func_erf_array_f32+0x2c>
 8002cd4:	ed95 0a00 	vldr	s0, [r5]
 8002cd8:	f007 fb5c 	bl	800a394 <erff>
 8002cdc:	ed86 0a00 	vstr	s0, [r6]
 8002ce0:	1f2d      	subs	r5, r5, #4
 8002ce2:	1f36      	subs	r6, r6, #4
 8002ce4:	42a5      	cmp	r5, r4
 8002ce6:	d2f5      	bcs.n	8002cd4 <nl_func_erf_array_f32+0x18>
 8002ce8:	bd70      	pop	{r4, r5, r6, pc}
	...

08002cec <forward_erf>:
 8002cec:	b5f0      	push	{r4, r5, r6, r7, lr}
 8002cee:	b081      	sub	sp, #4
 8002cf0:	6942      	ldr	r2, [r0, #20]
 8002cf2:	8811      	ldrh	r1, [r2, #0]
 8002cf4:	2900      	cmp	r1, #0
 8002cf6:	bf1a      	itte	ne
 8002cf8:	6850      	ldrne	r0, [r2, #4]
 8002cfa:	1d00      	addne	r0, r0, #4
 8002cfc:	2004      	moveq	r0, #4
 8002cfe:	f04f 0501 	mov.w	r5, #1
 8002d02:	6800      	ldr	r0, [r0, #0]
 8002d04:	2800      	cmp	r0, #0
 8002d06:	bf14      	ite	ne
 8002d08:	6803      	ldrne	r3, [r0, #0]
 8002d0a:	2300      	moveq	r3, #0
 8002d0c:	2902      	cmp	r1, #2
 8002d0e:	bfa6      	itte	ge
 8002d10:	6850      	ldrge	r0, [r2, #4]
 8002d12:	3010      	addge	r0, #16
 8002d14:	2004      	movlt	r0, #4
 8002d16:	6800      	ldr	r0, [r0, #0]
 8002d18:	2800      	cmp	r0, #0
 8002d1a:	bf19      	ittee	ne
 8002d1c:	6800      	ldrne	r0, [r0, #0]
 8002d1e:	f100 0418 	addne.w	r4, r0, #24
 8002d22:	2100      	moveq	r1, #0
 8002d24:	f101 0418 	addeq.w	r4, r1, #24
 8002d28:	f103 0108 	add.w	r1, r3, #8
 8002d2c:	680a      	ldr	r2, [r1, #0]
 8002d2e:	0a12      	lsrs	r2, r2, #8
 8002d30:	d01e      	beq.n	8002d70 <forward_erf+0x84>
 8002d32:	684e      	ldr	r6, [r1, #4]
 8002d34:	eb06 0182 	add.w	r1, r6, r2, lsl #2
 8002d38:	4610      	mov	r0, r2
 8002d3a:	1f0f      	subs	r7, r1, #4
 8002d3c:	f010 0103 	ands.w	r1, r0, #3
 8002d40:	d006      	beq.n	8002d50 <forward_erf+0x64>
 8002d42:	1e52      	subs	r2, r2, #1
 8002d44:	f857 c904 	ldr.w	ip, [r7], #-4
 8002d48:	1e49      	subs	r1, r1, #1
 8002d4a:	fb0c f505 	mul.w	r5, ip, r5
 8002d4e:	d1f8      	bne.n	8002d42 <forward_erf+0x56>
 8002d50:	0880      	lsrs	r0, r0, #2
 8002d52:	d00d      	beq.n	8002d70 <forward_erf+0x84>
 8002d54:	eb06 0182 	add.w	r1, r6, r2, lsl #2
 8002d58:	3910      	subs	r1, #16
 8002d5a:	68ca      	ldr	r2, [r1, #12]
 8002d5c:	688e      	ldr	r6, [r1, #8]
 8002d5e:	684f      	ldr	r7, [r1, #4]
 8002d60:	4372      	muls	r2, r6
 8002d62:	f851 6910 	ldr.w	r6, [r1], #-16
 8002d66:	437a      	muls	r2, r7
 8002d68:	4372      	muls	r2, r6
 8002d6a:	4355      	muls	r5, r2
 8002d6c:	1e40      	subs	r0, r0, #1
 8002d6e:	d1f4      	bne.n	8002d5a <forward_erf+0x6e>
 8002d70:	6998      	ldr	r0, [r3, #24]
 8002d72:	6886      	ldr	r6, [r0, #8]
 8002d74:	6821      	ldr	r1, [r4, #0]
 8002d76:	eb06 0085 	add.w	r0, r6, r5, lsl #2
 8002d7a:	1f07      	subs	r7, r0, #4
 8002d7c:	6888      	ldr	r0, [r1, #8]
 8002d7e:	eb00 0285 	add.w	r2, r0, r5, lsl #2
 8002d82:	1f14      	subs	r4, r2, #4
 8002d84:	42b7      	cmp	r7, r6
 8002d86:	d309      	bcc.n	8002d9c <forward_erf+0xb0>
 8002d88:	ed97 0a00 	vldr	s0, [r7]
 8002d8c:	f007 fb02 	bl	800a394 <erff>
 8002d90:	ed84 0a00 	vstr	s0, [r4]
 8002d94:	1f3f      	subs	r7, r7, #4
 8002d96:	1f24      	subs	r4, r4, #4
 8002d98:	42b7      	cmp	r7, r6
 8002d9a:	d2f5      	bcs.n	8002d88 <forward_erf+0x9c>
 8002d9c:	b001      	add	sp, #4
 8002d9e:	bdf0      	pop	{r4, r5, r6, r7, pc}

08002da0 <nl_func_log_array_f32>:
 8002da0:	b570      	push	{r4, r5, r6, lr}
 8002da2:	688c      	ldr	r4, [r1, #8]
 8002da4:	6880      	ldr	r0, [r0, #8]
 8002da6:	eb04 0182 	add.w	r1, r4, r2, lsl #2
 8002daa:	1f0d      	subs	r5, r1, #4
 8002dac:	eb00 0182 	add.w	r1, r0, r2, lsl #2
 8002db0:	1f0e      	subs	r6, r1, #4
 8002db2:	42a5      	cmp	r5, r4
 8002db4:	f0c0 800a 	bcc.w	8002dcc <nl_func_log_array_f32+0x2c>
 8002db8:	ed95 0a00 	vldr	s0, [r5]
 8002dbc:	f008 f9a8 	bl	800b110 <logf>
 8002dc0:	ed86 0a00 	vstr	s0, [r6]
 8002dc4:	1f2d      	subs	r5, r5, #4
 8002dc6:	1f36      	subs	r6, r6, #4
 8002dc8:	42a5      	cmp	r5, r4
 8002dca:	d2f5      	bcs.n	8002db8 <nl_func_log_array_f32+0x18>
 8002dcc:	bd70      	pop	{r4, r5, r6, pc}
	...

08002dd0 <forward_log>:
 8002dd0:	b5f0      	push	{r4, r5, r6, r7, lr}
 8002dd2:	b081      	sub	sp, #4
 8002dd4:	6942      	ldr	r2, [r0, #20]
 8002dd6:	8811      	ldrh	r1, [r2, #0]
 8002dd8:	2900      	cmp	r1, #0
 8002dda:	bf1a      	itte	ne
 8002ddc:	6850      	ldrne	r0, [r2, #4]
 8002dde:	1d00      	addne	r0, r0, #4
 8002de0:	2004      	moveq	r0, #4
 8002de2:	f04f 0501 	mov.w	r5, #1
 8002de6:	6800      	ldr	r0, [r0, #0]
 8002de8:	2800      	cmp	r0, #0
 8002dea:	bf14      	ite	ne
 8002dec:	6803      	ldrne	r3, [r0, #0]
 8002dee:	2300      	moveq	r3, #0
 8002df0:	2902      	cmp	r1, #2
 8002df2:	bfa6      	itte	ge
 8002df4:	6850      	ldrge	r0, [r2, #4]
 8002df6:	3010      	addge	r0, #16
 8002df8:	2004      	movlt	r0, #4
 8002dfa:	6800      	ldr	r0, [r0, #0]
 8002dfc:	2800      	cmp	r0, #0
 8002dfe:	bf19      	ittee	ne
 8002e00:	6800      	ldrne	r0, [r0, #0]
 8002e02:	f100 0418 	addne.w	r4, r0, #24
 8002e06:	2100      	moveq	r1, #0
 8002e08:	f101 0418 	addeq.w	r4, r1, #24
 8002e0c:	f103 0108 	add.w	r1, r3, #8
 8002e10:	680a      	ldr	r2, [r1, #0]
 8002e12:	0a12      	lsrs	r2, r2, #8
 8002e14:	d01e      	beq.n	8002e54 <forward_log+0x84>
 8002e16:	684e      	ldr	r6, [r1, #4]
 8002e18:	eb06 0182 	add.w	r1, r6, r2, lsl #2
 8002e1c:	4610      	mov	r0, r2
 8002e1e:	1f0f      	subs	r7, r1, #4
 8002e20:	f010 0103 	ands.w	r1, r0, #3
 8002e24:	d006      	beq.n	8002e34 <forward_log+0x64>
 8002e26:	1e52      	subs	r2, r2, #1
 8002e28:	f857 c904 	ldr.w	ip, [r7], #-4
 8002e2c:	1e49      	subs	r1, r1, #1
 8002e2e:	fb0c f505 	mul.w	r5, ip, r5
 8002e32:	d1f8      	bne.n	8002e26 <forward_log+0x56>
 8002e34:	0880      	lsrs	r0, r0, #2
 8002e36:	d00d      	beq.n	8002e54 <forward_log+0x84>
 8002e38:	eb06 0182 	add.w	r1, r6, r2, lsl #2
 8002e3c:	3910      	subs	r1, #16
 8002e3e:	68ca      	ldr	r2, [r1, #12]
 8002e40:	688e      	ldr	r6, [r1, #8]
 8002e42:	684f      	ldr	r7, [r1, #4]
 8002e44:	4372      	muls	r2, r6
 8002e46:	f851 6910 	ldr.w	r6, [r1], #-16
 8002e4a:	437a      	muls	r2, r7
 8002e4c:	4372      	muls	r2, r6
 8002e4e:	4355      	muls	r5, r2
 8002e50:	1e40      	subs	r0, r0, #1
 8002e52:	d1f4      	bne.n	8002e3e <forward_log+0x6e>
 8002e54:	6998      	ldr	r0, [r3, #24]
 8002e56:	6886      	ldr	r6, [r0, #8]
 8002e58:	6821      	ldr	r1, [r4, #0]
 8002e5a:	eb06 0085 	add.w	r0, r6, r5, lsl #2
 8002e5e:	1f07      	subs	r7, r0, #4
 8002e60:	6888      	ldr	r0, [r1, #8]
 8002e62:	eb00 0285 	add.w	r2, r0, r5, lsl #2
 8002e66:	1f14      	subs	r4, r2, #4
 8002e68:	42b7      	cmp	r7, r6
 8002e6a:	d309      	bcc.n	8002e80 <forward_log+0xb0>
 8002e6c:	ed97 0a00 	vldr	s0, [r7]
 8002e70:	f008 f94e 	bl	800b110 <logf>
 8002e74:	ed84 0a00 	vstr	s0, [r4]
 8002e78:	1f3f      	subs	r7, r7, #4
 8002e7a:	1f24      	subs	r4, r4, #4
 8002e7c:	42b7      	cmp	r7, r6
 8002e7e:	d2f5      	bcs.n	8002e6c <forward_log+0x9c>
 8002e80:	b001      	add	sp, #4
 8002e82:	bdf0      	pop	{r4, r5, r6, r7, pc}

08002e84 <nl_func_rsqrt_array_f32>:
 8002e84:	b570      	push	{r4, r5, r6, lr}
 8002e86:	460c      	mov	r4, r1
 8002e88:	6880      	ldr	r0, [r0, #8]
 8002e8a:	68a1      	ldr	r1, [r4, #8]
 8002e8c:	eb01 0382 	add.w	r3, r1, r2, lsl #2
 8002e90:	eb00 0282 	add.w	r2, r0, r2, lsl #2
 8002e94:	1f1d      	subs	r5, r3, #4
 8002e96:	1f16      	subs	r6, r2, #4
 8002e98:	428d      	cmp	r5, r1
 8002e9a:	d30e      	bcc.n	8002eba <nl_func_rsqrt_array_f32+0x36>
 8002e9c:	ed95 0a00 	vldr	s0, [r5]
 8002ea0:	f003 f930 	bl	8006104 <ai_math_sqrt>
 8002ea4:	eef7 0a00 	vmov.f32	s1, #112	; 0x3f800000  1.0
 8002ea8:	eec0 0a80 	vdiv.f32	s1, s1, s0
 8002eac:	edc6 0a00 	vstr	s1, [r6]
 8002eb0:	1f2d      	subs	r5, r5, #4
 8002eb2:	68a0      	ldr	r0, [r4, #8]
 8002eb4:	1f36      	subs	r6, r6, #4
 8002eb6:	4285      	cmp	r5, r0
 8002eb8:	d2f0      	bcs.n	8002e9c <nl_func_rsqrt_array_f32+0x18>
 8002eba:	bd70      	pop	{r4, r5, r6, pc}

08002ebc <forward_rsqrt>:
 8002ebc:	b5f0      	push	{r4, r5, r6, r7, lr}
 8002ebe:	b081      	sub	sp, #4
 8002ec0:	6942      	ldr	r2, [r0, #20]
 8002ec2:	8811      	ldrh	r1, [r2, #0]
 8002ec4:	2900      	cmp	r1, #0
 8002ec6:	bf1a      	itte	ne
 8002ec8:	6850      	ldrne	r0, [r2, #4]
 8002eca:	1d00      	addne	r0, r0, #4
 8002ecc:	2004      	moveq	r0, #4
 8002ece:	f04f 0501 	mov.w	r5, #1
 8002ed2:	6800      	ldr	r0, [r0, #0]
 8002ed4:	2800      	cmp	r0, #0
 8002ed6:	bf14      	ite	ne
 8002ed8:	6803      	ldrne	r3, [r0, #0]
 8002eda:	2300      	moveq	r3, #0
 8002edc:	2902      	cmp	r1, #2
 8002ede:	bfa6      	itte	ge
 8002ee0:	6850      	ldrge	r0, [r2, #4]
 8002ee2:	3010      	addge	r0, #16
 8002ee4:	2004      	movlt	r0, #4
 8002ee6:	6800      	ldr	r0, [r0, #0]
 8002ee8:	2800      	cmp	r0, #0
 8002eea:	bf19      	ittee	ne
 8002eec:	6800      	ldrne	r0, [r0, #0]
 8002eee:	f100 0418 	addne.w	r4, r0, #24
 8002ef2:	2100      	moveq	r1, #0
 8002ef4:	f101 0418 	addeq.w	r4, r1, #24
 8002ef8:	f103 0108 	add.w	r1, r3, #8
 8002efc:	680a      	ldr	r2, [r1, #0]
 8002efe:	0a12      	lsrs	r2, r2, #8
 8002f00:	d01e      	beq.n	8002f40 <forward_rsqrt+0x84>
 8002f02:	684e      	ldr	r6, [r1, #4]
 8002f04:	eb06 0182 	add.w	r1, r6, r2, lsl #2
 8002f08:	4610      	mov	r0, r2
 8002f0a:	1f0f      	subs	r7, r1, #4
 8002f0c:	f010 0103 	ands.w	r1, r0, #3
 8002f10:	d006      	beq.n	8002f20 <forward_rsqrt+0x64>
 8002f12:	1e52      	subs	r2, r2, #1
 8002f14:	f857 c904 	ldr.w	ip, [r7], #-4
 8002f18:	1e49      	subs	r1, r1, #1
 8002f1a:	fb0c f505 	mul.w	r5, ip, r5
 8002f1e:	d1f8      	bne.n	8002f12 <forward_rsqrt+0x56>
 8002f20:	0880      	lsrs	r0, r0, #2
 8002f22:	d00d      	beq.n	8002f40 <forward_rsqrt+0x84>
 8002f24:	eb06 0182 	add.w	r1, r6, r2, lsl #2
 8002f28:	3910      	subs	r1, #16
 8002f2a:	68ca      	ldr	r2, [r1, #12]
 8002f2c:	688e      	ldr	r6, [r1, #8]
 8002f2e:	684f      	ldr	r7, [r1, #4]
 8002f30:	4372      	muls	r2, r6
 8002f32:	f851 6910 	ldr.w	r6, [r1], #-16
 8002f36:	437a      	muls	r2, r7
 8002f38:	4372      	muls	r2, r6
 8002f3a:	4355      	muls	r5, r2
 8002f3c:	1e40      	subs	r0, r0, #1
 8002f3e:	d1f4      	bne.n	8002f2a <forward_rsqrt+0x6e>
 8002f40:	699e      	ldr	r6, [r3, #24]
 8002f42:	68b0      	ldr	r0, [r6, #8]
 8002f44:	6822      	ldr	r2, [r4, #0]
 8002f46:	eb00 0185 	add.w	r1, r0, r5, lsl #2
 8002f4a:	1f0f      	subs	r7, r1, #4
 8002f4c:	6891      	ldr	r1, [r2, #8]
 8002f4e:	eb01 0385 	add.w	r3, r1, r5, lsl #2
 8002f52:	1f1c      	subs	r4, r3, #4
 8002f54:	4287      	cmp	r7, r0
 8002f56:	d30e      	bcc.n	8002f76 <forward_rsqrt+0xba>
 8002f58:	ed97 0a00 	vldr	s0, [r7]
 8002f5c:	f003 f8d2 	bl	8006104 <ai_math_sqrt>
 8002f60:	eef7 0a00 	vmov.f32	s1, #112	; 0x3f800000  1.0
 8002f64:	eec0 0a80 	vdiv.f32	s1, s1, s0
 8002f68:	edc4 0a00 	vstr	s1, [r4]
 8002f6c:	1f3f      	subs	r7, r7, #4
 8002f6e:	68b0      	ldr	r0, [r6, #8]
 8002f70:	1f24      	subs	r4, r4, #4
 8002f72:	4287      	cmp	r7, r0
 8002f74:	d2f0      	bcs.n	8002f58 <forward_rsqrt+0x9c>
 8002f76:	b001      	add	sp, #4
 8002f78:	bdf0      	pop	{r4, r5, r6, r7, pc}
	...

08002f7c <nl_func_sin_array_f32>:
 8002f7c:	b570      	push	{r4, r5, r6, lr}
 8002f7e:	688c      	ldr	r4, [r1, #8]
 8002f80:	6880      	ldr	r0, [r0, #8]
 8002f82:	eb04 0182 	add.w	r1, r4, r2, lsl #2
 8002f86:	1f0d      	subs	r5, r1, #4
 8002f88:	eb00 0182 	add.w	r1, r0, r2, lsl #2
 8002f8c:	1f0e      	subs	r6, r1, #4
 8002f8e:	42a5      	cmp	r5, r4
 8002f90:	f0c0 800a 	bcc.w	8002fa8 <nl_func_sin_array_f32+0x2c>
 8002f94:	ed95 0a00 	vldr	s0, [r5]
 8002f98:	f007 fd54 	bl	800aa44 <sinf>
 8002f9c:	ed86 0a00 	vstr	s0, [r6]
 8002fa0:	1f2d      	subs	r5, r5, #4
 8002fa2:	1f36      	subs	r6, r6, #4
 8002fa4:	42a5      	cmp	r5, r4
 8002fa6:	d2f5      	bcs.n	8002f94 <nl_func_sin_array_f32+0x18>
 8002fa8:	bd70      	pop	{r4, r5, r6, pc}
	...

08002fac <forward_sin>:
 8002fac:	b5f0      	push	{r4, r5, r6, r7, lr}
 8002fae:	b081      	sub	sp, #4
 8002fb0:	6942      	ldr	r2, [r0, #20]
 8002fb2:	8811      	ldrh	r1, [r2, #0]
 8002fb4:	2900      	cmp	r1, #0
 8002fb6:	bf1a      	itte	ne
 8002fb8:	6850      	ldrne	r0, [r2, #4]
 8002fba:	1d00      	addne	r0, r0, #4
 8002fbc:	2004      	moveq	r0, #4
 8002fbe:	f04f 0501 	mov.w	r5, #1
 8002fc2:	6800      	ldr	r0, [r0, #0]
 8002fc4:	2800      	cmp	r0, #0
 8002fc6:	bf14      	ite	ne
 8002fc8:	6803      	ldrne	r3, [r0, #0]
 8002fca:	2300      	moveq	r3, #0
 8002fcc:	2902      	cmp	r1, #2
 8002fce:	bfa6      	itte	ge
 8002fd0:	6850      	ldrge	r0, [r2, #4]
 8002fd2:	3010      	addge	r0, #16
 8002fd4:	2004      	movlt	r0, #4
 8002fd6:	6800      	ldr	r0, [r0, #0]
 8002fd8:	2800      	cmp	r0, #0
 8002fda:	bf19      	ittee	ne
 8002fdc:	6800      	ldrne	r0, [r0, #0]
 8002fde:	f100 0418 	addne.w	r4, r0, #24
 8002fe2:	2100      	moveq	r1, #0
 8002fe4:	f101 0418 	addeq.w	r4, r1, #24
 8002fe8:	f103 0108 	add.w	r1, r3, #8
 8002fec:	680a      	ldr	r2, [r1, #0]
 8002fee:	0a12      	lsrs	r2, r2, #8
 8002ff0:	d01e      	beq.n	8003030 <forward_sin+0x84>
 8002ff2:	684e      	ldr	r6, [r1, #4]
 8002ff4:	eb06 0182 	add.w	r1, r6, r2, lsl #2
 8002ff8:	4610      	mov	r0, r2
 8002ffa:	1f0f      	subs	r7, r1, #4
 8002ffc:	f010 0103 	ands.w	r1, r0, #3
 8003000:	d006      	beq.n	8003010 <forward_sin+0x64>
 8003002:	1e52      	subs	r2, r2, #1
 8003004:	f857 c904 	ldr.w	ip, [r7], #-4
 8003008:	1e49      	subs	r1, r1, #1
 800300a:	fb0c f505 	mul.w	r5, ip, r5
 800300e:	d1f8      	bne.n	8003002 <forward_sin+0x56>
 8003010:	0880      	lsrs	r0, r0, #2
 8003012:	d00d      	beq.n	8003030 <forward_sin+0x84>
 8003014:	eb06 0182 	add.w	r1, r6, r2, lsl #2
 8003018:	3910      	subs	r1, #16
 800301a:	68ca      	ldr	r2, [r1, #12]
 800301c:	688e      	ldr	r6, [r1, #8]
 800301e:	684f      	ldr	r7, [r1, #4]
 8003020:	4372      	muls	r2, r6
 8003022:	f851 6910 	ldr.w	r6, [r1], #-16
 8003026:	437a      	muls	r2, r7
 8003028:	4372      	muls	r2, r6
 800302a:	4355      	muls	r5, r2
 800302c:	1e40      	subs	r0, r0, #1
 800302e:	d1f4      	bne.n	800301a <forward_sin+0x6e>
 8003030:	6998      	ldr	r0, [r3, #24]
 8003032:	6886      	ldr	r6, [r0, #8]
 8003034:	6821      	ldr	r1, [r4, #0]
 8003036:	eb06 0085 	add.w	r0, r6, r5, lsl #2
 800303a:	1f07      	subs	r7, r0, #4
 800303c:	6888      	ldr	r0, [r1, #8]
 800303e:	eb00 0285 	add.w	r2, r0, r5, lsl #2
 8003042:	1f14      	subs	r4, r2, #4
 8003044:	42b7      	cmp	r7, r6
 8003046:	d309      	bcc.n	800305c <forward_sin+0xb0>
 8003048:	ed97 0a00 	vldr	s0, [r7]
 800304c:	f007 fcfa 	bl	800aa44 <sinf>
 8003050:	ed84 0a00 	vstr	s0, [r4]
 8003054:	1f3f      	subs	r7, r7, #4
 8003056:	1f24      	subs	r4, r4, #4
 8003058:	42b7      	cmp	r7, r6
 800305a:	d2f5      	bcs.n	8003048 <forward_sin+0x9c>
 800305c:	b001      	add	sp, #4
 800305e:	bdf0      	pop	{r4, r5, r6, r7, pc}

08003060 <nl_func_sinh_array_f32>:
 8003060:	b570      	push	{r4, r5, r6, lr}
 8003062:	688c      	ldr	r4, [r1, #8]
 8003064:	6880      	ldr	r0, [r0, #8]
 8003066:	eb04 0182 	add.w	r1, r4, r2, lsl #2
 800306a:	1f0d      	subs	r5, r1, #4
 800306c:	eb00 0182 	add.w	r1, r0, r2, lsl #2
 8003070:	1f0e      	subs	r6, r1, #4
 8003072:	42a5      	cmp	r5, r4
